:020000040800F2
:10000000008000200567000845740008E1660008CC
:1000100047740008497400084B7400080000000091
:10002000000000000000000000000000D1C3000834
:100030004D7400080000000061C40008A5C4000859
:100040004F74000851740008537400085574000878
:100050005774000859740008D9730008DF7300084A
:10006000E5730008EB730008F17300085B74000887
:100070005D7400085F740008617400086374000810
:100080006574000867740008697400086B740008E0
:100090006D7400086F74000871740008F77300082D
:1000A0007374000875740008777400087974000888
:1000B0007B740008C97A00087D7400087F7400080A
:1000C0008174000883740008857400088774000830
:1000D00089740008757B0008BD7F00088B740008D8
:1000E0001B740008C17400088D7400088F74000828
:1000F00091740008000000000000000000000000F3
:1001000000000000000000005FF808F110B5054C89
:10011000237833B9044B13B10448AFF300800123B3
:10012000237010BD1006002000000000F8E901084F
:1001300008B5034B1BB103490348AFF3008008BD6A
:100140000000000014060020F8E90108704710B50F
:100150000446442115F044FC204610BD8168014846
:1001600009F0DEBFA4AA0108FF2110B5044618302B
:1001700006F09EF8A168E0B90F4809F0D1FFA16828
:100180000E4809F0CDFF2069002103681B689847DD
:10019000012203210A4806F097FF20690021036825
:1001A0005B689847BDE8104001220221044806F030
:1001B0008BBF0448E1E700BFB3AA01080DAB0108FB
:1001C00000000240E5AA010813B50F4B0F491A6859
:1001D0000988914213D90E4A11681A68541C1C6090
:1001E00088541B680B4B1C680DF02CFA0023024648
:1001F0000721204600930EF0EBF802B010BD06492F
:100200000A8801320A80ECE77C0600208006002084
:10021000780600203006002082060020024B19607C
:10022000024B1A80704700BF78060020800600202D
:10023000014B1868704700BF7C0600202DE9F04193
:10024000174C06462368092B28D92268154F023A15
:100250003968154815F0F8FA236805463868023BF6
:1002600018440AF05AF8854201460AD1012386F85B
:1002700040300023F06B1A46BDE8F04119460CF0FF
:10028000FDBA2A46094D0A4809F04AFF298811B1EA
:10029000084809F045FF002323602B80BDE8F0816A
:1002A0007C06002078060020040000208206002042
:1002B00027AB010845AB010870B504461F48204E26
:1002C0006060204886B0A0601F48C4E90312206027
:1002D0001946636104F1180004F1280505F0C4FF14
:1002E0000FCE0FC533680A212B60184B18480093B6
:1002F00000231A460EF04AF8164B012518604FF6F7
:10030000FF7341F221011A46CDE9005503A815F00B
:100310004BFA03AB03CB104A1B881060516013816A
:100320000021032228460CF085FAE06310B90B483F
:1003300009F0F6FE204606B070BD00BF71AB0108A3
:10034000DCAB01087BAB0108F8AB0108A503000892
:1003500081AB010830060020040000208BAB0108AF
:1003600010B50C4C03F092FA2368DB070FD400F1B0
:10037000580300F1440200F148010748FFF79CFFD1
:100380000123064A06490448236016F05BF9024837
:1003900010BD00BF2C060020340600200000002005
:1003A0004D01000808B5FFF7DBFFBDE80840FFF787
:1003B00045BF000010B50446C068084903685B6982
:1003C0009847E06804F1280103681B6898470023F8
:1003D000034A1360034A138010BD00BFC90100081F
:1003E0007C06002082060020C06810B50368074C18
:1003F0005B68984720460122022106F065FE2046F0
:10040000BDE810400122032106F05EBE000002405C
:1004100081F001021830082105F0F0BF81F00102DF
:100420001830022105F0EABF81F0010218300421E2
:1004300005F0E4BF81F001021830012105F0DEBFB4
:1004400010B5044681680F4809F06AFE04F11800EF
:1004500005F0C1FF002184F824002046FFF7E4FFE7
:1004600020460021FFF7DAFF20460021FFF7D0FFEA
:1004700020460121FFF7DEFF2046BDE810400021A5
:10048000FFF7D8BFA7AB010810B5044681681A482A
:1004900009F046FEA168194809F042FE20460121F4
:1004A000FFF7C8FF01212046FFF7B8FF4FF4967011
:1004B0000DF01AFA20460021FFF7B0FF0121204677
:1004C000FFF7B2FF4FF496700DF00EFA20460021B0
:1004D000FFF7AAFF01212046FFF79AFF4FF496701D
:1004E0000DF002FA20460021FFF792FF2046BDE8FA
:1004F00010400021FFF79EBFB1AB0108C1AB01085E
:1005000007F04ABE10B50446406C10B1042115F046
:1005100067FA204610BD10B50446006810B10121ED
:1005200015F05EFA204610BD2DE9F0410025069F2A
:10053000C0E90112C0E903353946C0E90555C0E9F3
:100540000755057045620446164600F11C0813F075
:1005500055FB38B93146074809F0E2FD202106482D
:1005600006F02CF83A464146204613F013FB20468D
:10057000BDE8F08110AC01087DDF010830B58DB019
:1005800014F054FC044603F081F9214603F078FC92
:100590002E4B2F4A0321009302A82E4BFFF7C4FFD6
:1005A00002A9204614F0EEFA09A8FFF7B4FF06A846
:1005B000FFF7B1FF284B294A0321009302A8284BDB
:1005C000FFF7B2FF02A9204614F0DCFA09A8FFF7F2
:1005D000A2FF06A8FFF79FFF02220023214D0392EE
:1005E000214A012102A8CDE90523CDE90733CDE950
:1005F00009338DF8083004950B9313F0A7F938B937
:1006000029461A4809F08CFD2021194805F0D6FF2B
:10061000012209A902A813F07BF902A9204614F0CF
:10062000B1FA09A8FFF777FF06A8FFF774FF204685
:10063000104B114A114914F069FB00F0B9FD052275
:1006400021460DB0BDE8304003F02EBC65AC01087A
:1006500073AC01083BAC0108D9AC0108D0AC01086F
:100660007CAC010803AD010811AD010810AC010814
:100670007DDF01080105000834AD010858AD01080F
:100680002DE9F74FD0E9008AAAEB0804A410B4F5CD
:10069000705F07460E469346894602D1224815F000
:1006A00063F9012C234638BF0123E418A1EB0803AA
:1006B0001ED204B3B4F5705F28BF4FF47054A0008D
:1006C000019309F0C9FD0546019BDBF80020EA50C3
:1006D00043462A1F9E4210D1331DA3EB08032B442F
:1006E0001A46D1450ED059F8041B42F8041BF8E70E
:1006F0004FF47054E3E72546E7E753F8041B42F84C
:10070000041FE7E7A9EB06061E44B8F1000F03D06B
:100710000421404615F064F905EB8404C7E900564E
:10072000BC6003B0BDE8F08F5EAD01082DE9F04379
:1007300091B014F07BFB584F06463D68574C15F0BE
:1007400001051AD120461A22294640F8045B17F009
:10075000C1FC1A22294604F12400256217F0BAFCD4
:10076000012320464E4A4F49C4E91055C4E91255A9
:10077000A4F850503B6015F065FF94F851301BB160
:100780001D21494805F01AFF0027484D30468DF8D5
:100790001F7013F099FE304605F050FB2B1F3046BA
:1007A00043490DF11F02009514F076F8414808AA5C
:1007B00005F120012062089709F09CFA089B1BB103
:1007C0008521394805F0FAFE30463B4914F00BF814
:1007D00005463A4FDFF8E880DFF8E8902064ADB1D5
:1007E0000EAB03930DAB02930CAB01930BAB0093D9
:1007F000394628460AAB09AA18F038FC06281FD04B
:10080000314809F08DFC01238DF81F3001230222AD
:100810003046CDE900322D492D4B0DF11F0213F06A
:10082000FBFF9DF81F302BB12A4809F079FC1020FE
:1008300007F0ADFC012384F8513011B0BDE8F0831E
:100840000D2017F0F1FB0F9008B92348D9E70E9B54
:100850000D2104930D9B424603930C9B02930B9B2B
:1008600001930A9B0093099B18F0ACFBD4E9121387
:1008700099420BD00F9B41F8043BA1642C212846E0
:1008800018F063FC0028C1D0451CA8E748460FAA11
:10089000FFF7F6FEF2E700BF84060020880600207E
:1008A00000000020050500087DDF01088C060020FF
:1008B00073AC010878AD0108D0AC010884AD010823
:1008C000FAAD0108CC06002096AD010803AD010881
:1008D000D806002013AE0108E6AD01082DE9F0416D
:1008E000FFF73EFD04460121FFF7A4FD2046FFF778
:1008F00061FD0CF0A1FE4EF65F27364E4FF47A7183
:100900003368C01AB842E06B22D80CF0A5F9DFF8C2
:10091000C8802046FFF78CFC0546D0BB0CF08CFE4F
:100920003368C01AB84234D8404609F0F9FB0121B7
:100930002046FFF773FDC8200CF0D6FF294620465D
:10094000FFF76CFD4FF47A71E06B0CF085F9E0E78E
:100950000CF082F90525204F2046FFF769FC06467A
:10096000B8B9013D15F0FF0513D0384609F0D8FBA2
:1009700001212046FFF752FDC8200CF0B5FF31469B
:100980002046FFF74BFD4FF47A71E06B0CF064F9F1
:10099000E2E72046FFF728FD20460021FFF74AFD49
:1009A0002046FFF745FC90B101212046FFF73CFDB2
:1009B0000A4809F0B5FB41F288300CF095FF0021A0
:1009C0002046FFF731FD064B1878BDE8F081054B56
:1009D000FAE700BFE406002026AE01084EAE01088B
:1009E000C41C0020C21C002070B52F4809F098FBE1
:1009F000FFF7B6FC2D4B04461A7862B100250121A1
:100A00001D70FFF705FD41F288300CF06DFF29469F
:100A10002046FFF7FDFC02F039FF036E60301B68D3
:100A20009847234B234EC3E9820101212046FFF75B
:100A300001FD2046FFF7BEFC41F28831E06B0CF06F
:100A40000BF92046FFF7D0FC00212046FFF7F2FC0F
:100A50002046FFF7EDFB054680B9174809F060FB1B
:100A600001212046FFF7DAFC4FF496700CF03CFFB2
:100A700029462046FFF7D2FC307870BD0121204680
:100A8000FFF7D2FC4FF496700CF02EFF00212046A9
:100A9000FFF7CAFC2046FFF7CBFB0849024608488F
:100AA00009F0B4FBE8E700BF5EAE010818000020C3
:100AB00020000020C01C002026AE010808080020ED
:100AC00072AE010810B9034809F02ABB03C809F047
:100AD0008DBB00BF85AE010810B9264809F020BBC8
:100AE0000178406801F07002502A01F00F0328D00D
:100AF00006D8A2B1402A0AD002681F4809F010BBEC
:100B0000602AF9D1012B0CD101781C4805E01C4961
:100B10001C4B002808BF19461B4809F001BBFFF712
:100B2000D1BF022B02D101881848F6E7042B02D16D
:100B300001881748F1E7082B01680CBF15481648D3
:100B4000EBE7012B03D190F900101448E5E7022BE5
:100B500003D1B0F900101248DFE7042B03D1B0F93C
:100B600000101048D9E7082B01680CBF0E480F4849
:100B7000D3E700BF95AE010816AF01089BAE010890
:100B80008AAE01088FAE0108C6B00108A7AE010801
:100B9000B4AE0108C1AE0108CFAE0108DBAE01085A
:100BA000E6AE0108F2AE0108FEAE01080BAF010887
:100BB00070B50020002105F01BF904460F4D104EC2
:100BC000C4B16179802911D122792168306813F08C
:100BD0002DFC204605F044FA2046082114F000FFC1
:100BE0000020002105F004F90446E9E7284609F051
:100BF00097FAEEE7034B187870BD00BF32AF0108DB
:100C0000081C0020C01C002008B502F03FFEBDE813
:100C1000084002F083BE0000F8B5414809F080FAB0
:100C2000FFF79EFB04460121FFF704FC2046FFF777
:100C3000C1FB41F28831E06B0CF00EF82046FFF763
:100C4000D3FB00212046FFF7F5FB2046FFF7F0FA23
:100C5000054600283DD1334809F062FA01212046BB
:100C6000FFF7DCFB4FF47A700CF03EFE294620467D
:100C7000FFF7D4FB2C4B1D702C4809F051FA2C4D7A
:100C800094F824202B4F284E002A14BF3A462A46B7
:100C9000294B2A492A4809F043FA3278264B002A80
:100CA00014BF3A462A462749254809F039FA264B07
:100CB00094F824102548002914BF1946294609F044
:100CC0002FFA234809F02CFA33783BB3214B1878DC
:100CD000F8BD214809F024FA0025204E204F204677
:100CE000FFF7A6FAA84206D9384616F8011B09F004
:100CF00017FA0135F3E71B4809F012FA01212046E3
:100D0000FFF792FB4FF47A700CF0EEFD00212046C5
:100D1000FFF78AFB0122044B1A70ADE7124BD6E7AE
:100D20005EAE010826AE01080C1C002055AF01087C
:100D30004DAF010848AF01087DDF010836B7010853
:100D400065AF01087CAF010852AF010882AF01080E
:100D500097AF0108C41C002072AE010808080020EB
:100D6000F4D401087CDF0108C21C00201FB56123F8
:100D7000CDE9013101A9039203F05AFF05B05DF8F6
:100D800004FB07B58DF8041001A98DF805208DF836
:100D9000063003F0F9FF03B05DF804FB70B5114EA7
:100DA000346814F001041BD10F4D1A222846214645
:100DB00040F8044B17F08EF91A22214605F1240061
:100DC0002C6217F087F901232846084A0849C5E92B
:100DD0001044C5E91244A5F85040336015F032FCC8
:100DE000014870BD84060020880600200000002015
:100DF0000505000808B5FFF7D1FF90F851301BB981
:100E00003321034805F0DAFBFFF7C8FF08BD00BF38
:100E10007DDF01082DE9F04F87B00BF02BFC044675
:100E20000BF036FC21460246A24809F079F902F09F
:100E30002DFD04460BF01EFC05460BF029FC29464F
:100E400002469C4809F06CF99B4809F069F9FFF7E4
:100E500087FA05460146204615F084FB204615F02A
:100E60003DFB4FF4A05295492846FFF7D7F9944827
:100E700009F056F9FFF782FBFA200CF035FD13F06C
:100E8000EFFF13F021FBFFF751FC204615F03CFB70
:100E90008C4809F045F9FFF7ADFF8B4E05463368E6
:100EA0008A4C13F0010F04D103F0A8FE0123206047
:100EB0003360266802F0EAFC00F16001304603F07E
:100EC0007CFD2068824903F07AFD26682A68814902
:100ED00003A803F05BFD03A9304603F0B3FD2568CA
:100EE00000230F228DF806007B4903A803F024FDA0
:100EF00003A9284603F0A6FD784A8DF80700784933
:100F00002068FFF733FF774A834677492068FFF769
:100F10002DFF764A814676492068FFF727FF754AFC
:100F2000824675492068FFF721FF724A8DF802005A
:100F300072492068FFF71AFF70250026704B8DF864
:100F4000030003A9206803950493059603F070FE3F
:100F50006C4B03A98DF800002068CDE90436039599
:100F600003F066FE8DF80100206804F0BFFD6649BD
:100F70008046206804F0A4FD644A8DF804006449AA
:100F80002068FFF7F3FE07462068624A624980F84E
:100F900028B0FFF7EBFE614A054661492068FFF77C
:100FA000E5FE604E4B46594632788DF805002068C4
:100FB000FFF7E7FEDFF870B149469DF8033032785D
:100FC0002068FFF7DEFE4946DFF8609143469BF854
:100FD00000202068FFF7D5FE434699F800209DF8D1
:100FE00003102068FFF7CDFE3B464146327820686B
:100FF000FFF7C7FE5346394632782068FFF7C1FE37
:1010000039469DF801309BF800202068FFF7B9FEB3
:101010003B469DF807209DF801102068FFF7B1FEC0
:1010200051469DF8023099F800202068FFF7A9FE8C
:101030002B4699F800209DF802102068FFF7A1FECA
:101040003B4A29469DF8043020681278FFF799FE44
:101050009DF8053032789DF804102068FFF791FE66
:101060002B4699F800209DF805102068FFF789FEAF
:1010700029469DF8003032782068FFF782FE5346FB
:101080009DF806209DF800102068FFF77AFE206882
:1010900004F02EF8274809F043F8206801224FF4A5
:1010A000C87103F0BFFF002007B0BDE8F04F0CF09F
:1010B00081B900BFA5AF0108C4AF0108080800202E
:1010C000D8AF0108E9AF0108E0060020F0070020D2
:1010D000090C000806B001080FB00108391100081A
:1010E000B1BC0108190C00081FB00108E90900088B
:1010F00032B001087112000837B0010840B0010891
:1011000013BC010857B001086CBC0108DD080008D9
:1011100065B001083D15000871B00108B10B000869
:101120007AB00108C41C0020C21C0020C01C002092
:10113000C31C002089B0010870B5154C154808F093
:10114000EFFF2368DB0708D413F08AFE80220146F4
:10115000114812F095FE012323600F4A0F4B104DEA
:101160001A600CF069FA0F4B18600F4808F0D8FFAE
:10117000FFF740FED0E91146A64205D0284654F8B4
:10118000041B08F0CDFFF7E7084B187870BD00BFCF
:10119000DC060020A3B00108EC060020081C00209B
:1011A000C4B00108E4060020B6B00108C41C002049
:1011B00002F06CBBF8B54B6905460E46BBB11C7816
:1011C00014F0700204D0402A13D004F00F0403E09E
:1011D0005A685468F72C05D830684268062A0AD045
:1011E000204800E02048BDE8F84008F099BF1C46C0
:1011F000F2E70124F0E7D5F8F42104F10801C2F583
:10120000FA77B94201D91948EDE70168AF180868C3
:10121000A8508A88BA80D5F8F421D01D2A44C5F890
:10122000F401947172692844127812F0700F05BFAE
:101230005B6822462246196818BF596816F022FFDB
:10124000D5F8F42133691444C5F8F44103B11B788F
:10125000621CC5F8F4212B55D5F8F8310133C5F8D7
:10126000F831F8BDDFB00108CAB00108F1B00108DB
:101270002DE9F04F89B0FFF7BDFD00248146FFF74F
:101280006FF88F4F0546C7E97D44C7E97F44FEF7F5
:10129000CFFF102810D801212846FFF7BFF84FF4E0
:1012A00096700CF021FB21462846FFF7B7F8854BD6
:1012B000187809B0BDE8F08F2846FEF7B9FF10286E
:1012C00004D840F2EF11804805F078F90023CDE909
:1012D00005337E4B28460393FEF7AAFF103804908F
:1012E000DDE904329A4220D203A801F03CFD20B986
:1012F000012103A801F03FFDF2E703A801F05EFA27
:10130000044603A801F024FD08B30699DDE9043280
:101310006F4808F005FF6F4808F002FFDDE904138D
:101320000398C91A184408F061FFD7E97D216A487B
:1013300008F0F6FE01212846FFF776F84FF4967084
:101340000CF0D2FA00212846FFF76EF8AFE76348A9
:1013500008F0E6FE63686248197808F0E1FEA368C9
:101360006048197808F0DCFE23695F48198808F0A6
:10137000D7FE5E4808F0D4FE2068FFF7A3FBE368C1
:101380005B481B68196808F0CBFEE3681B681A68A5
:1013900040F201739A4243D1564808F0C1FEE36817
:1013A000DFF854815B68DFF854A11E69DFF850B1A3
:1013B000002E35D033682BB1404608F0B1FE3068BE
:1013C000FFF780FB73682BB15A6850461278197882
:1013D00008F0A6FEB36813B1584608F0A1FEF36802
:1013E00023B11A784748114608F09AFE336923B1B1
:1013F00093F90010444808F093FE736933B14348F1
:10140000197808F08DFE7069FFF766FBB3692BB1A0
:101410003F4808F085FEB069FFF754FBF669C7E75F
:10142000E3681A68116840F2017291423CD15B682E
:10143000D9F844800093D9F84830DFF8D8B0019348
:10144000019A434642452FD0186801F0DCFA06465F
:10145000314808F065FE3046FFF734FB009B08F189
:101460000408D3F810A0BAF1000F21D0DAF8000078
:1014700060B9B6B9294808F053FEDAF81400FFF74E
:101480002BFB51460E48FFF795FE14E04EB1426823
:1014900071688A4205D13168006816F0E3FD0028C2
:1014A000E8D0DAF81CA0DEE7204601F06FF917E774
:1014B000584608F035FE304601F058FAC0E700BF44
:1014C00020000020C01C00207DDF01081008002043
:1014D00005B1010822B1010831B201082FB101089C
:1014E0003DB101084EB1010862B101086FB10108B8
:1014F00082B1010894B10108A9B10108B3B1010892
:10150000CCB10108DAB10108ECB10108FBB1010866
:101510000DB201084DB201081CB201085DB201080C
:10152000D0E97E329A423FBFD0F80032C0188079AD
:10153000083034BFC0B20020704700002DE9F04FE2
:1015400089B0FEF70DFF0446FFF754FC01218046E9
:101550002046FEF75DFF764D4FF496700CF0C4F90F
:1015600020460021FEF754FF2B685C6894B1714857
:1015700008F0D6FD2C6804F033FC6F49024604AB3A
:10158000204612F0D5FC6C4902469DF8100004F08C
:1015900013FC5CE006F0A6F8684A6D46D2E9003616
:1015A000B6F1004F08BF9C4207D0654FC31A61EBEC
:1015B00006069F4274EB06034EDA04ACC2E9000152
:1015C000604808F0ADFD14225F49204614F081F90F
:1015D00005F0E6F9074614F0E9FB0021064620462F
:1015E00014F0A2F90521204614F09EF902212046AC
:1015F00014F09AF90021204614F096F95349384620
:1016000015F03EFF16F028F901B2204614F09EF9BD
:101610003146204614F09AF994E80F0085E80F004F
:10162000284614F08EF90446E0B1494808F078FDE8
:10163000284614F084F90446284614F082F921461D
:10164000C2B2012004F0B8FB284614F07CF9414BEB
:10165000187809B0BDE8F08F10222146284616F010
:1016600039FDDDE73C4ED6E97E329A424DD004F09A
:10167000B7FB98F850308246022B2DD1D6E9822351
:101680002D4808F04EFE05244FF004083248FFF7BD
:1016900047FF00270546DFF8C4B0DFF8BC9055B31C
:1016A000AAEB0402D21B954219DD2FBB584608F065
:1016B00037FD4846FFF734FF48B1D6F8FC21013228
:1016C000C6F8FC21D6F800221044C6F800024846AD
:1016D000FFF726FF0546E2E74FF00308D6E7164B73
:1016E000D6F80012E01918442A46314416F0CAFC14
:1016F0007B19DFB2DDE747B13C442146184808F0CA
:101700000FFD40460C49E2B241E7164C23783BB14D
:10171000154808F005FD002207491046227036E7FB
:10172000124808F0FDFC04F077FE114B90E700BF73
:10173000081C00206BB20108FC06002010000020ED
:101740000851010081B20108F407002000007A442A
:10175000A0B20108C31C002020000020B5B201087F
:10176000C5B201088E1D0020DBB20108F2B20108EB
:10177000C41C002073B502F089F8036804469B6816
:1017800098470AF089FF05460AF086FF0126294698
:10179000002500F57052164808F0C2FC04F03CFE2B
:1017A0004FF496722B46CDE90065124912480BF0B2
:1017B0000BFD236831462046DB6898474FF4FA70EA
:1017C00005F054FA23682946DB68204698470B4801
:1017D00008F0A6FC0A4808F0A3FC0BF0DBFE40F280
:1017E0005631084804F0EAFE284602B070BD00BF3A
:1017F00008B3010821B30108150E00082AB3010837
:101800003DB301087DDF0108FF22014B1A707047CC
:10181000E806002010B5102008F01EFD0446102236
:10182000002116F057FC204610BD10B5044680B1CB
:10183000006801F09BF8606801F098F8A06801F07A
:1018400095F8E06801F077FD2046BDE8104008F00B
:10185000EDBC10BD38B50446FFF7DCFF0546204659
:1018600001F07BFA702806D00123E3602846FFF7D9
:10187000DCFF002528E0204601F04AFA0428F3D1D5
:10188000204601F080F82860204601F061FA002827
:10189000ECD1204601F077F86860204601F058FA54
:1018A0000028E3D1204601F06EF8A860204601F040
:1018B0004FFA0028DAD1204601F0E4FDE860204626
:1018C00001F046FA0028D1D1284638BD10B50446AB
:1018D000012008F0C1FC047010BD70B5044601F091
:1018E0004EFA30B9204601F038FA402803D00123DF
:1018F000E360002070BD204601F00AFA0128054689
:10190000F5D1204601F02FFA06462946204636B189
:1019100001F031FAFF20BDE87040FFF7D7BF01F0BA
:101920002AFA3046F7E708B108F080BC704708B5DE
:10193000042008F091FC0023036008BD10B50446A4
:1019400038B1006801F012F82046BDE8104008F0F8
:101950006DBC10BD38B50446FFF7E9FF05462046CB
:1019600001F0FBF9702806D00123E3602846FFF759
:10197000E5FF00250DE0204601F0CAF90128F3D16A
:10198000204601F000F82860204601F0E1F9002827
:10199000ECD1284638BD08B5042008F05DFC0023D2
:1019A000036008BD10B5044638B1006800F0DEFFE2
:1019B0002046BDE8104008F039BC10BD38B50446DB
:1019C000FFF7E9FF0546204601F0C7F9702806D069
:1019D0000123E3602846FFF7E5FF00250DE02046E0
:1019E00001F096F90128F3D1204600F0CCFF2860E1
:1019F000204601F0ADF90028ECD1284638BD10B5DD
:101A0000044698B1006800F0B1FF606800F0AEFFD6
:101A1000206900F0ABFFA06800F0A8FFE06800F0CC
:101A2000A5FF2046BDE8104008F000BC10BD38B549
:101A30000446142008F010FC14220021054616F07C
:101A400049FB204601F089F9702806D00123E360A4
:101A50002846FFF7D4FF002531E0204601F058F971
:101A60000528F3D1204600F08EFF2860204601F0C3
:101A70006FF90028ECD1204600F085FF6860204611
:101A800001F066F90028E3D1204600F07CFFA86051
:101A9000204601F05DF90028DAD1204600F073FFFE
:101AA000E860204601F054F90028D1D1204600F02A
:101AB0006AFF2861204601F04BF90028C8D128466A
:101AC00038BD10B51C2008F0C7FB04461C220021BD
:101AD00016F000FB204610BD10B50446C8B10068E2
:101AE00000F044FF606800F041FFA06800F03EFF96
:101AF000E06801F09BF9206900F0F2FC606900F0F9
:101B000035FFA06901F092F92046BDE8104008F0C9
:101B10008DBB10BD38B50446FFF7D3FF0546204600
:101B200001F01BF9702806D00123E3602846FFF777
:101B3000D3FF002543E0204601F0EAF80728F3D15F
:101B4000204600F020FF2860204601F001F900281F
:101B5000ECD1204600F017FF6860204601F0F8F84D
:101B60000028E3D1204600F00EFFA860204601F0D7
:101B7000EFF80028DAD1204601F067F9E860204646
:101B800001F0E6F80028D1D1204600F0B3FC28612E
:101B9000204601F0DDF80028C8D1204600F0F3FE11
:101BA0006861204601F0D4F80028BFD1204601F03A
:101BB0004CF9A861204601F0CBF80028B6D12846A0
:101BC00038BD10B5142008F047FB0446142200214C
:101BD00016F080FA204610BD10B5044698B1006892
:101BE00000F0C4FE606800F0C1FEA06800F0BEFE18
:101BF000E06801F075F9206900F0B8FE2046BDE804
:101C0000104008F013BB10BD38B50446FFF7D9FFEC
:101C10000546204601F0A1F8702806D00123E360B4
:101C20002846FFF7D9FF002531E0204601F070F883
:101C30000528F3D1204600F0A6FE2860204601F0DA
:101C400087F80028ECD1204600F09DFE6860204611
:101C500001F07EF80028E3D1204600F094FEA86051
:101C6000204601F075F80028DAD1204601F053F93A
:101C7000E860204601F06CF80028D1D1204600F041
:101C800082FE2861204601F063F80028C8D128466A
:101C900038BD08B50C2008F0DFFA0022026042606F
:101CA000826008BD10B5044668B1006800F05EFEB1
:101CB000606801F015F9A06801F03DFB2046BDE821
:101CC000104008F0B3BA10BD38B50446FFF7E1FF85
:101CD0000546204601F041F8702806D00123E36054
:101CE0002846FFF7DFFF00251FE0204601F010F82F
:101CF0000328F3D1204600F046FE2860204601F07C
:101D000027F80028ECD1204601F005F9686020464C
:101D100001F01EF80028E3D1204601F0B3FBA860D3
:101D2000204601F015F80028DAD1284638BD10B554
:101D3000242008F091FA04462422002116F0CAF962
:101D4000204610BD10B50446F8B1006800F00EFE44
:101D5000606801F06BF8A06800F0EDFDE06801F04C
:101D6000BFF8206901F062F8606900F0E4FDA06945
:101D700000F0E2FAE06900F0F9FD206A00F0F6FDFB
:101D80002046BDE8104008F051BA10BD38B50446F1
:101D9000FFF7CDFF0546204600F0DFFF702807D093
:101DA00001232846E360FFF7CDFF0025284638BD14
:101DB000204600F0ADFF0928F2D1204600F0E3FDF7
:101DC0002860204600F0C4FF0028E9D1204601F039
:101DD0003CF86860204600F0BBFF0028E0D10422F8
:101DE0006021204600F060FDA860204600F0B0FFB2
:101DF0000028D5D1204601F08EF8E860204600F09A
:101E0000A7FF0028CCD1204601F01FF8286120460A
:101E100000F09EFF0028C3D108226021204600F078
:101E200043FD6861204600F093FF0028B8D12046AA
:101E30000E4A0F4900F0A9FAA861204600F088FF79
:101E40000028ADD1204600F09EFDE861204600F05C
:101E50007FFF0028A4D1204600F095FD286220468F
:101E600000F076FF0028A1D09AE700BFAF3200084B
:101E70006F33000810B5242008F0EEF90446242240
:101E8000002116F027F9204610BD70B5044638B37E
:101E9000006800F06BFD606800F068FDA06800F06D
:101EA00065FDE068FFF73FFD206900F0BFFF606956
:101EB00000F0BCFFA06901F013F8E56945B12E46BA
:101EC00030686D6800F052FD304608F0AFF9F5E774
:101ED000206A01F030FA2046BDE8704008F0A6B94B
:101EE00070BD2DE9F8430446FFF7C4FF05462046C0
:101EF00000F033FF702806D00123E3602846FFF787
:101F0000C4FF002550E0204600F002FF0928F3D16D
:101F1000204600F038FD2860204600F019FF002818
:101F2000ECD1204600F02FFD6860204600F010FF45
:101F30000028E3D1204600F026FDA860204600F0EE
:101F400007FF0028DAD12046FFF7C7FCE8602046EB
:101F500000F0FEFE0028D1D1204600F076FF286177
:101F6000204600F0F5FE0028C8D1204600F06DFFA5
:101F70006861204600F0ECFE0028BFD1204600F04A
:101F8000CAFFA861204600F0E3FE0028B6D1204633
:101F900000F0F5FE58B1204601F074FA28622046A0
:101FA00000F0D6FE0028A9D12846BDE8F8832046D7
:101FB00000F0D3FE70289FD1204600F0A9FE4FF01C
:101FC00000080746C146002FE5DD082008F044F967
:101FD0000646C0F80090C0F80490204600F0D3FCFC
:101FE0003060204600F0B4FE002887D1EB691BB9B1
:101FF000EE61B046013FE6E7C8F80460F9E710B5C6
:10200000044668B1006800F0B1FC606800F093FC21
:10201000A06800F090FC2046BDE8104008F006B92A
:1020200010BD10B5044680B1006800F0FFFE606886
:1020300000F081FCA06800F07FF9E06800F096FCF9
:102040002046BDE8104008F0F1B810BD10B50446B8
:1020500050B1006801F069FA606800F087FC204622
:10206000BDE8104008F0E2B810BD10B5202008F01F
:10207000F3F804462022002116F02CF8204610BD6B
:1020800010B50446E0B1006800F070FC606800F034
:10209000CDFEA06800F04FFCE06800F021FF206951
:1020A00000F04AF9606900F047F9A06900F05EFCB1
:1020B000E06900F05BFC2046BDE8104008F0B6B8CF
:1020C00010BD000038B50446FFF7CFFF0546204697
:1020D00000F043FE702807D001232846E360FFF795
:1020E000CFFF0025284638BD204600F011FE082805
:1020F000F2D1204600F047FC2860204600F028FE80
:102100000028E9D1204600F0A0FE6860204600F0DB
:102110001FFE0028E0D104226021204600F0C4FB0D
:10212000A860204600F014FE0028D5D1204600F01B
:10213000F2FEE860204600F00BFE0028CCD12046DD
:10214000134A144900F021F92861204600F000FEEE
:102150000028C1D12046104A104900F016F96861E4
:10216000204600F0F5FD0028B6D1204600F00BFC1B
:10217000A861204600F0ECFD0028ADD1204600F01B
:1021800002FCE861204600F0E3FD0028AAD0A3E7A6
:10219000FF1F0008B321000823200008392200088F
:1021A00008B50C2008F058F80022026042608260F6
:1021B00008BD38B50446FFF7F3FF0546204600F09A
:1021C000CCFD702807D001232846E360FFF717FFF6
:1021D0000025284638BD204600F09AFD0328F2D19C
:1021E000204600F0D0FB2860204600F0B1FD00281A
:1021F000E9D101226021204600F056FB68602046AC
:1022000000F0A6FD0028DED101225021204600F07A
:102210004BFBA860204600F09BFD0028D9D0D2E7F8
:1022200010B5102008F018F804461022002115F00F
:1022300051FF204610BD000038B50446FFF7F0FFFF
:102240000546204600F089FD702807D00123284666
:10225000E360FFF7E6FE0025284638BD204600F083
:1022600057FD0428F2D1204600F0EFFD28602046FB
:1022700000F06EFD0028E9D108226021204600F020
:1022800013FB6860204600F063FD0028DED1204685
:10229000094A0A4900F079F8A860204600F058FD84
:1022A0000028D3D1204600F06EFBE860204600F005
:1022B0004FFD0028D0D0C9E74D200008D1220008EA
:1022C00008B5082007F0C8FF00220260426008BD80
:1022D00038B50446FFF7F4FF0546204600F03DFD03
:1022E000702807D001232846E360FFF7AFFE0025E2
:1022F000284638BD204600F00BFD0228F2D12046CA
:1023000001F029F92860204600F022FD0028E9D1DB
:10231000204600F038FB6860204600F019FD0028D8
:10232000E6D0DFE710B504460C2007F095FF002249
:1023300002604260846010BD38B5044688B938BD7B
:1023400050F82500A36898470135D4E900039D4261
:10235000F6DB08B107F06AFF2046BDE8384007F019
:1023600065BF0025F1E738B5436804460133436093
:102370000D460068990016F0B3FD6368206003F114
:102380008043013B40F8235038BD2DE9F843054612
:102390008846164600F0E1FC70281AD13046FFF757
:1023A000C1FF0446284600F0B3FC00270646B742AA
:1023B00002DB2046BDE8F8832846C0478146284610
:1023C00000F0C6FC28B949462046FFF7CCFF01378C
:1023D000EDE701232046EB60FFF7AEFF0024E8E7BE
:1023E00010B5202007F038FF04462022002115F008
:1023F00071FE204610BD38B5044600F0AEFC7028D2
:1024000004D001230025E360284638BD204600F0B3
:102410007FFC0728F5D1FFF7E3FF0546204600F0D3
:10242000B2FA2860204600F093FC0028E9D120464B
:1024300000F0C3FC6860204600F08AFC0028E0D170
:10244000204600F002FDA860204600F081FC002834
:10245000D7D101226021204600F026FAE86020460C
:1024600000F076FC0028CCD101225021204600F05B
:102470001BFA2861204600F06BFC0028C1D12046E1
:1024800001F069F86861204600F062FC0028B8D1CC
:10249000204600F078FAA861204600F059FC002898
:1024A000B2D0AEE710B50446C8B1006800F05EFADD
:1024B000606800F076FCA06800F0B8FCE06800F00E
:1024C0003AFA206900F037FA606901F02EF8A06945
:1024D00000F04CFA2046BDE8104007F0A7BE10BD42
:1024E00010B530B1C469FFF7DDFF14B12046E469CF
:1024F000F9E710BDF8B5054600F041FC044608B107
:10250000002406E0284600F028FC702803D00123B0
:10251000EB602046F8BD284600F0FAFB061EEFDD12
:102520002846FFF768FF0446284600F011FC70B902
:102530002746013E002EECD02846FFF75CFFF861ED
:10254000284600F005FC10B9FF69013EF2E70123BF
:102550002046EB60FFF7C4FFD2E7000038B5054620
:10256000082007F079FE00230446036043602846F4
:1025700000F0F3FB702806D00123EB60204607F043
:1025800055FE002459E0284600F0C2FB0228F3D192
:1025900004226021284600F087F92060284600F0D8
:1025A000D7FB0028EAD12368196840F20143994219
:1025B00055D020D840F20123994248D00DD840F29E
:1025C000011399423BD0B1F5007F3CD0B1F5807F3B
:1025D0002FD02D4816F000FC2FE040F20133994235
:1025E00039D0B1F5806F02D0B1F5407FF1D12846E6
:1025F000FFF777FC20E0B1F5E06F3CD00DD840F25A
:10260000015399422FD0B1F5C06F30D0B1F5A06F12
:10261000DFD12846FFF7F8FA0EE040F20173994245
:102620002DD04FF601739942D3D12846FFF712F906
:1026300002E0284600F035FA6060204638BD2846A2
:1026400000F0AEFAF8E72846FFF784F9F4E72846E9
:10265000FFF7B4F9F0E72846FFF734FDECE728462A
:10266000FFF794FBE8E72846FFF72EFBE4E7284650
:1026700000F009FBE0E72846FFF7D9F9DCE7284638
:10268000FFF748FAD8E700BF6EB3010810B504465B
:10269000002875D003681A6840F201439A425BD063
:1026A00021D840F201239A424ED00ED840F20113B5
:1026B0009A4241D0B2F5007F42D0B2F5807F30D04F
:1026C0003049314816F088FB2EE040F201339A423F
:1026D0003ED0B2F5806F02D0B2F5407FF0D1606895
:1026E000FFF7D3FB20E0B2F5E06F41D00DD840F208
:1026F00001539A4234D0B2F5C06F35D0B2F5A06F15
:10270000DED14068FFF768FA0EE040F201739A42AA
:1027100032D04FF601739A42D2D14068FFF785F864
:1027200002E0406800F09FF9206800F004F92046BC
:10273000BDE8104007F07ABD406800F016FAF3E7F4
:102740004068FFF7FBF8EFE74068FFF72BF9EBE78E
:102750004068FFF795FCE7E74068FFF7F3FAE3E727
:102760004068FFF79FFADFE7406800F074FADBE7A4
:102770004068FFF744F9D7E74068FFF7ADF9D3E7C2
:1027800010BD00BFBBB301089CB3010810B50446DF
:1027900098B1006800F0EAF8606800F0CCF8A06832
:1027A00000F0C9F8E068FFF771FF206900F0C3F896
:1027B0002046BDE8104007F039BD10BD38B50446CD
:1027C000142007F049FD14220021054615F082FC73
:1027D000204600F0C2FA702806D00123E3602846A4
:1027E000FFF7D4FF00253FE0204600F091FA0628CD
:1027F000F3D1204600F0C7F82860204600F0A8FA80
:102800000028ECD101226021204600F04DF86860DC
:10281000204600F09DFA0028E1D1012260212046E7
:1028200000F042F8A860204600F092FA0028D6D1C5
:102830002046FFF793FEE860204600F089FA002862
:10284000CDD102226021204600F02EF828612046DA
:1028500000F07EFA0028C2D1204600F084FA18B9B0
:102860000121204600F087FA284638BDB0B504465D
:102870000D46CB1D23F0070300AFADEB030D0A4659
:102880000146684615F0FEFB631E0DEB0502C4F120
:102890000104E1188D4202F1FF3201DCBD46B0BDFA
:1028A000117803F8011FF4E72DE9F04705460C46BF
:1028B000904600F064FA064638B9284600F04DFA12
:1028C000A042814603D00123EB60002430E028467B
:1028D00000F01EFA071EF6DB4745F4DC404607F021
:1028E000BBFC31464246044615F0F4FB284600F096
:1028F0003AFAB9F1500F08BFC0F3C016284600F0ED
:1029000036FAA8EB070904EB090A01463A46504695
:1029100015F0B8FB26B14A46FF21204615F0DAFB38
:1029200041462046FFF7A2FF3946284600F023FA29
:102930002046BDE8F08708B107F078BC704770B555
:10294000064608200D4607F087FC00239D420446FA
:102950000360436008DD284607F07EFC2A463146C6
:10296000206015F08FFB6560204670BD10B50446F1
:1029700040B1006808B107F059FC2046BDE810409E
:1029800007F054BC10BD70B5044600F0F8F928B942
:10299000204600F0E2F918B10123E36000250FE0C2
:1029A000204600F0B5F9061EF6DB204600F0DFF900
:1029B0003146FFF7C4FF31460546204600F0DBF9FB
:1029C000284670BD03463038C0B209280DD9A3F19E
:1029D0006102052A02D8573BD8B27047A3F14102E1
:1029E000052A01D8373BF7E70020704710B50146AC
:1029F0000078FFF7E7FF04464878FFF7E3FF40EA77
:102A00000410C0B210BD2DE9F84300AF044616F023
:102A1000BBFBC3071AD44510EB1D23F00703ADEB36
:102A2000030DE8460DF1FF3604EB45094C4506D190
:102A300029464046FFF783FFBD46BDE8F8832046A0
:102A4000FFF7D4FF023406F8010FEFE70020F3E7A9
:102A500010B51C2007F000FC04461C22002115F0D4
:102A600039FB204610BD10B50446C8B10068FFF719
:102A70007DFF6068FFF77AFFA068FFF777FFE068E7
:102A8000FFF774FF2069FFF771FF6069FFF76EFFC2
:102A9000A069FFF750FF2046BDE8104007F0C6BB15
:102AA00010BD38B50446FFF7D3FF0546204600F0B9
:102AB00054F9702806D00123E3602846FFF7D3FFBE
:102AC000002545E0204600F023F90728F3D12046F1
:102AD000FFF759FF2860204600F03AF90028ECD1B2
:102AE0002046FFF750FF6860204600F031F90028CB
:102AF000E3D12046FFF747FFA860204600F028F901
:102B00000028DAD12046FFF73EFFE860204600F0BB
:102B10001FF90028D1D12046FFF735FF2861204654
:102B200000F016F90028C8D12046FFF72CFF686195
:102B3000204600F00DF90028BFD101226021204677
:102B4000FFF7B2FEA861204600F002F90028B4D1D8
:102B5000284638BD10B5182007F07EFB0446182221
:102B6000002115F0B7FA204610BD10B50446B0B1EB
:102B70000068FFF7FBFE6068FFF7F8FEA068FFF74C
:102B8000F5FEE068FFF7F2FE206900F04FF960699A
:102B9000FFF7D1FE2046BDE8104007F047BB10BD4F
:102BA00038B50446FFF7D6FF0546204600F0D5F8B5
:102BB000702806D00123E3602846FFF7D6FF0025E2
:102BC0003CE0204600F0A4F80628F3D12046FFF7A9
:102BD000DAFE2860204600F0BBF80028ECD1204641
:102BE000FFF7D1FE6860204600F0B2F80028E3D17C
:102BF0002046FFF7C8FEA860204600F0A9F800288C
:102C0000DAD12046FFF7BFFEE860204600F0A0F8CA
:102C10000028D1D1204600F018F92861204600F0A4
:102C200097F80028C8D1012260212046FFF73CFE1A
:102C30006861204600F08CF80028BDD1284638BDD8
:102C400010B5142007F008FB04461422002115F0EB
:102C500041FA204610BD10B5044698B10068FFF750
:102C600085FE6068FFF782FEA068FFF77FFEE068E0
:102C700000F036F9206900F05EFB2046BDE8104008
:102C800007F0D4BA10BD38B50446FFF7D9FF0546A2
:102C9000204600F062F8702806D00123E360284641
:102CA000FFF7D9FF002531E0204600F031F8052874
:102CB000F3D12046FFF767FE2860204600F048F871
:102CC0000028ECD12046FFF75EFE6860204600F049
:102CD0003FF80028E3D12046FFF755FEA8602046C4
:102CE00000F036F80028DAD1204600F014F9E86048
:102CF000204600F02DF80028D1D1204600F0C2FB7C
:102D00002861204600F024F80028C8D1284638BDA4
:102D1000F0B5836805680022EB5C466803F0700339
:102D2000703B18BF4FF0FF338168B14201F10104DD
:102D300002D38460D018F0BD695C01F00F0709066A
:102D400047EA0212F5D58460002BEDD0013BEBE79A
:102D5000C068003818BF0120704702688368D05CE3
:102D600000F07000704702688368D05C70470268AA
:102D700080681044704783680B4483607047034643
:102D800082680168885C01280ABF013200209A60CD
:102D9000704708B5082007F05FFA00220260426021
:102DA00008BD10B5044638B14068FFF7C4FD2046A1
:102DB000BDE8104007F03ABA10BDF8B50646FFF777
:102DC000DEFF30BB3046FFF7C8FF05463046FFF751
:102DD000CAFF0746FFF7DDFF602D057004464FF080
:102DE000010519D107F00F07013F00E06D00AF4268
:102DF000FCDC2A4660213046FFF756FD23786060F0
:102E00002B4323703046FFF7A3FF18B12046FFF78E
:102E1000C8FF00242046F8BDF560F3E708B5082098
:102E200007F01AFA00220260426008BD10B504469D
:102E300050B10068FFF77FFD6068FFF77CFD20461A
:102E4000BDE8104007F0F2B910BD38B50446FFF7F1
:102E500096FF60B9FFF7E2FF05462046FFF77DFFCA
:102E6000702806D00123E3602846FFF7DFFF002526
:102E70001AE02046FFF74CFF0228F3D1012260211F
:102E80002046FFF711FD28602046FFF761FF00286C
:102E9000EAD1042260212046FFF706FD6860204643
:102EA000FFF756FF0028DFD1284638BD08B50820B7
:102EB00007F0D2F900220260426008BD38B503680D
:102EC0000446013303600D464068990016F008F887
:102ED0002368606003F18043013B40F8235038BD14
:102EE00038B50446B0B143687BB10368002B0CDDF4
:102EF0000025636853F82500FFF738FD2368013586
:102F0000AB42F6DC606807F091F92046BDE8384036
:102F100007F08CB938BDF8B50546FFF730FF48B962
:102F2000FFF7C4FF04462846FFF717FF702803D0B9
:102F30000123EB60002405E02846FFF7E9FE064682
:102F4000002E01DC2046F8BD2846FFF71CFD074691
:102F50002846FFF7FDFE28B101232046EB60FFF76E
:102F6000BFFFE7E71FB139462046FFF7A7FF013E45
:102F7000E6E710B5102007F06FF904461022002193
:102F800015F0A8F8204610BD38B5C36804460133D3
:102F9000C3600D468068990015F0A2FFE368A06049
:102FA00003F18043013B40F8235038BD10B55C204D
:102FB00007F052F904465C22002115F08BF82046F8
:102FC00010BD10B50446002849D00068FFF7CEFCBC
:102FD0006068FFF72BFFA068FFF7ADFCE068FFF724
:102FE000AAFC2069FFF7A7FC6069FFF7A4FCA069B1
:102FF000FFF7A1FCE069FFF79EFC206AFFF79BFC4E
:10300000606AFFF798FCA06AFFF795FCE06AFFF79B
:1030100092FC206BFFF7AAFC606BFFF78CFCA06BA7
:10302000FFF789FCE06BFFF786FC206CFFF783FC61
:10303000606CFFF780FCA06CFFF77DFCE06CFFF795
:103040007AFC206DFFF777FC606DFFF774FCA06DD4
:10305000FFF78CFC2046BDE8104007F0E7B810BD34
:1030600038B50446FFF78BFE60B9FFF79FFF0546B2
:103070002046FFF772FE702806D00123E360284641
:10308000FFF79FFF002505E12046FFF741FE1728C7
:10309000F3D12046FFF777FC28602046FFF758FE63
:1030A0000028ECD12046FFF7D0FE68602046FFF7ED
:1030B0004FFE0028E3D1082260212046FFF7F4FBF1
:1030C000A8602046FFF744FE0028D8D101226021E5
:1030D0002046FFF7E9FBE8602046FFF739FE0028AD
:1030E000CDD1012250212046FFF7DEFB286120468A
:1030F000FFF72EFE0028C2D1082250212046FFF7FC
:10310000D3FB68612046FFF723FE0028B7D10122D8
:1031100060212046FFF7C8FBA8612046FFF718FE94
:103120000028ACD1012250212046FFF7BDFBE86109
:103130002046FFF70DFE0028A1D10822502120468D
:10314000FFF7B2FB28622046FFF702FE002896D167
:10315000012260212046FFF7A7FB68622046FFF7A7
:10316000F7FD00288BD1012250212046FFF79CFB60
:10317000A8622046FFF7ECFD002880D108225021EC
:103180002046FFF791FBE8622046FFF7E1FD0028AB
:103190007FF475AF2046FFF7F6FB28632046FFF764
:1031A000D7FD00287FF46BAF012260212046FFF796
:1031B0007BFB68632046FFF7CBFD00287FF45FAF01
:1031C000012250212046FFF76FFBA8632046FFF73E
:1031D000BFFD00287FF453AF082250212046FFF79F
:1031E00063FBE8632046FFF7B3FD00287FF447AF99
:1031F000012260212046FFF757FB28642046FFF795
:10320000A7FD00287FF43BAF012250212046FFF7A5
:103210004BFB68642046FFF79BFD00287FF42FAF2F
:10322000082250212046FFF73FFBA8642046FFF705
:103230008FFD00287FF423AF012260212046FFF795
:1032400033FBE8642046FFF783FD00287FF417AFC7
:10325000012250212046FFF727FB28652046FFF773
:1032600077FD00287FF40BAF082250212046FFF79E
:103270001BFB68652046FFF76BFD00287FF4FFAE5F
:103280002046FFF780FBA8652046FFF761FD002878
:103290007FF4F5AE284638BD10B5142006F0DCFFEB
:1032A00004461422002114F015FF204610BD10B56D
:1032B000044698B10068FFF759FB6068FFF73BFBD5
:1032C000A068FFF738FBE06800F02FF92069FFF7EE
:1032D0004DFB2046BDE8104006F0A8BF10BD10B55C
:1032E000044638B3D0E90030FBB11B78013B032B17
:1032F00016D8DFE803F0020C0F1200F016F9206870
:10330000FFF719FB2046BDE8104006F08FBFFFF71E
:10331000CEFFF4E7FFF755FEF1E7FFF787FDEEE795
:103320000028ECD006F082FFE9E70028EAD006F09A
:103330007DFFE7E710BD38B50446B8B10068FFF778
:1033400015FB6068FFF7CBFF0025D4E902039D421F
:1033500006DB06F06BFF2046BDE8384006F066BF8E
:1033600050F82500FFF7E7FF0135EEE738BD38B527
:103370000446FFF704FD60B9FFF78EFF05462046BF
:10338000FFF7EBFC702806D00123E3602846FFF727
:103390008EFF002535E02046FFF7BAFC0528F3D163
:1033A0002046FFF7F0FA28602046FFF7D1FC0028FE
:1033B000ECD1012260212046FFF776FA68602046B2
:1033C000FFF7C6FC0028E1D1012250212046FFF77B
:1033D0006BFAA8602046FFF7BBFC0028D6D1204638
:1033E00000F0B9F8E8602046FFF7B2FC0028CDD124
:1033F0002046FFF7C8FA28612046FFF7A9FC0028FD
:10340000C4D1284638BD38B50546FFF7B8FC60B9C9
:10341000FFF74CFD04462846FFF79FFC702806D0B6
:103420000123EB602046FFF75AFF00241CE02846EA
:10343000FFF76EFC0228F3D1012260212846FFF736
:1034400033FA20602846FFF783FC0028EAD123687E
:103450001B78013B032BE3D8DFE803F002080C10D4
:10346000284600F078F86060204638BD2846FFF70F
:103470007EFFF8E72846FFF7F3FDF4E72846FFF75D
:10348000E4FCF0E7F8B50446FFF779FC60B9FFF714
:1034900070FD05462046FFF760FC702806D001232A
:1034A000E3602846FFF747FF002525E02046FFF7A9
:1034B0002FFC0328F3D12046FFF765FA2860204649
:1034C000FFF746FC0028ECD12046FFF79CFF686020
:1034D0002046FFF73DFC0028E3D12046FFF74FFCD4
:1034E00050B92046FFF739FC7028D8D12046FFF7A5
:1034F0000FFC0646002E01DC2846F8BD2046FFF7EB
:10350000C1FF07462046FFF723FC0028C9D11FB1A1
:1035100039462846FFF738FD013EEBE708B508209D
:1035200006F09AFE0023036008BD10B5044688B17A
:103530000378406823B1402B09D0FFF7FCF901E084
:10354000FFF714FA2046BDE8104006F06FBEFEF704
:10355000EAF9F7E710BDF8B50546FFF710FC38BBF0
:103560002846FFF7FAFB07462846FFF7FCFB06460E
:10357000FFF7D4FFF9B2402F044601701BD003DCE3
:103580005FB10123EB600CE0502F01D0602FF8D128
:1035900006F00F060127013E12E02846FFF7F3F977
:1035A00060602846FFF7D4FB18B12046FFF7BDFF47
:1035B00000242046F8BD2846FEF78FF9F0E77F008B
:1035C000BE42FCDC3A462846FFF76EF9237860607D
:1035D0003B432370E5E7000038B50A4C054601215E
:1035E000204603F0F7FD002320461A46012103F090
:1035F0002BFD204685F001020121BDE8384003F093
:10360000F3BD00BF0000024008B50120FFF7E4FF52
:10361000BDE80840032004F00FBD0846FFF7DCBFFB
:1036200010B50446024B036012F0B6FF204610BDF1
:10363000C4B7010810B50446054B503040F8503C63
:10364000044B40F8083CFFF7EBFF204610BD00BFDD
:10365000D8B7010824BA010810B50446FFF7E0FF07
:103660002046082112F0BCF9204610BD10B50446D2
:10367000FFF7E0FF20467C2112F0B2F9204610BD92
:1036800004F08ABD10B50C460AF0ACFB022808D144
:103690004FF47A704443B4FBF0F0BDE810400AF0F8
:1036A00023B92046BDE8104003F0E0BA10B5094C3C
:1036B000094806F035FD20460B2103F08BFD002361
:1036C00020461A460B2103F0BFFCBDE8104003F072
:1036D000B3BA00BF00000240D1B3010808B50348E7
:1036E00006F01EFDBDE8084004F056BDEDB301082C
:1036F000021E18BF01220321014803F075BD00BF5F
:10370000000402400321014803F077BD0004024099
:10371000024B0121186803681B6818471C1C002015
:1037200008B5022003F0D8F903F044FA00F096FC43
:1037300003F074FA00F07CFE03F0DEFF0C4802F0A8
:1037400003FF4FF4E13004F0EBFA0A4B1A680AB9B0
:10375000094A1A60094B1A680AB9074A1A600848E8
:1037600006F0DEFCBDE80840064806F0D9BC00BF04
:1037700009360008101F0020D17B0008141F00200C
:103780000BB4010823B401082DE9F3410446264691
:103790004FF01B0812F098FE264B04F1210746F863
:1037A000113B10220021304614F094FC42460021C7
:1037B000384614F08FFC002521461F4BC4E90F55F5
:1037C00004F1480041F8443F01F026F81B4BC4E9DE
:1037D0001B55A3651A4B84F85C50C4E91835194B86
:1037E00084F87450A567184DA366184806F098FC35
:1037F0006B6E174A01936B6D414600932B6D3846F3
:1038000015F0E0FB296D304606F095FD696D04F179
:10381000150006F090FD696E04F1190006F08BFDAD
:10382000296D04F11D0006F086FD204602B0BDE8BA
:10383000F08100BFD8B7010884B8010894B8010826
:10384000ECB80108B0B801080000F81F39B401084D
:103850004EB4010810B5094CFFF762FF2368DB077F
:1038600009D40748FFF790FF0123064A0649044898
:10387000236012F0E7FE024810BD00BF141C0020B8
:10388000201C0020000000203536000838B5064D09
:10389000064C2B6813F0010F04D1FFF7DBFF012367
:1038A00020602B60206838BD181C00209C1C002064
:1038B00010B5FFF7EBFF836F11203BB104F05AFC0A
:1038C000FFF7E4FFBDE81040836F1847BDE81040E4
:1038D00004F05DBC08B50B21054803F095FC28B148
:1038E000BDE808400B21024803F0A4BC08BD00BF9E
:1038F0000000024008B519B1BDE80840FFF7D6BE88
:10390000044806F00DFCBDE8084002220B210248E5
:1039100003F0DABB60B401080000024070B5044651
:103920002E4804F1440506F0FBFB2846002100F078
:103930009BFD0021284600F0ADFD204612F0F4FD6D
:103940000CF05CF920460021FFF7D4FF0BF054F88F
:1039500001220C21224803F0B7FB04F001F804F126
:10396000480000F03BFF23682046DB6804F168054F
:10397000002198471B4E0021284600F017FE03F057
:10398000B5FC194806F0CCFB04F0C6F803F046F984
:10399000304601220D2103F097FB012230460E2113
:1039A00003F092FB0021084603F086FF04F1580063
:1039B00000F086FD0121284600F0F8FD4FF4E130CB
:1039C00004F0AEF9094806F0ABFB0AF041FF03F042
:1039D000C5FF2046BDE8704012F0B3BD78B40108C1
:1039E00000040240000002409CB4010886BD0108AA
:1039F00038B50546FFF76EFF044628B1002128467A
:103A0000FFF778FF03F018F902F0CAFF05460CB182
:103A1000FFF74CFE284638BD70B50C4606461549E2
:103A2000204613F0E9FE20B90021204613F0C6FE1F
:103A300070B11149204613F023FD13F0E7FE014653
:103A40000E4806F06DFB4FF4C0710D4802F0B6FD54
:103A50003046FFF73FFF054648B93046FFF7C8FF3D
:103A60000146204613F0C8FE08B1FFF71FFE2846A6
:103A700070BD00BF3333534000007A44AAB401083C
:103A80007DDF010870B52D4A05461368D6B0DB0707
:103A900005D42B4900F168030B6001231360294909
:103AA0002846FFF7B9FF0646274806F039FB0021F4
:103AB00005F1440000F0EEFC244C254BE360254B5F
:103AC0002361254BA360254B6360254B2360254B69
:103AD0006361254BA361254BE36104F110030FCB18
:103AE0008DE80F0094E80F0012F044FA002305A8B7
:103AF000EB632B6412F0C6F99DF8143005F13C0419
:103B0000012B14D1DDF8153005A8EB63DDF8193071
:103B10002B6412F087F9164806F002FB08212046B4
:103B200006F064FBBDF91611124806F0F9FA3146A9
:103B30002846FFF7DFFE56B070BD00BF101C002006
:103B40001C1C002000004040D9B40108EC2A0020D1
:103B50006D6C0008E16B000811370008053700089C
:103B6000F136000821A10008F5C3000831C400089F
:103B7000FAB4010820B501087FB5F82300F1580513
:103B8000064628468DF80F3000F0A0FC02230DF108
:103B90000F0100930122A123284600F09BFC4FF463
:103BA00000430822009306F16C01A1230446284635
:103BB00000F0BCFC0440E4B2284600F089FC20463A
:103BC00004B070BD30B58BB0044604F063FA014612
:103BD0005A4806F0A5FA04F0B7FA0146584806F02C
:103BE0009FFA584806F09CFA204600F0D7FB04F1F3
:103BF000580500F00DFB00F0B9FA5348534906F0A0
:103C00008FFA284600F05CFC38B9514806F088FA73
:103C100040F23B114F4802F0D1FC03F00DF8204672
:103C2000FFF7AAFF20B94FF4A0714A4802F0C6FC82
:103C300094F8733094F86D20049394F8723094F8EB
:103C40006C10039394F871304348029394F87030E9
:103C5000019394F86F30009394F86E3006F060FA98
:103C6000284600F085FA284600F0E4FA04F14405FD
:103C7000002184F87400284600F0F6FB012000F0D3
:103C8000D9FD0021284600F005FC012000F0F0FDE0
:103C90002046FFF7F7FE204600F018FB2F4806F0FD
:103CA0003FFA4FF4FA7014F0BFF9054600283ED1F0
:103CB0002B4806F035FA2B4806F032FA2A4806F06F
:103CC0002FFA2A4806F02CFA294806F029FA294842
:103CD00006F026FA284806F023FA284806F020FACB
:103CE000274806F01DFA274A2749284806F018FAFF
:103CF0002749284806F014FA274806F011FA04F17B
:103D00002101264806F00CFA2549264806F008FA53
:103D100007A803F093FC07A806F05CF901462248C7
:103D200006F0FEF9104806F0FBF90BB030BD1F4855
:103D300006F0F6F9284614F07FF9BCE740B5010813
:103D400056B501086CB5010883B50108A0860100CD
:103D50009EB501087DDF0108B4B50108E9B5010889
:103D60001CB601087BDF01085AB601088BB60108B2
:103D70009AB60108BCB60108DFB6010803B701080E
:103D80007CDF010826B701082CB701083BB7010802
:103D90004AB7010851B701085CB701087CB70108B0
:103DA00087B701088DB70108A7B7010850B6010809
:103DB0002DE9FF4100F15805284600F087FB042457
:103DC0000226DFF8A080013C14F0FF0431D0A123CB
:103DD000012241462846009600F07CFB4FF4004348
:103DE000074600930422A123284602A900F09EFB67
:103DF000002FE8D00028E6D09DF80830442B1FD1D2
:103E00009DF809306E2B1BD10DF10A0006F077FAF0
:103E1000441CA4B221460DF109008DF8086006F09B
:103E200093FA002303220093A023284602A900F05E
:103E300051FB284600F04CFB204604B0BDE8F08161
:103E4000442300248DF809306E2321460DF10B0028
:103E50008DF80A308DF8084006F076FAA023052286
:103E60000094E2E7CCB7010838B50D46044611319D
:103E70000BF086FDEB6E204623602B6F636038BD30
:103E800030B50D469DB0044601466846FFF7ECFF8D
:103E9000694628460BF026FC04F1110321346B63BC
:103EA0002C631DB030BD000070B5084690B01546BB
:103EB000114B124A124910F029FF0021114B124EEA
:103EC0000B93124B10220C93114B0E910D9307ABD9
:103ED00018460F9614F0FEF80E4A0895099201ADA7
:103EE0000FC885E80F000BAC009694E80F0011F0A6
:103EF0006DF810B070BD00BF8136000834AD010808
:103F000058AD01083D6D0008B1380008C56C0008C7
:103F1000DD3600080000080810B50446FFF7B6FCBF
:103F20002146BDE81040FFF743BF0000024B186870
:103F300003689B68184700BFA81C0020024B186844
:103F400003685B68184700BFA81C0020024B186874
:103F500003681B68184700BFA81C002037B502245F
:103F600005461346044A106802680094D4680A465D
:103F70002946A04703B030BDA81C002037B5002457
:103F800005461346044A106802680094D4680A463D
:103F90002946A04703B030BDA81C002037B54FF418
:103FA000004405461346054A1068026800941469E7
:103FB0000A462946A04703B030BD00BFA81C002018
:103FC0004FF47A735843B0FBF3F009F08DBC000056
:103FD0001FB58DF80C1000218DF80D20054A034601
:103FE000106802680091D46803A90222A04704B0B7
:103FF00010BD00BFAC1C00200023F0B513701446A8
:10400000022205460C4E85B030688DF80F1003680B
:104010000092DF6801222B460DF10F01B84748B12D
:104020004FF4004230682146036800921E69012265
:104030002B46B04705B0F0BDAC1C0020024B186801
:1040400003689B68184700BFAC1C0020024B18682F
:1040500003685B68184700BFAC1C002010B5424CD9
:104060000AF01CFD20460222002103F02DF8012257
:104070002046114603F028F820460122022103F0D1
:1040800023F820460222032103F01EF820460022D6
:10409000042103F019F820460222082103F014F845
:1040A00020460122092103F00FF8204601220A21AF
:1040B00003F00AF8204602220B2103F005F802F073
:1040C000ADFD002320461A460C2102F0BDFF20461C
:1040D00000220C2103F088F82046002204F58064B9
:1040E0000F2102F0F1FF20460122002102F0ECFF37
:1040F00020460022022102F0E7FF20460022032191
:1041000002F0E2FF20460222062102F0DDFF2046F7
:104110000022082102F0D8FF20460022092102F0E7
:10412000D3FF204601220C2102F0CEFF20460222BE
:104130000D2102F0C9FF204602220E2102F0C4FF29
:10414000204602220F2102F0BFFF002304F5806405
:1041500020461A460D2102F077FF2046BDE81040A8
:1041600000220D2103F040B80000024003F0C4BA61
:104170001C4B00B51A6889B0D2075FBF1A4A10609D
:1041800001221A60194B0493194B0593194B0393A1
:10419000194B0293194B0793194B069308AB13E97C
:1041A00003008DE8030002AB0FCB11F08FFD90B13F
:1041B000144805F0B5FF00221348114602F084FFB1
:1041C0000F2302220021104802F01CFE09B05DF806
:1041D00004EB11F015BD6A210C4809B05DF804EB41
:1041E00002F0ECB9A41C0020AC1C00204D400008DB
:1041F0003D400008F93F0008D13F000821A1000818
:10420000C13F0008ECB70108000002407DDF010853
:10421000002307B5ADF8043001238DF8063001986E
:104220000AF098FB02F0FAFC03B05DF804EB0AF028
:10423000E3BB0000194B10B51A688CB0D2075FBF02
:10424000174A106001221A60164B0793164B05930C
:10425000164B0693164B0893164B0993164B0A936D
:10426000164B0B930CAB13E907008DE8070005AB69
:104270000FCB11F04DFC044601220F21104802F033
:1042800023FF3CB10F4805F04BFF11F01FFC204607
:104290000CB010BD0C4805F043FFF8E7A01C00204F
:1042A000A81C00209D3F00087D3F00085D3F0008DE
:1042B0004D3F00083D3F00082D3F000821A10008A8
:1042C00000000240FDB7010830B801082DE9F047B1
:1042D0009AB00AF06FFFDFF89CA0274C274FDFF859
:1042E000A08012AD50B9CDE91544CDE91387CDF8C2
:1042F00048A0009495E80F000AF076FF214B0026B5
:104300001393214B4FF001091293204B06A91493EC
:104310001F4B284615931F4BCDE91887CDE916345E
:104320000423CDE906368DF81D9006F015FC06F045
:1043300007FC06F04FF8184ACDE9096611920322EE
:10434000CDE90C440B9608928DF8269008AB02AC90
:104350000FCBCDE90F87CDF838A084E80F00DDE959
:1043600010018DE803000CAB0FCB0BF04BFB1AB028
:10437000BDE8F087E576000821A100082DA200081D
:1043800059A200087DE9000851E8000861E700082B
:10439000F9E600080DE70008193F00082DE9F0478D
:1043A000044602F0FDFA1E49054613F069F813F0C1
:1043B0002DFA01461B4805F0B3FE4FF08041284618
:1043C00013F0FCF948B30025DFF85C90DFF850806B
:1043D000164F02F0E5FA4946064613F003FAA8B96B
:1043E0004146304613F04CF813F010FA01463846B7
:1043F00005F096FE236885F0010520462946DB6816
:1044000098474FF47A7002F031FCE2E723682046C7
:10441000BDE8F0470021DB681847BDE8F08700BF22
:1044200000007A444EB801080000204060B801083E
:1044300008B50120084902F0BDFF0B20074902F032
:10444000B9FF0A20064902F0B5FFBDE80840072081
:10445000044902F0AFBF00BFA5BE000845C2000876
:1044600065C00008BDC20008002310B50C461A46FE
:104470000D21074802F0E8FD14B1012C00D010BD59
:104480002246BDE810400D21014802F0ADBE00BF3C
:1044900000080240002310B50C461A460C210748BC
:1044A00002F0D2FD14B1012C00D010BD2246BDE8AF
:1044B00010400C21014802F097BE00BF00000240EE
:1044C000014802F001BF00BFA086010002F0CCBE8F
:1044D00002F0E6BE2DE9F041DDF818801E4608F036
:1044E0000303032B07460C46154603D12F210E4824
:1044F00002F064F818F0020F32462946204609D02F
:1045000002F01CFF10B10120BDE8F0810123002062
:104510003B71F9E718F0010F02D002F01DFFF1E73F
:1045200002F0FEFEEEE700BF7DDF01082DE9F0415D
:10453000DDF81880074618F0010F0C4615461E4698
:1045400003D04C210E4802F039F818F0020F03D0C6
:104550004F210B4802F032F818F4004F324629463A
:10456000204609D002F006FF10B10120BDE8F0811D
:10457000012300203B71F9E702F0C4FEF4E700BF1D
:104580007DDF0108032108B5034802F036FE00383C
:1045900018BF012008BD00BF000402400A460248BF
:1045A000032102F021BE00BF0004024008B581B122
:1045B000012303211A460A4802F046FD0321084858
:1045C00002F008FEBDE8084003220548114602F04B
:1045D0001BBD0122BDE808400321014802F074BD63
:1045E0000004024003F07EB81FB501A805F0B5FC39
:1045F00001A803F05BF905B05DF804FB03F0C4B853
:1046000003F0DCB8084602F055BF7FB50023CDE9C2
:104610000133ADF80C3001238DF807308DF80830E8
:104620006FF01D038DF809300723044601A88DF8AB
:104630000A3005F0B7FC236806461B6820460D4685
:104640009847864275EB0103B4BF0120002004B0F7
:1046500070BD70B50646194610461C4615460AF050
:104660000DFE736823B128462146BDE87040184707
:1046700070BD00002DE9FF4714461D46804603F03B
:1046800031F806460F46B4EB000A22462B4601A835
:1046900065EB010905F061FC3046394605F0C4FCC4
:1046A00029460646204605F0BFFC494604465046CA
:1046B00005F0D0FC224603463146074805F030FDA0
:1046C00001A802F0ABFF20B152464B464046FFF72F
:1046D000C0FF04B0BDE8F087BCB801087047704760
:1046E0007FB500F10806054630460C4611F07EFF06
:1046F00060BB324805F014FDA27C617C304805F0B7
:104700000FFD637C3BB16868002103681B68984714
:10471000022000F08FF8A37C3BB168680021036899
:104720005B689847022000F0A3F861684E2918D012
:104730004F2916D0452914D01621224801F03EFFFA
:104740001721214B214A224813F062FA6421304696
:1047500011F038FF0028CFD143211A4801F02EFF75
:10476000CAE7A268D31F022B14D8E368D2B20F2B7A
:1047700019D00BDC052B16D00A2B13D0342111488D
:1047800001F01CFF3521104B124ADCE7142BF5D148
:10479000022308E024210B4801F010FF25210A4BD9
:1047A0000D4AD0E70123A07C0290607C0190207C20
:1047B0000090206803F0EEFA04B070BD08B901085B
:1047C00021B901087DDF01088FAE01083EB901085B
:1047D0006EB90108E6B90108AEB9010810B5044682
:1047E00003F0AAFA04F10800BDE8104011F001BF7F
:1047F000084603F0A3BB38B50C468D18AC4204D074
:1048000014F8010B03F09AFBF8E738BD03F0BABACD
:10481000084603F0C1BB000010B50446044BC0E9D4
:1048200000310121083011F0EFFE204610BD00BF1D
:1048300024BA0108042817D8DFE800F00309100E95
:104840001200002303211A46084802F0FDBB002293
:104850000321064802F038BC0222F9E70122F7E7FB
:104860000321024802F056BC704700BF000002401E
:10487000042817D8DFE800F00309100E1200002307
:1048800002211A46084802F0DFBB00220221064836
:1048900002F01ABC0222F9E70122F7E702210248DE
:1048A00002F038BC704700BF0000024010B504465B
:1048B000C06908B105F0BAFC206908B105F0B6FC82
:1048C000606808B105F0B2FC204610BD10B5044682
:1048D000006808F099FB204610BD00001FB5536822
:1048E0000293137801934B6800930B684268017838
:1048F000024805F015FC05B05DF804FB44BA010858
:10490000FE2307B58DF80430054B01A91868002374
:1049100000681A4608F06AF803B05DF804FB00BFAF
:10492000BC1C0020814203D0CB21024801F046BECE
:10493000704700BF7DDF010870B51D467423C0E9D4
:1049400000310023044683600820164611F028F841
:10495000C0E90065A060204670BD000037B5044680
:104960000D4600686321FFF7DDFF00232846A1689C
:1049700001AA019305F0BEF9019B1BB13821024841
:1049800001F01CFE03B030BD7DDF0108F8B56323E4
:104990000027C0E90031044687601A20154610F050
:1049A000FFFF06461A22394613F094FB204629469B
:1049B000A660FFF7D3FF2046F8BD81647047C1644D
:1049C000704700002DE9F843D0E9017488460026BD
:1049D0004FF00C090A4BE41BA4105C43F5B2A5424E
:1049E0000BD209FB05734146586814F0BBFB013636
:1049F0000028F3D12846BDE8F8834FF0FF30FAE7EE
:104A0000ABAAAAAA2DE9F843D0E904748846002687
:104A10004FF00C090A4BE41BA4105C43F5B2A5420D
:104A20000BD209FB05734146586814F09BFB013615
:104A30000028F3D12846BDE8F8834FF0FF30FAE7AD
:104A4000ABAAAAAAF8B50E4649680446FFF7BAFF12
:104A5000C0B2FF2803D07C21204801F0AFFDD4E98B
:104A600001239B1AB3F5BD6F03D97F211B4801F0C9
:104A7000A5FDD4E90153E0685A1B194902F10C075E
:104A80001B1A92104A439B104B4301329A420DD895
:104A90003D44A560D4E9013496E80700E31A04E92F
:104AA00007000F489B1058430138F8BD384605F001
:104AB000D3FB054618B96921084801F07FFDD4E908
:104AC00001128A4203D02846521A13F0E9FA6068AC
:104AD00005F0ACFB65603D44E560DAE77DDF010889
:104AE000ABAAAAAA1FB56E23CDE90131002301A903
:104AF0000393FFF7A7FF05B05DF804FBFF22F8B5AD
:104B0000002304460526002780F828204FF0FF35B3
:104B10006FF07F42C0E90033C0E90233C0E90433DB
:104B2000C0E90633C0E908334FF000410020C4E972
:104B30001467234EC4E910523268C4E90C0112F024
:104B40000102C4E90E01C4E91233C4E91801A365E6
:104B500013D101211B4D08462A60696007F06AFEE7
:104B6000286018B95121184801F028FD0123174A7F
:104B700017491448336011F065FD164B1A680AB9DD
:104B8000104A1A6020461449FFF7ACFF134B144932
:104B900018702046FFF7A6FF124B134918702046E5
:104BA000FFF7A0FF114B124918702046FFF79AFF3C
:104BB000FE22104B1870104B20461A70F8BD00BF33
:104BC000B81C0020401D00207DDF010800000020EF
:104BD000CD480008BC1C002062BA0108C41C00209B
:104BE0006ABA0108C21C002072BA0108C01C002069
:104BF00077BA0108C31C0020C11C002010B5084C66
:104C00002368DB0709D40748FFF778FF0123064A2A
:104C100006490448236011F015FD024810BD00BF8D
:104C2000B41C0020D81C002000000020AD48000863
:104C3000F8B50E4649680446FFF7E4FEC0B2FF2807
:104C400003D08721204801F0B9FCD4E904239B1A42
:104C5000B3F5BD6F03D98A211B4801F0AFFCD4E93D
:104C60000453A0695A1B194902F10C071B1A921030
:104C70004A439B104B4301329A420DD83D44656133
:104C8000D4E9043496E80700E31A04E907000F4862
:104C90009B1058430138F8BD384605F0DDFA05464B
:104CA00018B96921084801F089FCD4E904128A4244
:104CB00003D02846521A13F0F3F9206905F0B6FA2A
:104CC00025613D44A561DAE77DDF0108ABAAAAAA08
:104CD00038B5D0E901239B1A074A9B105343CDB244
:104CE0009D42044603D3A621044801F067FC0C2032
:104CF000636800FB053038BDABAAAAAA7DDF0108B6
:104D000038B5CCB2114905460B6813F0010307D141
:104D100070200F4A10600F48C2E9010301230B60A5
:104D2000FF2C10D0D5E904239B1A0B4A9B10534348
:104D30009C4203D3B221094801F040FC0C212869B0
:104D400001FB040038BD0248FCE700BFB01C002096
:104D5000C81C00207FBA0108ABAAAAAA7DDF0108FF
:104D600010B5D0E90730C9B2D2B2834209D01C785D
:104D70008C4204D15C78944201D1987810BD033301
:104D8000F3E74FF0FF30F9E72DE9F0410D460A78DF
:104D9000D0E904135B1A49499B104B439A420446DD
:104DA00003D39321464801F009FCD4E901135B1AAF
:104DB00042499B104B436A789A4203D3942140485E
:104DC00001F0FCFBD4E904135B1A3C499B104B43F4
:104DD000AA789A4205D3FE2A03D09521384801F0DB
:104DE000EDFB2F78204639466A78FFF7B9FFC3B24A
:104DF000FF2B064629D039462046FFF781FF697808
:104E000007462046FFF764FF314680462046FFF7FD
:104E100077FF414602463846FFF760FD2978204675
:104E2000FFF76EFF697806462046FFF751FFA97825
:104E300007462046FFF764FF394602463046FFF733
:104E40004DFD9C211E4801F0B9FBD4E907239B1AB4
:104E5000B3F5BD7F03D99F21194801F0AFFBD4E919
:104E600007631649606A9A1BD71C1B1A4A434B43B7
:104E700001329A420AD83E4426622A88236A23F8DD
:104E8000032CAA7803F8012CBDE8F081384605F020
:104E9000E3F9064618B96921094801F08FFBD4E906
:104EA00007128A4203D03046521A13F0F9F8E0692B
:104EB00005F0BCF9E6613E446662DDE7ABAAAAAA4A
:104EC0007DDF010838B58168006814461D4605F08D
:104ED00073FA0146001945EBE17138BD2DE9F04741
:104EE0000F680E46722F9046994633D0742F08D023
:104EF000632F1ED000254FF0004428462146BDE810
:104F0000F08739463846FFF70DFDB368D3E9005402
:104F1000B4F1004F08BF002DEFD039463068FFF7DD
:104F200001FDB368D3E9005418EB050549EB04040F
:104F3000E3E739463846FFF7F5FC42464B46B06892
:104F400004F09AFF0C1E0546D7DADD21074801F070
:104F500035FBD2E738463946FFF7E4FC42464B467C
:104F6000B068BDE8F047FFF7ADBF00BF7DDF0108C7
:104F70002DE9F8430F4606460024FFB2FFF7C0FEB6
:104F8000D6E90759A94516D02B78BB4211D16978CB
:104F90003046FFF79DFE01688046692909D1084621
:104FA000FFF7C0FCD8F808301B6803B198470134FC
:104FB000E4B20335E6E72046BDE8F8832DE9F74380
:104FC00006460F460025FFF79BFEF469336A03345B
:104FD00003F10309FFB24C4520D014F8013C34F82A
:104FE000032C8DF8063014F8033CADF804209F42E2
:104FF00012D19DF805103046FFF76AFE0168804621
:10500000692909D10846FFF78DFCD8F808305B689C
:1050100003B198470135EDB20334DCE7284603B00D
:10502000BDE8F083836C73B504460D46164623B97C
:105030004FF48E710B4801F0C1FA23462A46CDE9A0
:1050400000640949094808F0BFF8012807D04FF467
:105050009171044802B0BDE8704001F0AFBA02B0EF
:1050600070BD00BF7DDF01088DBA010841570008FF
:1050700038B590F847300446032B0D4604D940F26A
:105080003511064801F09AFA94F84700431C84F859
:105090004730044484F8425038BD00BF7DDF01082A
:1050A00010B590F84730044623B94FF49D71064877
:1050B00001F084FA94F847000138C0B284F8470040
:1050C000044494F8420010BD7DDF0108CBB2FE2BF2
:1050D00010B504460AD0FFF713FE03686D2B05D107
:1050E000017A2046BDE81040FFF70ABE10BD00005F
:1050F0002DE9F84304460026114FD4E904239B1AF6
:105100009B107B435FFA86F8984516D241462046AD
:10511000FFF7DCFFD4E90759A9450CD02B784345AC
:1051200007D169782046FFF7D3FD2046A978FFF71D
:10513000CDFF0335F0E70136DFE7BDE8F88300BFB8
:10514000ABAAAAAA70B56FF04106044600F1420569
:10515000361A94F8472073199A4205DD204615F84F
:10516000011BFFF7CDFDF4E770BD2DE9F74F4FF0C0
:105170000009DDE90CBA04468846C0E90899D8E977
:1051800007734FF000410020C4E90001C4E90201A7
:10519000C4E90401C4E90601FF210093D3B284F8F5
:1051A00020100193009BD4E900569F4222D03A7808
:1051B000019B9A421CD179784046FFF789FD5A46F7
:1051C000014653464046FFF789FEB1F1004F08BF44
:1051D00048450DD0B6F1004F08BF4D4503D0A84259
:1051E00071EB060304DA7A78C4E9000184F8202020
:1051F0000337D7E7B6F1004F08BF002D05D0B5EB58
:105200000B0566EB0A03C4E90453204603B0BDE86E
:10521000F08F70B515461C46FFF75AFD866874215D
:105220000068FFF77FFBC6E9005470BD836C10B5C2
:10523000044623B940F29D21024801F0BFF9A06C59
:1052400010BD00BF7DDF0108036870B504460D4640
:1052500016461BB92921064801F0B0F93246294605
:10526000206807F067FC431E5842584170BD00BFDC
:105270007DDF010813B5FF24074B0A46186801A912
:105280008DF80440FFF7E0FF18B19DF8040002B06C
:1052900010BD2046FBE700BFBC1C0020F8B50D4642
:1052A0000B4B8969064659434FF47A73B1FBF3F10E
:1052B000FFF7E0FF0446C7B2B06C03681B6898476D
:1052C000FF2FC6E90E0114BF204695F82000F8BD57
:1052D00040420F0038B5C36C04460D461BB9BDE80B
:1052E0003840FFF7DBBF806C174903685B6998475C
:1052F000A06C0368DB689847D5E9020104F094FECE
:105300000146124804F00CFFA06C03689968D5E9C7
:1053100002238847A06C03681B699847E36C984791
:10532000A06C0368DB689847A06C03681B6898470B
:10533000C4E90E0100212046FFF79CFFC0B2FE2801
:1053400008BF95F8200038BD0149000898BA010847
:10535000F8B5D1E90663B3F1004F08BF002E05464A
:105360000C4608D11AB1BDE8F840FFF797BFBDE879
:10537000F840FFF7AFBF012E73F1000702DA91F892
:105380002000F8BD92B121462846FFF787FF94F828
:105390002030C0B28342F4D1D5E90E62D4E90013C3
:1053A0008E4272EB0303B8BFFF20EAE7D0E9147224
:1053B000BE429341E7DBFFF78DFFE8E72DE9F047B9
:1053C0008CB004460D46FFF79BFC03680646702B25
:1053D00004D04FF4A071694801F0F0F8A06C0368A4
:1053E0001B6898472A46C4E90C01CDE90001214613
:1053F00002A8FFF7BAFE29462046FFF7B9FD9DF83F
:1054000028300746FF2B05D120B940F24B115B48ED
:1054100001F0D4F8D4E90C0104F006FE0146584826
:1054200004F07EFE3946574804F07AFE9DF82810B5
:10543000FF297CD100224FF00043CDE90623DDE9AE
:105440000223CDE90423DDE90623CDE90823A36D7A
:1054500013B39847DDE90223D4E91801B3F1004FF3
:1054600008BF002A09D0069B10F10B0741F100028A
:105470009F42079B72EB03030EDAD4E90C321B1830
:1054800042EB0102CDE90801CDE9043204F0E2FD6E
:1054900001463D4804F044FE4FF00009DFF8EC807F
:1054A000394F2046327A02A9FFF752FFA36D824698
:1054B00003B198475FFA8AF3FF2B57D1DDE9023237
:1054C000D4E90E01181A62EB0101CDE90432CDE9ED
:1054D0000601CDE9080104F0BDFD0146404604F097
:1054E0001FFEA36D002BDCD0DDE90223D4E91801F7
:1054F000B3F1004F08BF4A4509D0069B10F10B0CD1
:1055000041F100029C45079B72EB0303C9DAD4E921
:105510000E321B1841EB0202CDE90801CDE904323D
:1055200004F098FD0146384604F0FAFDB9E720463C
:10553000FFF7CEFBD0E90078DDE9020104F074FD4D
:10554000424603463946124804F0EAFDD4E90C32DB
:1055500002980399C01A61EB0201CDE9060104F03B
:1055600079FD01460B4804F0DBFD68E7294620463B
:10557000FFF724FD50460CB0BDE8F0877DDF010841
:10558000ABBA0108CABA010827BB01083FBB010832
:10559000E5BA010809BB010870B504460D46FFF7DE
:1055A000AFFB03686D2B0FD0702B07D0836894F886
:1055B000411094F84000BDE8704018472946204645
:1055C000BDE87040FFF7FABE40F22F11024800F02C
:1055D000F5FF4FF0FF3070BD7DDF01082DE9F0478A
:1055E00090F828300446FF2B04D14FF4E5714D4864
:1055F00000F0E4FF94F828102046FFF781FB426892
:105600000178494804F08CFD94F82830DFF81C81BB
:1056100084F8463094F846102046FFF771FB036883
:1056200005466D2B204694F846100BD1FFF720FD60
:10563000297A204684F84610FFF762FB2046FFF7E0
:1056400081FDE7E7FFF7A8FFC3B2FF2B07460BD1A9
:1056500040F2DF11334800F0B1FF40F2DF11344B6C
:10566000344A354812F0D4FA94F846500246294696
:105670002046FFF775FBC6B2FF2E14D139462046EF
:10568000FFF726FB41682D4804F04AFD4FF4F37103
:10569000244800F093FF4FF4F371254B254AE0E7CF
:1056A0002046FFF74FFDFE2E294620461CD1FFF76E
:1056B000F7FC054601462046FFF722FB3A462946FD
:1056C0002046FFF74DFBC6B2FF2EE9D139462046F2
:1056D000FFF7FEFA4FF4F971124800F06FFF4FF434
:1056E000F971134B134ABCE7FFF70AFB394605462D
:1056F0002046FFF7EDFA314681462046FFF700FBD2
:105700008246404604F00CFD524649462846FFF7C3
:10571000E5F894F8463084F8417084F8403084F815
:10572000466077E77DDF010867BB0108F4BB01082D
:105730008FAE010885BB0108AABB0108ECBB0108BC
:1057400008B504F051FEFFF759FAFFF747FF0000D4
:10575000FF23054A1370054A1370054A1370054A62
:105760001370054A13707047C41C0020C21C00202F
:10577000C01C0020C31C0020C11C002010B5044622
:10578000006807F041FC204610BD000073B50AF028
:105790007BFA28240AF056FA20B10A2008F0A4F86F
:1057A000013CF7D14FF6FF71314A324D13888B42DD
:1057B0001CBF01331380FFF721FAFFF737FD0368A1
:1057C0001B6898476E78DEB92B4B1C89C4B12B4AF5
:1057D000D2E90032B2F1004F08BFB3420ED083428B
:1057E00072EB01060CDA264EC31A06FB04F461EBD9
:1057F0000202E617A34272EB060301DB01236B7082
:105800000023ADF804308DF806306B782BB10123FE
:105810008DF80430194BC3E900012A78194B82B185
:1058200001228DF805201A70174A18491848019B63
:105830001278097800680AF093FA164B187802B0CB
:1058400070BD1A700C4B9B89002BEDD04AF6C0023C
:105850005343114CDD17D4E90024801A61EB040195
:10586000984271EB0503A4BF01238DF80530DBE7F7
:105870008A1D0020681D0020741D002040020020A9
:1058800080510100711D00206B1D00206A1D002049
:10589000641D0020C01C002030020020104B1B891A
:1058A00013B9104B1878704700220F4BD3E900133F
:1058B000B3F1004F08BF9142F3D10C490B7801338B
:1058C000DBB2012B0B70ECD8094B1A70094B1A7024
:1058D000094B1A60094B1A7001225A70084BE1E714
:1058E000741D0020C01C0020380200209C1D0020D8
:1058F0006B1D00206A1D0020641D0020681D002013
:10590000C31C00201FB57023CDE90131002301A97C
:105910000393FFF78DF905B05DF804FB2DE9F04F17
:105920004B4B04461A7885B0002A40F08E80012641
:1059300048491E70FFF7D6F8474B48491870204673
:10594000FFF7D0F8DFF818A146498AF80000204692
:10595000FFF7C8F8DFF810910A220023434989F8BD
:10596000000001A8FEF7E8FF01A92046FFF76AF84A
:10597000DFF8FC803F4988F800002046FFF7B2F8C6
:105980003D4B3E4918702046FFF7ACF83C4B3D4973
:1059900018702046FFF7A6F83B4B3C49187020468C
:1059A000FFF7A0F83A4B3B4A18703B492046FBF7FB
:1059B000DDF9DFF8E8B03A4A3A498BF800002046B2
:1059C000FBF7D4F9384905462046FFF79BFF7023C3
:1059D0000193364B074601A92046CDE90236FFF771
:1059E00027F90646324A2B46204612789BF80010CB
:1059F000FBF7C7F93B46294620469AF80020FBF7FB
:105A0000C0F933462946204699F80020FBF7B9F93A
:105A10002B463946204698F80020FBF7B2F92B4672
:105A20003146204698F80020FBF7ABF9214A2B4677
:105A3000294620461278FBF7A4F91F4B1F4A294636
:105A400020461B781278FBF79CF905B0BDE8F08F73
:105A50009D1D002004BC01086C1D00200EBC010827
:105A6000701D002019BC0108501D002025BC010834
:105A7000511D002032BC0108891D002040BC0108D6
:105A8000881D00204CBC01088C1D002059BC010859
:105A90008D1D00208D57000867BC01086E1D002079
:105AA0009D61000871BC010885BC010898BC010813
:105AB000C01C0020C31C0020C11C0020C41C0020EE
:105AC00030B5044685B00D46FFF728FF6D22064B22
:105AD00020461B7801A9CDE901258DF80C30FFF790
:105AE000A7F805B030BD00BF6E1D00202DE9F84FAE
:105AF000434B04461A68434D12F0010F79D1FF223F
:105B00002A7001221A602046FFF708FF20463E4A0D
:105B10003E49FBF72BF93E4A28703E492046FBF7E9
:105B200025F93D4F3D4A38703D492046FBF71EF9A7
:105B30003C4E3D4930702046FFF7C2FF3B4980464E
:105B40002046FFF7DFFE3A4982462046FFF7DAFE9D
:105B50008146384A20463B7829781278FBF711F9BC
:105B6000354ADFF8D8B02046337829781278FBF729
:105B700008F9204633789BF800203978FBF701F9C3
:105B800020462B789BF800203178FBF7FAF82C4A56
:105B90005346204639781278FBF7F3F82949204616
:105BA0003B780A785146FBF7ECF8274A4B462046EB
:105BB00039781278FBF7E5F8224920463B780A78D5
:105BC0004946FBF7DEF81C4A4346204631781278F6
:105BD000FBF7D7F84146204633789BF80020FBF7C7
:105BE000D0F81A4A20462B7812783178FBF7C9F89A
:105BF00002E02B78FF2B86D02878BDE8F88F00BF15
:105C00004C1D00209F1D0020315F0008ACBC010826
:105C1000715C0008B6BC01086D1D00209D5800088D
:105C2000C0BC01086F1D0020CABC0108D6BC010819
:105C3000E4BC01086C1D0020C31C0020C41C002013
:105C4000701D0020511D0020C21C0020C01C00201F
:105C500070B50C460546FEF7D1FF04492A46234697
:105C6000BDE870400978FFF7D4BA00BF511D00208D
:105C700070B5484E3368013333600AF005F80AF016
:105C800031F844F620600AF015F8417804460429FA
:105C900008D0414804F044FA204604F0C7FA012035
:105CA000002147E00578446804F0C0FA012D4DD189
:105CB00033683A4C042B0BD90FF0D2F803783BB180
:105CC000A36803B1984740F29311354800F076FC81
:105CD00023690BB10020984734681E21013CE4B2CF
:105CE0001E2C28BF1E24A4F12005C4F1200321FA94
:105CF00003F301FA05F51D4347F2810301FA04F4A9
:105D00009C4275F1000319D2B4F5616F75F100037F
:105D100017D2B4F5167F75F1000315DA3C2C75F136
:105D2000000300DA0A21002004F046FB01460019B6
:105D300045EBE171FFF78CFF1A4B0EE04FF4E144A5
:105D400000254FF41671EEE73C21ECE7032D06D158
:105D500020460021FFF77CFF134B187870BD9DB9DA
:105D6000356009F04BFFFEF749FFFFF75FFA036864
:105D70001B6898470D4BC3E90001084B1B690BB129
:105D8000012098470A4BE8E70A48294604F0C8F979
:105D90000A2085E7981D0020F3BC0108A01D002003
:105DA0007DDF0108C21C0020701D00203002002091
:105DB000C41C002014BD0108054B1870054B1A7057
:105DC0000022054B1960054B1A705A70704700BFCE
:105DD0006B1D00206A1D0020641D0020681D00202E
:105DE00008B50AF06DF8C0B2F22828BFF22008BD4D
:105DF000002337B54FF47A7201930B4B02FB00F48A
:105E00001D68B4FBF2F42B681BB92921074800F088
:105E1000D5FB2246286801A906F08CFE012814BF94
:105E20000020019803B030BD541D00207DDF010823
:105E3000022818BF00200AF03BB90000F0B5304B33
:105E400005461E7885B0002E57D101228DF80F60CF
:105E50001A7009F07DFA07230C222A4CCDE9003292
:105E600028460DF10F022849231D0EF0D5FC0E2304
:105E7000264928464FF47A776371A37126610EF0A4
:105E80008FFC2349607004F1080328460DF10F02CE
:105E9000CDE900670EF0E0FC42F210730DF10F0245
:105EA0002846CDE900631B4904F10A030EF0D4FC37
:105EB000194928460EF074FC04F10C031749A07030
:105EC0000DF10F022846CDE900670EF0C5FC28460B
:105ED00013490EF065FC9DF80F30E07053B1114886
:105EE00004F01EF9104B1B6803B1984768210F4856
:105EF00000F064FB2069FFF79BFF05B0F0BD00BF19
:105F00009E1D0020741D002039BD01083CBD010804
:105F100040BD010849BD010855DE010852BD010818
:105F20005DBD010862BD0108A01D00207DDF0108E4
:105F300070B5294BC0B21B78984206D10EF090FF85
:105F40000EF05AFC254B187870BD254C0EF088FFDA
:105F5000FFF774FF94F905000BF002FE09F0C4FF8F
:105F600020790BF0CCFD09F0B5FF1E4EA07909F0A9
:105F7000C3FF60780AF096F8326812F0010213D17C
:105F80000421194D08462A60696006F053FC286018
:105F900018B95121154800F011FB0123144A154985
:105FA0001148336010F04EFB134B1A680AB90E4AC1
:105FB0001A60FEF723FEFFF739F903681B6898475C
:105FC00001220E4BC3E900010D4B5A72E3780BB16D
:105FD0000C4BB8E70C4BB6E76F1D0020C41C00202B
:105FE000741D0020481D0020901D00207DDF010849
:105FF000000000207D570008541D002030020020C2
:10600000581D00206C1D0020C31C0020034B93F87A
:106010002F30022B0CBF022000207047D00200203E
:10602000F8B51D4600234171BDF818100446174607
:106030000360C18002B115B923712046F8BD28461E
:1060400006490FF0C9FC064610B920712660F4E736
:106050002A46394612F016F82571F7E7E4E50108FB
:1060600010B50446006808B10FF0B8FC204610BD1A
:106070007FB5304E0446336823B940F2C9112E482B
:1060800000F09CFA002C52D000222C4B1A80D4E94C
:106090001C23134317D02A4B1D6807F0CDFA014685
:1060A0002848A847FEF7AAFDFFF7C0F8036859681B
:1060B000D4E91C238847D4E91C232349C1E90023E0
:1060C0002249C1E90023FEF799FDFFF7AFF8036805
:1060D0001B6898471E4B1F4AC3E90001237AC3F38C
:1060E000C0031370637F13B3237F03B308201A49DF
:1060F0000FF068FC054630B163890093237FA26EE0
:10610000617FFFF78DFF03958DB1002330681A463C
:10611000006803A906F0B2FB012808D0039C34B143
:106120002046FFF79DFF082120460FF059FC04B0E0
:1061300070BD00BF541D00207DDF01088A1D0020B6
:10614000D002002075BD0108380200204002002066
:10615000300200208E1D0020E4E5010838B542F22F
:10616000107009F0A7FD0446A0B10578032D03D1F6
:1061700000214068FFF76CFDD4F8A000FFF778FF1E
:10618000237A13B10022044B1A7020460BF0ACFAAC
:10619000284638BD0125FBE7711D0020002310B5FE
:1061A000114C84F8343009F04DFD08B109F06CFD54
:1061B000FFF7D4FF012809D903280AD00B484FF470
:1061C0002E7100F0FBF94FF0FF3001E0084B18781A
:1061D00010BDFFF71BFF022809BF0123054B84F800
:1061E0003430054BF3E700BFD00200207DDF01080B
:1061F000C41C0020701D0020501D0020FF23002122
:106200000D4A13700D4A13700D4A13700D4A137026
:106210000D4A13700D4A13700D4A13700D4A137016
:106220000D4A13700D4A13700D4A13700D4AC2E9DE
:1062300000111372704700BF6E1D00206D1D0020FD
:106240006F1D0020891D0020881D00208D1D00204D
:106250008C1D00206C1D0020701D0020501D002092
:10626000511D0020581D0020034AC0E900210022D2
:1062700002818272704700BF4849F8F9437A10B52D
:1062800004461BB92721094800F098F9207A08B97B
:10629000002010BDA37A002BFBD0606803681B6848
:1062A00098470028F4D00023A372F2E77DDF0108AD
:1062B0002DE9F041002427462646A04686B0054633
:1062C0008DF80F108DF81740FFF7D8FF9DF80F30AD
:1062D00003F00F038DF80F30686803685B68984718
:1062E000C8B1686801220368CDF80080DE680DF14E
:1062F0000F012B78B0470646686801220368CDF885
:1063000000801F690DF117016B78B8470746686870
:1063100003689B6898470134E4B246B13FB19DF8E9
:1063200017309DF80F2003F00F039A4203D0052C7D
:10633000D2D1002002E0601F18BF012006B0BDE8E6
:10634000F0817FB505460E46FFF798FF6868036841
:106350005B689847044620B302226B7868688DF822
:106360000C30EB7803A98DF80D3003680092DC68DF
:106370000122AB78A0470446686814B90123AB72C8
:106380000CE04FF40042036800921C69032231467E
:10639000AB78A04704466868002CEFD003689B6880
:1063A0009847204604B070BD13B501A90446FFF715
:1063B000C8FF70B19DF80530082B07D19DF8042067
:1063C0009DF80630134301D101232372207A02B0D5
:1063D00010BD2072FAE7002310B5038183720446D2
:1063E000406803681B68984730B1012320466372F8
:1063F000BDE81040FFF7D8BF10BD000010B4054C39
:10640000237822B11943217010BCFFF751BF23EA52
:106410000101F8E7480200202DE9F04340488BB025
:1064200003F07EFE07F016F92425079007993D48F2
:1064300003F076FE0798684303F00EFF04463A48DF
:1064400003F06EFE8CB1204607990DEB050207F0B4
:1064500063FC0023354E364F07900893089A079B3C
:106460009A421DD3204603F0E1FE06F003F90446EC
:1064700006F00EF9214602462E4803F051FE2E4B3F
:106480002E4819889A888B1A03F04AFE2C4B1B68F9
:1064900003B198472B480BB0BDE8F04303F040BE72
:1064A000089B05FB03431B7B042B98BFF25C099BF5
:1064B00088BF3F22642B83BF6420B3FBF0F30899AD
:1064C000002382BF05FB01418969B1FBF3F3089901
:1064D0000898DDF820C0DDF820E0DDF82080DDF848
:1064E000209005FB004005FB0949D9F81C9005FBED
:1064F0000141CDE9033905FB08439B69029305FB84
:106500000E439B68019305FB0C431B8C00930369AE
:106510004968384603F004FE089B013308939DE761
:1065200082BD01088EBD010899BD01088ABE01081F
:10653000CEBD0108A5AF01089C1F002000BE0108C8
:106540002C1E002062B30108014B1860704700BF89
:10655000481E002073B5134E054632780C46124B88
:106560001AB91A780AB172B6FEE7012200211A7030
:106570000E48642211F0AEFD234664210C4A0B48FC
:10658000009512F01FFD0B4B1B6803B198470124C7
:10659000064D284603F008FE72B6074B3470013BE7
:1065A000FDD1F6E7251E0020B91D0020BA1D0020F0
:1065B00024BE0108481E0020FFFF0F00F7B5184E4B
:1065C000054632780C46174B1AB91A780AB172B6DA
:1065D000FEE7012200211A701348642211F07AFDAF
:1065E00023466421114A1048009512F0EBFC104B31
:1065F0001B680BB10C4898470E4B1B6803B19847BA
:106600000124094D0C4F284603F0CEFD384603F017
:10661000CBFD72B6094B347000BF013BFCD1F2E7F1
:10662000241E0020B81D0020BA1D00204CBE010809
:10663000B41D0020481E00205BBE0108FFFF0F00B4
:10664000F8B5DFF870C003681B4FCCF80030436822
:106650001A4E3B6083681A4D3360C36819492B603A
:106660000369194A0B604369184C13608369C06958
:106670002360174B1860DCF8000038683068286821
:10668000144E0968144D126822681B6864220021A8
:10669000284611F01FFD236832466421284612F077
:1066A00091FC284603F080FD0C4B00BF013BFCD160
:1066B000ECE700BF341E0020381E0020401E0020E2
:1066C000441E00203C1E0020201E0020281E00200A
:1066D000301E002077BE0108BA1D0020FFFF0F000A
:1066E000074B1B6803B198471EF0040F0CBFEFF374
:1066F0000880EFF309808169004A1047416600086D
:10670000481E0020002103E00A4B5B58435004312F
:1067100009480A4B42189A42F6D3094A02E000237C
:1067200042F8043B074B9A42F9D300F00DF8FBF70F
:1067300021F8704704EA010800000020100600203C
:10674000100600206C2B0020314B82B01A6842F4F6
:1067500080721A6099682F4A0A409A601A6822F07B
:10676000885222F001121A601A6822F480221A60FC
:106770009A6822F47D029A600022DA6001921B6816
:1067800013F4007318BF01230193019B012B37D130
:106790004FF48051204B1A68A3F5806322F0010268
:1067A000C3F80024D3F8002422F00202C3F8002426
:1067B000D3F8002422F00402C3F800245A6A42F0FD
:1067C00080525A62154A11605168C906FCD49A6811
:1067D0009A609A689A609A689A605A6822F460424D
:1067E0005A605A6842F440425A609A6822F00302A2
:1067F0009A609A689A60064A936813F00C0FFBD16E
:106800004FF00062064B9A60064ADA6002B07047A9
:10681000003802400CC0FF88003C0240007000407D
:1068200000ED00E00003FA0570B5064688B02D487B
:1068300001F0DAFC2C4B1A680092009A91073AD5C5
:1068400001214FF4007001F01BFF012001F01AFD3F
:10685000264A536843F400335360A2F53742536825
:106860001B07FCD50024012502A801F0F7FC1D48F8
:1068700002A906948DF81C50ADF80C4001F0C8FC3C
:106880002A4606233146174801F008FD29461548D7
:1068900001F0EFFC0221134801F090FD114801F0D6
:1068A0007FFD134D01940F4C0221204601F080FD25
:1068B00058B108B070BD1A6842F001021A60009A1F
:1068C0009207BDD41A680092F9E7019B0133019346
:1068D000019BB3F5805FE7DB38212846FFF76EFEAA
:1068E000E2E700BF002401400038024000270140D9
:1068F0007DDF010808B5002001F0C4FC0021074835
:1069000001F0B7FC00214FF4007001F0B9FE044A19
:10691000136823F00103136008BD00BF0024014089
:106920000038024013B5072301460122114801F047
:10693000B5FC02210F4801F041FD0E4801F030FD89
:1069400000230D4C019302210A4801F031FD28B1CA
:10695000084802B0BDE8104001F027BD019B01339B
:106960000193019BB3F5805FEDDB4C212046FFF7DF
:1069700025FEE8E7002401407DDF010870B50646EA
:106980000825FFF751FF00243046FFF7CBFF013DFC
:106990000444F9D1FFF7AEFFC4F3CF0070BD00008F
:1069A00008B51120FFF7EAFF10F012FD0146084874
:1069B00010F01AFE10F0F4F803A3D3E9002310F04E
:1069C00047F910F0FFFB08BD2FDD24068195F33F4A
:1069D00000F07F450F4A536A43F080535362A2F59B
:1069E000E4325368D906FCD41368022823F4C05358
:1069F00006D143F4C05313605368DB06FCD47047E0
:106A0000012802D143F48053F5E70028F3D143F481
:106A10000063F0E70038024010B50D4B5A68D2060B
:106A2000FCD41C6804F4C052B2F5C05F0BD014F45F
:106A300080500AD114F4006404D106482B21FFF7DA
:106A4000BDFD204610BD0220FCE70120FAE700BF93
:106A5000007000407DDF010810B50446012001F000
:106A6000BDFC012C27D1174A136843F001031360C2
:106A7000154B1A6842F480321A601A689103FCD5EB
:106A800000229A609A68002AFCD19A6842F00202B9
:106A90009A600D4B9A681207FCD54FF480321A6049
:106AA0000A4B0B4A20461A60FFF794FFBDE81040DE
:106AB000002001F087BC022CDAD142210548FFF703
:106AC0007DFDD5E7003C0240003802404C0200202A
:106AD0000024F4007DDF010838B50546012001F0EF
:106AE0007DFC022D01BF144A136843F001031360BB
:106AF000124B1A6842F480721A601A689205FCD52B
:106B00005A6822F4604242F440425A6000229A607D
:106B10000A4A946814F00C04FBD14FF4807313609C
:106B2000074B084A28461A60FFF754FF2046BDE885
:106B3000384001F047BC00BF003C02400038024032
:106B40004C020020D0FE3F00114B5A6B92051DD421
:106B50005A6A42F080525A62A3F5E4331A6842F44A
:106B600080721A601A68D005FCD5094B5A6B42F442
:106B700080725A635A6BD105FCD55A6B9205FCD5CD
:106B8000044B1A6822F480721A601B68704700BFB9
:106B90000038024000700040054B5A6B910706D444
:106BA0005A6B42F001025A635A6B9207FCD5704748
:106BB00000380240094B5A6A42F020025A629A6930
:106BC00042F020029A619A6922F020029A61002222
:106BD000A3F509331A801A855A62704700380240BB
:106BE00015210D4B02389A69484342F020029A6100
:106BF0009A69012122F020029A610022A3F509334B
:106C00001A85D86299825A621A8219801A8AD20722
:106C1000FCD500221A80704700380240002349F654
:106C2000FE7282B00193019B934201DD02B0704776
:106C3000019B01330193F6E7002340F6FE7282B018
:106C40000193019B934201DD02B07047019B013328
:106C50000193F6E7002382B00193019BB3F5CC7F4B
:106C600001DD02B07047019B0133F5E718B301283D
:106C700001D1FFF7EFBF104B00219A69013842F0B4
:106C800020029A619A6922F020029A610B4B1A68DD
:106C90004FF47A73B2FBF3F2094B013A92B21A85C0
:106CA0000122D8629A82596219821A801A8AD207FE
:106CB000FCD500221A807047003802404C020020A8
:106CC0000014004000F1774303F57803B3F5804FDB
:106CD0002DE9F04105460C4616462DD202F1F73358
:106CE00003F608030344B3F5804F25D2FFF794FE63
:106CF000804610B10020FFF76DFE01F087FB0127F1
:106D000026442D1BA6420AD101F090FBB8F1000FDA
:106D100002D04046FFF75EFE3846BDE8F08141F6FE
:106D2000027001F08BFB281914F8011B01F0E2FB43
:106D3000042818BF0027E5E70027EDE710B5044653
:106D4000084604F1774101F57801B1F5804F0CD286
:106D500002F1F73303F608032344B3F5804F04D25E
:106D6000214611F08FF9012010BD0020FCE7000042
:106D700008B5114B984215D003F58063984213D0A3
:106D800003F58063984211D003F5806398420FD0D9
:106D900003F5006398420DD01421084B084A0948B6
:106DA00010F036FF002008BD0120FCE70220FAE7C2
:106DB0000320F8E70520F6E7000002408FBE010837
:106DC00009BF0108A8BE01080F2808B505D93B2155
:106DD000084B094A094810F01BFF0122084B02FA30
:106DE00000F0596821EA000159601A6822EA00009F
:106DF000186008BDF1BE010834BF0108A8BE010833
:106E0000000401400F292DE9F84F81460C469246B7
:106E10001E4605D954215A4B5A4A5B4810F0F8FED9
:106E20004FF00108594F00F0B9F87B6808FA04F8F0
:106E300023EA08037B603B68554A23EA08033B606A
:106E4000136A032C43F00103524D136230D80F2212
:106E5000AB684FEA840B02FA0BF223EA0203AB6041
:106E60004846FFF785FFAB6800FA0BF01843A860AF
:106E70001AF0020F18BFBB684FEA06121CBF43EAA4
:106E80000803BB601AF0040F18BFFB68D2B21CBF26
:106E900043EA0803FB603B6843EA08033B603E4B60
:106EA000002C44D183F8062340221A60BDE8F88FF5
:106EB000072C12D80F22201FEB684FEA800B02FA32
:106EC0000BF223EA0203EB604846FFF751FFEB6841
:106ED00000FA0BF01843E860CAE70B2C13D80F2216
:106EE000A4F108002B694FEA800B02FA0BF223EAA7
:106EF00002032B614846FFF73BFF2B6900FA0BF0BA
:106F000018432861B4E70F22A4F10C006B694FEA23
:106F1000800B02FA0BF223EA02036B614846FFF78B
:106F200027FF6B6900FA0BF018436861A0E7012C9A
:106F300003D183F807238022B7E7022C04D183F81A
:106F400008234FF48072B0E7032C04D183F809239F
:106F50004FF40072A9E7042C04D183F80A234FF4FC
:106F60008062A2E7092C04D883F817234FF40002AB
:106F70009BE783F828234FF480725A6096E700BF9E
:106F8000FDBE010813BF0108A8BE010800040140AE
:106F9000003802400000014000E100E0144B98423C
:106FA00005D1144AD36943F00103D3617047124BF2
:106FB000984204D10F4AD36943F00203F5E70F4B1F
:106FC000984204D10B4AD36943F00403EDE70C4B1C
:106FD000984204D1074AD36943F00803E5E7094B17
:106FE0009842E3D1034AD36943F02003DDE700BFB1
:106FF0000000024000380240000402400008024045
:10700000000C0240001402400323490010B58468BC
:107010008B4024EA030484600124022A04FA01F468
:1070200007D0032A0DD0012A07D183682343836048
:1070300003E083688A401A43826083681C4384604B
:1070400010BD82681343F2E70F292DE9F041044691
:10705000884615461F4603D94B211A48FFF7AEFA5A
:107060002046FFF79BFF0323012021684FEA4802D7
:1070700093406FEA030C21EA03032360236800FABC
:1070800002F63343236000FA08F1A38809B267B11E
:10709000194389B2A180E368012D0CEA0303E36080
:1070A00007D0022D09D0BDE8F0819BB223EA01018F
:1070B000F0E7E3681E43E660F5E7E36895401D43AB
:1070C000E560F0E77DDF01080F2970B505460C4645
:1070D000164603D96B210E48FFF770FA2846FFF7D2
:1070E0005DFF0323E86861008B40DA43012E20EA4C
:1070F0000303EB6005D0022E03D02B6813402B60F6
:1071000070BDEB6806FA01F11943E960F5E700BFCD
:107110007DDF01080F2910B505D98121074B084AE9
:10712000084810F075FDFFF739FF03230268490096
:1071300003FA01F11143016010BD00BFF1BE010867
:10714000C7BF01084FBF01080F2938B504461546CF
:1071500005D987211B4B1C4A1C4810F059FD0F2AEA
:1071600003D988211A4B184AF6E7FFF717FF0729BA
:107170004FF00F0318D8006A8A00934020EA0303F7
:107180002362236A05FA02F21A4322620322236869
:1071900049008A4023EA020323600223226803FA9B
:1071A00001F11143216038BDA1F10802406A92004B
:1071B000934020EA03036362636A95401D4365625E
:1071C000E4E700BFF1BE0108A9BF01084FBF0108F5
:1071D00096BF010801238B409BB2038370470123B4
:1071E0008B409BB243837047012303FA01F189B2BC
:1071F0000AB10183704741837047008A80B2084119
:1072000000F00100704700000F2938B505460C4614
:1072100003D9B4210648FFF7D1F92868640020FAA1
:1072200004F404F00300431E5842584138BD00BF27
:107230007DDF0108808A80B2084100F001007047BC
:1072400010B5074C236853B9012005F0BDFB206041
:1072500028B9BDE8104036210248FFF7AFB910BD8C
:107260004C1E00207DDF010810B50B4C23681BB9B4
:107270003C210A48FFF7A2F9206842F2107105F09C
:10728000EBFC01280CBF0124002403D0402103485B
:10729000FFF794F9204610BD4C1E00207DDF010849
:1072A00010B5074C23681BB951210648FFF786F932
:1072B000002320681A46BDE81040194605F0DEBAE2
:1072C0004C1E00207DDF010810B50446FFF7B8FF13
:1072D000FFF7CAFF21461022034801F0DBFE0446F7
:1072E000FFF7DEFF204610BD0054004010B5FFF749
:1072F000A7FFFFF7B9FF01F085FE0446FFF7D0FFB7
:10730000204610BD08B513460A460146034801F061
:10731000B3FA003818BF012008BD00BF0054004078
:1073200008B513460A460146034801F0A5FB00389C
:1073300018BF012008BD00BF0054004008B5134627
:107340000A460146034801F075FC003818BF0120C9
:1073500008BD00BF0054004008B513460A46014668
:10736000034801F0F9FC003818BF012008BD00BF38
:107370000054004008B513460A460146034801F090
:1073800045FD003818BF012008BD00BF0054004073
:107390000123064A83405169194205D05361044BC9
:1073A00053F8203003B11847704700BF0004014074
:1073B000501E00200F2838B504460D4603D926215B
:1073C0000348FFF7FBF8034B43F8245038BD00BFD8
:1073D0007DDF0108501E00200020FFF7D9BF0120EB
:1073E000FFF7D6BF0220FFF7D3BF0320FFF7D0BFC0
:1073F0000420FFF7CDBF08B50920FFF7C9FF08201B
:10740000FFF7C6FF0720FFF7C3FF0620FFF7C0FF07
:10741000BDE808400520FFF7BBBF08B50F20FFF708
:10742000B7FF0E20FFF7B4FF0D20FFF7B1FF0C20D0
:10743000FFF7AEFF0B20FFF7ABFFBDE808400A20C7
:10744000FFF7A6BFFEE7FEE7FEE7FEE7FEE7FEE783
:10745000FEE7FEE7FEE7FEE7FEE7FEE7FEE7FEE704
:10746000FEE7FEE7FEE7FEE7FEE7FEE7FEE7FEE7F4
:10747000FEE7FEE7FEE7FEE7FEE7FEE7FEE7FEE7E4
:10748000FEE7FEE7FEE7FEE7FEE7FEE7FEE7FEE7D4
:10749000FEE70A22B0FBF2F302FB130040EA0310FE
:1074A000C0B27047CA22024B5A6253225A627047D6
:1074B00000280040014B1860704700BF901E00205C
:1074C0004FF400320F4B10B50F4C5A61E368DB05E7
:1074D00003D430210D48FFF771F8FFF7E3FF4FF4B5
:1074E0000072A36823F48853A360094BC3F8842077
:1074F000FF236362074B1B6813B1BDE810401847B8
:1075000010BD00BF00040140002800407DDF0108DD
:1075100000E100E0901E00202DE9F04F9046394A2E
:1075200087B014781F4681469DF840309DF844B0DE
:107530002CB99521344B354A354810F069FB421E71
:107540001E2A5DD80C295BD8A8F5FA62632A57D8A1
:10755000172F55D83B2B019352D8BBF13B0F4FD877
:1075600008F13000C0B2FFF794FF82460846FFF7EB
:1075700090FF05024846FFF78CFF45EA0A4A40EAB9
:107580000A0A3846FFF785FF019B06461846FFF7B3
:1075900080FF05025846FFF77CFF45EA0645284371
:1075A0001C4DFFF77FFFEA68019B42F080024AF41E
:1075B000005AEA60EA685606FCD5C5F804A02860BF
:1075C000EA6822F08002EA60124AD0688006FCD5A0
:1075D000FF20506203A88DF80D308DF80F908DF8C4
:1075E0001010ADF811808DF80E708DF80CB002F00F
:1075F000D9FC094BC3E90001204607B0BDE8F08F74
:107600000024F9E7941E0020DABF010850C00108E9
:10761000E3BF010800280040981E002007B503784A
:107620000193437800938378B0F805200179C078FE
:10763000FFF772FF03B05DF804FB0000264B10B5A6
:107640001B7804461BB9ED212448FEF7B7FF244AF6
:10765000D36823F02003D360D3689B06FCD513685E
:107660005268C2F3035101EB8100C2F3034101EB05
:107670004001C9B201F5FA61A4F80510C2F3003166
:10768000C2F3032001EB810100EB41012171C2F340
:10769000011101EB810102F00F0202EB4102E270E5
:1076A000C3F30152C3F3034102EB820201EB420236
:1076B000A270C3F30232C3F3032102EB820201EB97
:1076C00042026270C3F3021202EB820203F00F0364
:1076D00003EB4203237010BD941E00207DDF0108E0
:1076E000002800401FB501A8FFF7A8FF01A802F07D
:1076F00059FC05B05DF804FB08B5FFF725FA1D4BF2
:107700001A6842F480721A601A68D005FCD5FFF737
:10771000C9FE194A536B23F4403343F48203536385
:10772000164BDA6842F08002DA60DA685106FCD55E
:10773000FF221A611A6942F4FE021A619A6822F065
:1077400040029A609A6822F44C529A60DA6822F0F9
:107750008002DA60094BDA689206FCD5FF225A6291
:107760000122074B1A70FFF7BDFF064BC3E900016A
:1077700008BD00BF007000400038024000280040F3
:10778000941E0020981E002008B5094B1B7823B9D1
:107790004FF494710748FEF711FFFFF783FE064B85
:1077A0009A6822F480729A60FF225A6208BD00BF74
:1077B000941E00207DDF01080028004008B5144B0E
:1077C0001B7833B94FF49871124B134A134810F0D9
:1077D0001FFAFFF767FE124BDA6822F48072DA6054
:1077E000104A916841F400319160116841F4003110
:1077F0001160F0210C4A82F829134FF40071516096
:107800009A6842F488529A60FF225A6208BD00BF0B
:10781000941E0020DABF01083BC00108E3BF010845
:10782000002800400004014000E100E0F8B51E46D9
:10783000194B15461B7833B940F25311174B184AB0
:10784000184810F0E5F9184CFFF72CFEA36823F454
:107850008073A360E36823F48073E360FFF719FE8D
:1078600007460846FFF715FE01042846FFF711FEFC
:1078700005463046FFF70DFE41EA0761014341EA44
:107880000521E368DB07FCD5FF23E1616362BDE806
:10789000F840FFF793BF00BF941E0020DABF010835
:1078A00029C00108E3BF010800280040037842789E
:1078B0008178C078FFF7BABF38B50D46044604F0AA
:1078C00099FD4FF0E022136923F00103136104F0E6
:1078D000AFFD25B11B4A536843F00603536072B6EF
:1078E000BFF34F8FBFF36F8F174A0120136823F048
:1078F000030343F4007343F00103136000F07AFDC7
:10790000124B1A6942F004021A6130BF1A6922F060
:1079100004021A610E4B0F4A1B6893420BD10220DE
:10792000FFF7DAF84FF0E022136943F00103136127
:1079300004B162B638BD084A9342F3D10020FFF784
:107940008BF8EFE7002004E00070004000ED00E05D
:107950004C020020D0FE3F000024F40062B67047C5
:1079600000220E4B10B51A700D4A0E4C138820469B
:1079700023F040031B041B0C13800D210222FFF790
:10798000A3FB204602220E21FFF79EFB2046BDE806
:10799000104002220F21FFF797BB00BFA01E00205E
:1079A0000038004000040240294A38B5136A0546F1
:1079B00043F480531362052226480C461146FFF714
:1079C000C3FB052206212348FFF7BEFB0522072142
:1079D0002048FFF7B9FBC5B1022205211D48FFF77A
:1079E00013FB022206211B48FFF70EFB0222072190
:1079F0001848FFF709FB012C1BD144F451740122F4
:107A0000154B1C80154B1A7038BD2A4605211148AC
:107A1000FFF7FAFA2A4606210E48FFF7F5FA2A463A
:107A200007210C48FFF7F0FA012C09D144F45974EE
:107A3000E5E7022CE1D0032C0CBF03240024DCE793
:107A4000022CF3D0032C14BF00240324EEE700BF64
:107A5000003802400000024000300140A11E00201A
:107A600000220E4B10B51A700D4A0E4C138820469A
:107A700023F040031B041B0C138005210222FFF797
:107A800023FB204602220621FFF71EFB2046BDE80D
:107A9000104002220721FFF717BB00BFA11E0020E4
:107AA0000030014000000240054A064B12789881E0
:107AB0001989C90701D4002AFAD19889C0B2704740
:107AC000A11E00200030014010B50121094800F03E
:107AD00037FE68B10121074800F02EFE012105485C
:107AE00000F039FE044B1B6813B1BDE81040184785
:107AF00010BD00BF00040040A41E0020054AD3684A
:107B000023F4E0631B041B0C43F0BF6343F4003316
:107B1000D360704700ED00E020220021114B10B52A
:107B2000C3F88420104B114C1A6A204642F480425C
:107B30001A625A6942F480425A615A6922F48042B8
:107B40005A610B4A91811A6A092122F480421A6211
:107B50000222FFF7B9FA2046BDE8104002220A21AE
:107B6000FFF7B2BA00E100E0003802400000024036
:107B700000380140084A08B513889B0605D5074B15
:107B80001B6813B19088C0B29847034B044A9B8886
:107B9000DBB2137008BD00BF00380140AC1E0020EE
:107BA000A81E002010B504468021084800F056FEAB
:107BB0000028F9D02146054800F030FE034C402152
:107BC000204600F04BFE0028F9D010BD00380140DF
:107BD00010B5441E14F8010F00B910BDFFF7E2FF05
:107BE000F8E7000008B5024800F01CFEC0B208BD6E
:107BF000003801402DE9F0410E4601214FF4C068E4
:107C0000074688B0084614461D4600F02DFD0121A8
:107C10004FF4804000F034FD3C4B3D4802A9CDE9D3
:107C2000028300F08DFC07220921394800F0C4FCD2
:107C300007220A21364800F0BFFC452E04973CD1AC
:107C40004FF48063ADF81830072C42D10023ADF813
:107C50001430052D4ED14FF48053ADF8163000236B
:107C6000ADF81C300C232B4804A9ADF81A3000F0F5
:107C700077FD294B1A6802B1012240F225512548AF
:107C800000F0D4FD0121234800F0BCFDFFF7AAFF5E
:107C900025238DF804309DF8383001A88DF8053083
:107CA00000238DF8063001238DF80730FFF726FFFB
:107CB00000F07EFA08B0BDE8F0814F2E02D1ADF899
:107CC0001880C1E70023072CADF818300DD15921D9
:107CD00007E0082C02D14FF48053B8E7092CB8D143
:107CE00054210E48FEF76AFCB3E7082CAED0092CED
:107CF000AFD1F0E70F2D02D14FF44053ADE7022D85
:107D00000CBF4FF400530023A7E700BF020200019D
:107D10000000024000380140AC1E00207DDF010859
:107D20000E2307B5082200934E210123FFF762FFBF
:107D300003B05DF804FB0000402200210D4B0E480B
:107D4000C3F884200D4B5A6A42F400325A629A6991
:107D500042F400329A619A6922F400329A61084A28
:107D600091815A6A032122F400325A620222FFF7FB
:107D7000ABB900BF00E100E0000002400038024063
:107D80000044004008B5024800F04CFDC0B208BDF8
:107D9000004400402DE9F0471D46262388B08DF8A9
:107DA000043000239DF84080824601A814468DF8D7
:107DB00006308DF807300E469DF844709DF84890C7
:107DC0008DF80580FFF79AFE00F0F2F901210846D0
:107DD00000F04AFC01214FF4003000F05DFC67B177
:107DE0000821514B5148CDE9021302A900F0A8FB2C
:107DF000072203214D4800F0DFFBB9F1000F0CD042
:107E00000422494B494802A9CDE9022300F098FB1E
:107E100007220221454800F0CFFB452ECDF810A0E7
:107E200044D14FF48063072CADF818304BD10023B8
:107E3000ADF81430052D57D14FF480530024ADF820
:107E40001630ADF81C40B9F1000F58D1ADF81A90BA
:107E500077B1BDF81A3043F00403ADF81A30344B53
:107E60001A6802B1012240F22551324800F0DEFCCE
:107E7000304804A900F074FC01212E4800F0C2FC37
:107E80000FB1FFF77FFF26238DF8043000238DF814
:107E90000630012301A88DF807308DF80580FFF723
:107EA0002DFE00F085F908B0BDE8F0874F2E02D115
:107EB0004FF4C063B7E70023072CADF818300ED19C
:107EC0004FF4827107E0082C02D14FF48053AFE7E2
:107ED000092CAFD1FF211848FEF770FBAAE7082C48
:107EE000A5D0092CA6D1F0E70F2D02D14FF44053B5
:107EF000A4E7022D0CBF4FF4005300239EE7082394
:107F0000224640F227710B48ADF81A3000F08EFC83
:107F100040F22661074800F0A7FC224640F22661A5
:107F2000044800F083FC93E70201000100000240D6
:107F3000B01E0020004400407DDF010870B50446FB
:107F40000025134E8021134800F088FC60B12146C3
:107F5000104800F063FC00240E4D0D4E40212846D1
:107F600000F07CFC50B170BD0135B5F5801FE9D340
:107F700040F251113046FEF721FBE3E70134B4F53E
:107F8000801FEBD34FF4AD713046FEF717FBE5E7EA
:107F90007DDF01080044004008B5064B024618602A
:107FA00000B1012240F22551034800F03FFC0120BE
:107FB00008BD00BFB01E002000440040124810B5AC
:107FC0000388124C13F0200F08D0114B1B682BB103
:107FD0000288D20713D48088C0B298470A48038821
:107FE0005B0607D540F2266100F03EFC094B1B689A
:107FF00003B19847044B9B88DBB2237010BD00F09F
:1080000011FCC0B22070E9E700440040A81E002027
:10801000B01E0020B41E0020BFF34F8F0449054B53
:10802000CA6802F4E0621343CB60BFF34F8FFEE7F0
:1080300000ED00E00400FA0510B5441EE3B2052B84
:1080400003D917211148FEF7B9FAFEF7A5FD45F24D
:1080500055520F4B1A60DA68D207FCD4052C06D8AB
:10806000DFE804F0030A0C0E101201225A604CF6ED
:10807000CC42074B1A6010BD0222F7E70322F5E756
:108080000422F3E70522F1E70622EFE77DDF01088E
:108090000030004038B5224C236853B95F2000F00F
:1080A00013FB204D38B1204B236001232B7000F0CF
:1080B0001BFB206838BD5E2000F006FB18B11B4B8F
:1080C00023600223F2E75D2000F0FEFA18B1184B9E
:1080D00023600323EAE75C2000F0F6FA18B1154BA1
:1080E00023600423E2E75B2000F0EEFA18B1124BA4
:1080F00023600523DAE75A2000F0E6FA18B10F4BA7
:1081000023600623D2E7592000F0DEFA18B10C4BA9
:1081100023600723CAE70B4B2360FF23C6E700BF9A
:10812000BC1E0020C01E00205CC001086CC00108FD
:1081300082C001089DC00108ACC00108BBC0010895
:10814000D4C00108EBC8010838B5084B084D1A78AF
:1081500052B9012420461C7000F0DEFA287020F08D
:10816000FF01204600F0C8FA287838BDB81E00206C
:10817000B91E002010B50446012000F0CDFA20F011
:10818000FF0121430120BDE8104000F0B5BA08B559
:10819000FFF7F0FFFFF740FF012008B500F0BCFA41
:1081A000C0B210B90120FFF7F2FFFFF735FF000062
:1081B00030B5012403780A4D03F01F029440C278C1
:1081C000590952B1074A2B44D26842781201D2B2FF
:1081D00083F8002345F8214030BD2031FAE700BF85
:1081E00000E100E000ED00E008B5084B98420BD13B
:1081F00001214FF4007000F05BFABDE80840002157
:108200004FF4007000F054BA08BD00BF00240140D4
:1082100043680A7923F0407323F4807343EA02230E
:108220000A6810B513434360D1E9032313438A68F6
:1082300084681343084A224013434A7943EA4203BD
:1082400083600A7D036B013A23F0F873D2B243EAEC
:108250000253036310BD00BFFDF7FFC000234FF0C2
:1082600040720360C0E903238380836001230375A8
:108270007047836819B143F001038360704723F0AE
:108280000103FAE7044B5A6818B142F400025A603D
:10829000704722F40002FAE7002701401D2970B55B
:1082A0001AD90726A1F11E04C56D04EB4404A640AB
:1082B00025EA0605A3402B43C365062A35D81F24AB
:1082C000013A036C02EB8202944023EA040301FAB0
:1082D00002F21A43026470BD13290CD90726A1F1DA
:1082E0001404C56804EB4404A64025EA0605A3402F
:1082F0002B43C360E1E709290CD90726A1F10A0441
:10830000056904EB4404A64025EA0605A3402B4377
:108310000361D2E70725446901EB4106B54024EA31
:108320000504B34023434361C7E70C2A0CD8D41F8C
:108330001F22C36B04EB8404A24023EA020301FA68
:1083400004F21A43C263C6E7122A0DD8A2F10D0344
:108350001F22846B03EB83039A4024EA020401FA90
:1083600003F222438263B6E7182A0CD81F24133A7B
:10837000436B02EB8202944023EA040301FA02F207
:108380001A434263A7E71F24193A036B02EB8202E8
:10839000944023EA040301FA02F21A4302639AE7C3
:1083A000836843F0804383607047806D80B270477C
:1083B0000368194214BF012000207047C9430160BF
:1083C00070470000044B1A6818B142F002021A60AC
:1083D000704722F00202FAE7003C0240044B1A68A0
:1083E00018B142F004021A60704722F00402FAE762
:1083F000003C0240044B1A6818B142F008021A60AF
:10840000704722F00802FAE7003C0240044B5A6829
:10841000D20741BF034ADA60034ADA60704700BFFF
:10842000003C0240EFCDAB8905040302024A5368C9
:1084300043F0010353607047003C0240014B9861D8
:10844000704700BF003C0240084B9A69D10709D42D
:108450009A69D20508D49B6913F4F05F14BF032016
:10846000042070470120704702207047003C024002
:10847000042313B504468DF80730FFF7E5FF8DF8A8
:1084800007009DF80730012B0AD11CB905238DF890
:10849000073007E0FFF7D8FF013C8DF80700F0E751
:1084A000002CF3D09DF8070002B010BD10B50446B3
:1084B0004FF40040FFF7DCFF042804BF00232360D3
:1084C00010BD000038B504464FF400400D46FFF7DC
:1084D000CFFF04280BD1064A4FF40040536823F421
:1084E000807353602560BDE83840FFF7C1BF38BDD9
:1084F000003C024038B504464FF400400D46FFF7FB
:10850000B7FF04281BD135B125704FF40040BDE8FA
:108510003840FFF7ADBFFF2324F0030504F0030448
:108520002968E40003FA04F421EA04042846FFF76A
:10853000BDFF21462846BDE83840FFF7C3BF38BD20
:108540002DE9F0410022012703260B6807FA02FEFD
:108550003EEA03032BD1036891F804C0540006FAE5
:1085600004F86FEA080523EA08080CFA04F30CF192
:10857000FF3C43EA0803BCF1010F03600ED8836897
:108580002B404D79A5401D43856083889BB223EA2B
:108590000E058B7993409BB22B438380C36806FA08
:1085A00004F523EA0505CB79A3402B43C3600132D0
:1085B000102ACAD1BDE8F08110B50F2401F00703DD
:1085C000C90800EB8100016A9B009C4021EA04017C
:1085D0000162016A9A400A43026210BD1E4B10B547
:1085E0009A6802F00C02082A1DD00BD80AB1042A9E
:1085F00019D04FF400425B68C3F34233013302FAEF
:1086000003F311E00C2AF4D19A68144CC2F38342AC
:108610009968A25C9B68124B5343C1F381520132AB
:10862000B3FBF2F300E00E4B0B4A036093680D4975
:10863000C3F30313CC5C0368E34043609468C4F362
:1086400002240C5D23FA04F484609268C2F3C2220F
:108650008A5CD340C36010BD003802406002002035
:108660000024F40050020020044BDA6911B11043D9
:10867000D861704722EA0000FAE700BF00380240E4
:10868000044B1A6A11B110431862704722EA0000C5
:10869000FAE700BF00380240044B5A6A11B1104398
:1086A0005862704722EA0000FAE700BF0038024033
:1086B000044B5A6911B110435861704722EA000017
:1086C000FAE700BF003802404309012B054B00F0D8
:1086D0001F000CBF1B685B6B23FA00F000F0010069
:1086E000704700BF00380240024A536B43F080736A
:1086F0005363704700380240002382B00193054B5A
:108700000193019B03EB80030193019B196002B06D
:10871000704700BF50280040002382B00193054BF2
:108720000193019B03EB80030193019B186802B046
:10873000704700BF50280040C94389B2018270478A
:10874000038A828911EA030092B203D00A4214BF5D
:10875000012000207047C94389B2018270470000A0
:1087600030B50D460446038AEA889BB223F4405391
:108770001343898903828389288923F4B052AB8803
:1087800022F00C020343688912040343120C9BB2CB
:108790001343A381A38A85B09BB223F440730B4398
:1087A0006846A382FFF71AFFDDE9023214498C42C2
:1087B00008BF13461922A18953432A680D044CBFF0
:1087C000520092006421B3FBF2F3B3FBF1F001FB22
:1087D00010330201A08900044BBFDB001B013233C0
:1087E00032334BBFB3FBF1F3B3FBF1F303F00703F9
:1087F00003F00F0313439BB2238105B030BD00BFCC
:1088000000380140838921B19BB243F40053838136
:10881000704723F400531B041B0CF8E7C1F3080155
:10882000818070478088C0F308007047012310B52D
:10883000C1F342149C4201F01F0103FA01F105D17A
:108840000C3003683AB11943016010BD022C0CBF13
:1088500010301430F5E723EA0101F5E703881942E7
:1088600014BF0120002070470123090A8B40DB431D
:108870009BB20380704700002DE9F3411F4600239F
:1088800004460D46164601931AB9012002B0BDE810
:10889000F08140F6FF7301934FF40031204600F061
:1088A0005DFD002852D10121204600F023FD4FF24A
:1088B000FF71204600F038FD0121204600F002FD46
:1088C00040F6FF73DFF89C8101934146204600F09B
:1088D00039FD002841D039460122204600F016FD1E
:1088E00040F6FF73604F01933946204600F036FD95
:1088F000002838D0012E42D10021204600F0FAFC99
:1089000003F078FD31462046238B00F0E7FC03F0AE
:108910008FFD40F6FF73554E01933146204600F01F
:108920001DFD30B3204600F0FCFC287040F6FF73BC
:108930004F4D01932946204600F010FD0028A4D099
:10894000019B5A1E0192002BF4D104E0019B5A1E98
:108950000192002BA0D1002098E7019B5A1E0192A2
:10896000002BB2D1F7E7019B5A1E0192002BBBD11D
:10897000F1E7019B5A1E0192002BCED1EBE7022EAC
:1089800025D103F037FD4FF40061204600F0CCFC08
:108990000021204600F0AEFC238B03F049FD40F699
:1089A000FF73344E01933146204600F0D7FC40B1AE
:1089B0000121204600F092FC238A2B70238A6B70E1
:1089C000B4E7019B5A1E0192002BECD1C3E740F69D
:1089D000FF77033E238BDFF89C802E44B54201973E
:1089E00028D1244E3146204600F0B8FC70B3002157
:1089F000204600F07FFC204600F093FC40F6FF7319
:108A00001C4E287001933146204600F0A7FC18B395
:108A10000121204600F062FC204600F082FC6870D4
:108A2000204600F07EFCA87080E7019B5A1E019250
:108A3000002B90D04146204600F090FC0028F4D056
:108A4000204600F06EFC05F8010BC7E7019B5A1E9B
:108A50000192002BC6D17EE7019B5A1E0192002B8A
:108A6000D1D178E70100030002000010400000109F
:108A700010000010040000102DE9F3411E460023F1
:108A8000019340F6FF7304460D4617460193002AF2
:108A900000F082804FF40031204600F05FFC002897
:108AA00043D10121204600F00DFC40F6FF73DFF8B2
:108AB000708101934146204600F044FC00283DD0DF
:108AC00031460022204600F021FC40F6FF73554E4F
:108AD00001933146204600F035FC002834D02E4664
:108AE000204616F8011B3D4400F019FC40F6FF77C4
:108AF000DFF83481AE42019731D14B4D29462046F3
:108B000000F02CFC002836D02046012100F0E6FBC6
:108B100040F6FF73454D464C01932946204600F030
:108B20001DFC00282DD1012005E0019B5A1E019259
:108B3000002BAFD1002002B0BDE8F081019B5A1E8E
:108B40000192002BB6D1F5E7019B5A1E0192002B32
:108B5000BFD1EFE7019B5A1E0192002BEAD041469C
:108B6000204600F0FBFB0028F4D0204616F8011B3D
:108B700000F0D5FBBEE7019B5A1E0192002BBDD130
:108B8000D8E7019B5A1E0192002BC6D1D2E7019B68
:108B90005A1E0192002BCDD04FF40031204600F038
:108BA000DDFB0028F3D10121204600F08BFB40F6CD
:108BB000FF731B4D01932946204600F0C3FB10B301
:108BC00000223146204600F0A1FB40F6FF73154D10
:108BD00001932946204600F0B5FBD0B12046012183
:108BE00000F07CFB40F6FF73104D114C01932946B9
:108BF000204600F0B3FB002895D0019B5A1E01923D
:108C0000002BF4D196E7019B5A1E0192002BD2D182
:108C100090E7019B5A1E0192002BDAD18AE700BF30
:108C20000100030082000700040000101000001083
:108C3000005400402DE9F3411E46002304460D4632
:108C4000174601931AB9012002B0BDE8F08140F641
:108C5000FF7301934FF40031204600F07FFB0028A2
:108C600038D10121204600F02DFB40F6FF73DFF8DC
:108C7000D48001934146204600F064FB002843D095
:108C800031460022204600F041FB40F6FF732E4E95
:108C900001933146204600F055FB00283AD02E467D
:108CA000204616F8011B3D4400F039FB40F6FF77E3
:108CB000DFF89880AE42019737D1244D29462046EF
:108CC00000F04CFB0028BED1019B5A1E0192002BE4
:108CD000F4D104E0019B5A1E0192002BBAD1204628
:108CE000012100F0FBFA40F6FF73194D194C019376
:108CF0002946204600F032FB20B1019B5A1E01920A
:108D0000002BF5D100209FE7019B5A1E0192002BFA
:108D1000B0D1E4E7019B5A1E0192002BB9D1DEE7E6
:108D2000019B5A1E0192002BD9D04146204600F0EB
:108D300015FB0028F4D0204616F8011B00F0EFFACE
:108D4000B8E700BF01000300820007000400001024
:108D5000100000100054004000232DE9F3410D469F
:108D60004FF4003104461746019300F0F7FA18B9A2
:108D7000002002B0BDE8F0810FB90120F9E72E46CE
:108D8000204616F8011B3D4400F0C9FA40F6FF7773
:108D9000DFF86C80AE4201971FD1194D294620465D
:108DA00000F0DCFA28B32046012100F097FA40F6E3
:108DB000FF73144D144C01932946204600F0CEFA5F
:108DC0000028DAD0019B5A1E0192002BF4D1CFE784
:108DD000019B5A1E0192002BCAD04146204600F04A
:108DE000BDFA0028F4D0204616F8011B00F097FACF
:108DF000D0E7019B5A1E0192002BCFD1B8E700BFEC
:108E00000400001010000010005400402DE9F34150
:108E10001F46002304460D46164601931AB9012049
:108E200002B0BDE8F0814FF4003100F097FA08B9C4
:108E30000020F5E70121204600F05CFA4FF2FF71B7
:108E4000204600F071FA0121204600F03BFA40F67E
:108E5000FF73DFF89C8101934146204600F072FACF
:108E600000283AD039460122204600F04FFA40F659
:108E7000FF73604F01933946204600F06FFA0028D7
:108E800031D0012E3BD10021204600F033FA03F00F
:108E9000B1FA31462046238B00F020FA03F0C8FADD
:108EA00040F6FF73544E01933146204600F056FAC7
:108EB000F8B1204600F035FA287040F6FF734F4DA8
:108EC00001932946204600F049FA0028A7D0019BCB
:108ED0005A1E0192002BF4D1AAE7019B5A1E01925F
:108EE000002BB9D1A4E7019B5A1E0192002BC2D1DD
:108EF0009EE7019B5A1E0192002BD5D198E7022EC6
:108F000029D14FF40061204600F00EFA03F072FA06
:108F100000212046238B00F0EDF903F089FA40F69A
:108F2000FF73374E01933146204600F017FA60B1C7
:108F300003F060FA0121204600F0D0F9238A2B705B
:108F4000238A6B7003F074FAB7E7019B5A1E0192F3
:108F5000002BE8D16CE740F6FF77033E238BDFF868
:108F6000A0802E44B542019729D1254E3146204696
:108F700000F0F4F978B30021204600F0BBF9204658
:108F800000F0CFF940F6FF731D4E28700193314673
:108F9000204600F0E3F920B30121204600F09EF9BD
:108FA000204600F0BEF96870204600F0BAF9A870BB
:108FB00083E7019B5A1E0192002B3FF439AF4146D3
:108FC000204600F0CBF90028F3D0204600F0A9F9A4
:108FD00005F8010BC6E7019B5A1E0192002BC5D173
:108FE00026E7019B5A1E0192002BD0D120E700BF3B
:108FF00001000300020000104000001010000010EB
:109000000400001038B5204B08219A691F4842F42B
:1090100000129A619A6922F400129A615A6A22F443
:1090200000125A62FEF7D6F8012308211A461748A3
:10903000FEF70AF8092115480122FEF745F8092133
:109040001248FEF7DAF8D8B1012038BD08212846C9
:10905000FEF7C0F8FDF7FEFD08212846FEF7BFF831
:10906000FDF7F8FD013CF1D109210848FEF7C5F8EC
:1090700020B940F27D110648FDF7A0FA2046E4E74A
:109080003324024DEEE700BF0038024000040240E6
:109090007DDF01082DE9FF41444B054698420E460D
:1090A00017467CD103F5F2335A6A082142F40012C4
:1090B0005A629A693E4842F400129A619A6922F40F
:1090C00000129A61FEF786F8012308211A463848F3
:1090D000FDF7BAFF092136480122FDF7F5FF092106
:1090E0003348FEF78AF8002855D0012308211A4694
:1090F0002F48FDF7A9FF042208212D48FEF724F888
:10910000012309211A462A48FDF79EFF042209215E
:109110002748FEF719F8274B9A6942F400129A6122
:109120009A6922F400129A61684600F0B1F8224B65
:10913000694601934FF48063ADF80A304FF48043E1
:109140002846ADF80C30ADF80870009600F038F8FD
:109150002846012100F0AAF8012019E00821404624
:10916000FEF738F8FDF776FD08214046FEF737F8A0
:10917000FDF770FD013CF1D109210D48FEF73DF8E6
:109180000028B2D10D4840F2A511FDF717FA20468C
:1091900004B0BDE8F0813324DFF81480EAE74FF42F
:1091A000DA710648FDF70AFABEE700BF0054004036
:1091B00000040240003802400000FFBF7DDF0108CC
:1091C0007FB50446868868460D46FFF707FA029A7F
:1091D0002D4926F03F06B2FBF1F13604360C88B279
:1091E0000643A6802388294E23F001031B041B0C91
:1091F00023802B68B34223D85B00B2FBF3F39BB20E
:10920000042B38BF0423013080B22084A383238839
:10921000AA889BB243F0010323802388698923F441
:10922000816323F002031B040A431B0C13439BB20C
:109230002A892380AB8913439BB2238104B070BD7C
:109240004BF6FF70EE8886421BBF1920434303EBA9
:109250004303B2FBF3F30BBFB2FBF3F39BB29BB23E
:1092600043F48043C3F30B020AB943F001034FF404
:10927000967251434FF47A72B1FBF2F1013189B227
:1092800043F400432184C1E740420F00A08601005F
:1092900041F28832044BC0E90023002383604FF47D
:1092A00080438381704700BF0000FFBF038821B166
:1092B0009BB243F001030380704723F001031B04BA
:1092C0001B0CF8E7038821B19BB243F48073038041
:1092D000704723F480731B041B0CF8E7038821B14B
:1092E0009BB243F400730380704723F400731B04A4
:1092F0001B0CF8E7038821B19BB243F48063038021
:10930000704723F480631B041B0CF8E722B141F083
:10931000010189B20182704701F0FE01F9E7018283
:109320007047008AC0B270470388B1F5006F15BF5F
:1093300023F400639BB21B0443F4006318BF1B0CAF
:1093400003807047838A008B9BB243EA00430B4043
:1093500023F07F435B1A584258417047002382B084
:10936000009301930B0F01900093009B21F07F412C
:1093700053B1019B14330193019B1B680B4214BF33
:109380000120002002B07047019B090C1833F2E75E
:10939000F8B50E46054680B14F1C384600F05CFF1C
:1093A000044640B13A4600210EF094FE324629466A
:1093B00020460EF067FE2046F8BD0446FBE738B5B0
:1093C0000D46044628B10FF0DFFE234620448342B9
:1093D00001D1002038BD13F8012BAA42F7D101209A
:1093E000F8E773B505460E4600240EF03DFC224614
:1093F000046001A928460FF08BFF05460EF034FCEF
:109400000368222B0BD0019B1B7843B9A542ADBF4B
:109410002846204601232346336002B070BD012355
:109420002046F9E72DE9F04F05464FF0010B0026E5
:1094300087B0CDE9021206F10903122B8CBF03207D
:10944000022000F009FF0746F0B1324637490FF01D
:10945000EDFD029B53F826A0F5B90024384600F034
:10946000E5FEBBF1000F02D1284600F0DFFE8CB113
:10947000039B0136B3424FF0000B03D1204607B0E7
:10948000BDE8F08F2546D6E7BBF1000F02D1284694
:1094900000F0CCFE0024F1E7254B4FF00009BAF1B3
:1094A000000F08BF9A4650460FF06EFE00903846F7
:1094B0000FF06AFE0190284651460FF094FEB8B9AD
:1094C00028460FF061FEDDE9002301309B1A09FBFD
:1094D000030000F0C1FE04460028BED00346A846A3
:1094E000B9F1010909D2414618460FF045FEB5E72A
:1094F000009B09F101091844DEE7514640460593F7
:109500000FF071FE059BA0EB08024146184604923D
:109510000FF056FE049A394610440FF02DFE0099C4
:10952000049A019B0A44C3189044D9E793AD0108FB
:109530007DDF010830B580B10346021F00F1180439
:1095400052F8045F8D4208D0A242F9D11C301A466D
:1095500014680433013401D1116030BD8342F6D167
:10956000FBE700000649431E13F8010F00B97047DE
:109570000A5C02F00302022A08BF20381870F3E7E1
:1095800022E6010870B50E46044670B10025AE42D1
:1095900004D12046BDE8704000F048BE54F82500D4
:1095A00008B100F043FE0135F1E770BD2DE9F74F3A
:1095B0008A4604460092002839D00027E35D8BBB21
:1095C000A04622461E46384804EB070B5A4537D1C1
:1095D00003B10136002E5FD00137384600F03CFE63
:1095E000044628B33A4600210EF074FDB00000F0A6
:1095F00033FE0546002851D04FF000090021C34535
:109600002CD131B12046FFF7C3FE002846D045F8E3
:109610002900204600F00AFE009B1E60284603B089
:10962000BDE8F08F0137B7F5807FC7D1002426460B
:10963000002531462046FFF7A5FF009B1D60EDE7A2
:1096400012F8011B514504D1002BBFD00023013675
:10965000BCE7095C090758BF0133B7E718F8013BBD
:10966000534512D10029CAD02046FFF791FEA8B178
:1096700009F1010345F829003A46002120460193EB
:109680000EF028FD019B9946B8E7074A985C02074F
:109690005CBF63540131B2E73546BFE7204600F0B6
:1096A000C5FD2C46C4E700BF22E601082DE9F743BB
:1096B000002507460820884691461E46009500F082
:1096C000CBFD0446002865D0C0E9005538460FF0B0
:1096D0005BFD01280FD13B782A2B0CD109F1FF3318
:1096E000C4F80080636022684A4502D263684B4533
:1096F00040D3294B0DE02D213846FFF760FE05468B
:10970000B8B9019001A93846FFF76BFE019B63B120
:10971000224B336028460099FFF734FF002C35D0E8
:10972000204600F083FD002430E01D46C4E900001F
:10973000D9E76A462D213846FFF738FF009B0546DA
:10974000013B012B01D9164BE3E70023006801A977
:109750000193FFF746FE2060019B0BB1114BD8E748
:10976000686801A9FFF73DFE6060019B002BBAD03D
:109770000D4BCEE7424501D3434501D20B4BC8E721
:1097800028460099FFF7FEFE00233360204603B011
:10979000BDE8F0830546BDE764C10108DEC00108ED
:1097A000FDC0010826C1010845C1010884C10108A6
:1097B00008B520B34A1C22D0062920D8DFE801F0E2
:1097C000040D101316191C00002303600EF062FD37
:1097D0000840431C5842584108BD00234360F5E748
:1097E00000238360F2E700238361EFE70123C36076
:1097F000ECE700230361E9E700234361E6E701208A
:10980000EAE770B5054688B181B10E1F01F1180471
:1098100056F8041F4B1C03D1A642F9D1002070BD9D
:109820002846FFF7C5FF0028F6D0F8E70120F6E745
:1098300008B538B34A1C25D0062923D8DFE801F043
:10984000040E1216161A1E000368013303600EF090
:1098500021FD0840431C5842584108BD436801336C
:109860004360F4E7836801338360F0E7C368013342
:10987000C360ECE7036901330361E8E7436901333F
:109880004361E4E70120E8E700290B46B8BFCB1DA0
:109890004A4202F0070201F0070158BF514201227B
:1098A000C3F3C703C9B202FA01F1C25C1143C15448
:1098B000704700290B46B8BFCB1D4A4202F0070291
:1098C00001F0070158BF51420122C3F3C703C9B2D7
:1098D0008A40C15C21EA0201C15470470B4600294D
:1098E000B8BFCB1DC3F3C703C05C4B4203F00703F3
:1098F00001F0070158BF5942C9B2084100F0010008
:1099000070472DE9F843089E884617469946054654
:1099100010B11446A0450BD848460999FFF788FFB7
:1099200068B1012200240B9B1A602046BDE8F88331
:1099300021462846FFF7D2FFE8B90134EAE731466D
:109940004846FFF735FF04460028EAD1B5B1214665
:109950002846FFF7C3FF70B90134A045F7D104468C
:10996000B9F1000FDDD0711E042909D8DFE801F03C
:109970001A1D20232600A742F2D1D6E72C46EFE796
:10998000C9F8004048460EF085FCB1F1FF3F08BF22
:10999000B0F1FF3FC5D048460A99FFF732FF0028D3
:1099A000C3D0BEE7C9F80440ECE7C9F80840E9E7CE
:1099B000C9F81840E6E7C9F80C40E3E7C9F81040D9
:1099C000E0E72DE9F04F4FF000098BB006461C2070
:1099D0000C469046CDF8249000F03EFC0546002849
:1099E00000F0EE801C2000F037FC0746002800F055
:1099F000E78005F11B031B1A362B40F2A1801C22C5
:109A0000FF2128460EF066FB1C22FF2138460EF08F
:109A100061FB00230121D4F800A00DF12409CDE958
:109A2000003152463C2123463046CDE90279FFF70A
:109A300068FF0999002940F09680824502D12846A6
:109A4000FFF778FD02234FF0010AD4F804B0CDE906
:109A500000A35A4623463C21CDE9025906F10800ED
:109A6000FFF74FFF099B002B7DD1834573D15146F2
:109A70002846FFF75FFD03234FF0020AD4F808B031
:109A8000CDE900A35A4623461821CDE9025906F133
:109A90001000FFF736FF099B002B64D183456DD181
:109AA00051462846FFF746FDE368D4F818B0049302
:109AB00006F11403069306F11303079340F26F13A4
:109AC000DDF810A0059351460698FFF707FF20B177
:109AD00059460798FFF702FF68B9059B013B0593BC
:109AE00009D004212046FFF7A3FE00284FD0012310
:109AF0004FF0000A0993099BABBB049B53454FD120
:109B000004212846FFF716FD05230622D4F810A0ED
:109B1000CDE900320C2123465246CDE9025906F127
:109B20001800FFF7EEFE099BEBB982451BD0636975
:109B3000A3EB0803042B3CD94FF0FF33099312E049
:109B40004B464FF0FF3245F8232047F823200133DE
:109B5000072BF8D15DE7424621463046FFF731FF3B
:109B60000990002887D0284600F060FB17B13846DE
:109B700000F05CFB09980BB0BDE8F08F424621462F
:109B80003046FFF71EFF099000288DD0EBE72946ED
:109B90002046D4F80CA0D4F818B0FFF732FE92E7B4
:109BA000424621463046FFF70CFF09900028ABD013
:109BB000D9E7424621463046FFF703FF0990D2E736
:109BC0004FF0FF330993002DD4D00027CBE70000DE
:109BD0002DE9F04F002487B0894692462C2103AA34
:109BE0009846109E0394FFF7E1FC074688B93E4B68
:109BF000336038460399FFF7C5FC07B0BDE8F08F26
:109C0000D0F800B06B685B451CD2284600F00EFB14
:109C10000134039BA342ECD957F824502F21284646
:109C2000FFF7CDFBA8B93346284642465146FFF719
:109C30003DFD33680546002BE2D00028D9D000F066
:109C4000F5FAD6E759464846FFF71EFE0BF1010B21
:109C5000D8E700232F21284604AA0493FFF7A6FC87
:109C6000049905464B1E012B04D9204B3360FFF7A6
:109C700089FCBEE74246334651460068FFF716FDB1
:109C8000326883462AB108B100F0D0FA2846049918
:109C9000EDE72D212868FFF792FB18B908F1FF3294
:109CA000CBF80420002305A968680593FFF799FB0A
:109CB0000599024619B10E4A58463260E4E7DBF8CE
:109CC0000010DBF80400884205D228460499FFF70B
:109CD00059FC58469AE74846CDE90012FFF7D4FDF3
:109CE000DDE900121144ECE7A9C10108BBC101087C
:109CF000E0C101082DE9FF41002305460E46144648
:109D0000039302B902AC236045B9574B2360284640
:109D10000399FFF737FC04B0BDE8F0812846202105
:109D200003AAFFF743FC039B0546062B01D04F4BCC
:109D3000ECE71A22002130460EF0CCF90094002204
:109D40003C2331462868FFF743FF2268002ADED112
:109D500000943C23686806F10801FFF739FF226888
:109D6000002AD4D100941823A86806F11001FFF747
:109D70002FFF2368002BCAD1686908B1FFF7F2FBF7
:109D800007223B496869FFF74DFB07460FF0FCF9D6
:109D9000012806F1130804D13B783F2B04BF2A2386
:109DA0003B7000220823414638460094FFF710FF1D
:109DB000384600F03BFA2268002AA8D10721404625
:109DC000FFF78CFD30B111464046FFF75DFD0721DE
:109DD000FFF76FFDEF6806F1140838460FF0D4F96D
:109DE000012804D13B783F2B04BF2A233B7020235A
:109DF0000022414638460094FFF7EAFE0021404623
:109E0000FFF757FD2368002B81D12F69002F3FF406
:109E10007EAF3846FFF7A6FB00287FF478AF3846C0
:109E20000D221449FFF7FEFA074600283FF46FAFF2
:109E300018360D23012231460094FFF7C9FE38463B
:109E400000F0F4F9012421463046FFF747FD30B118
:109E5000611E3046FFF718FD2146FFF72AFD013449
:109E60000D2CF0D153E700BFFFC1010817C2010854
:109E70006C020020880200202DE9F0418CB00546DC
:109E8000CDE9002328B94FF0FF3001460CB0BDE802
:109E9000F0812422002103A80EF01CF9684603A9D2
:109EA0000EF00EF804460028EDD00EF0F3F9B1F1F3
:109EB000FF3F08BFB0F1FF3F80460F46E3D0214689
:109EC00028466269FFF77DFD06460028DBD1204663
:109ED0000EF0E0F9B1F1FF3F08BFB0F1FF3FD2D083
:109EE0008F4208BF804503D020460EF0D3F9CDE75E
:109EF00031462046FFF79CFC0028C4D12146284665
:109F00006269FFF75EFD0028EED0BCE770B58AB04D
:109F1000DDE90E4501953C2594FBF5F605FB16445D
:109F20000294182493FBF4F505FB1433CDE90330B8
:109F30000C23013991FBF3F003FB10110023CDE951
:109F400007339DF84030A2F26C7201A80591069289
:109F500009930EF09FF90AB070BDF7B50446684644
:109F6000CDE900230DF08EFF0269037A551C42698A
:109F700090F804C0077B067E02F26C71C26900682B
:109F8000A370003B18BF012320702046013284F8E3
:109F900001C0E7702571A4F80510E67122726372A2
:109FA00003B0F0BD1FB5437A029303780193437861
:109FB00000938378B0F805200179C078FFF7A6FFF9
:109FC00005B05DF804FB904271EB0303B4BF0120C0
:109FD00000207047032210B5104986B00B7801337A
:109FE000B3FBF2F202EB42029B1A0D4A0B7052F8DD
:109FF000234003781A21049343780A4A0393837811
:10A000000293C378019303790093B0F8053020469A
:10A010000EF0D8FF204606B010BD00BF0F1F002075
:10A02000E0C20108A5C20108B1F1004F08BF002835
:10A030001FB502460B4608D001A8FFF78EFF01A806
:10A04000FFF7C8FF05B05DF804FB0148FAE700BF61
:10A05000C3C201082DE9FF470322044629480D1E0B
:10A06000037803F10103B3FBF2F202EB4202A3EB2C
:10A070000203254A037052F823903DDA4FF0010A9B
:10A08000644265EB45050023204A204629460DF031
:10A0900003FC00230646294620461C4A0DF0FCFB23
:10A0A000104619464FF4616200230DF0F5FB4FF4A2
:10A0B000616207460023204629460DF0EDFB10465D
:10A0C00019463C2200230DF0E7FB3C22804600238A
:10A0D000204629460DF0E0FB3346CDE9018200978A
:10A0E000BAF1000F0BD00A4A1A2148460EF06AFF57
:10A0F000484604B0BDE8F0874FF0000AC3E7054AC0
:10A10000F2E700BF0F1F0020E0C2010880510100EC
:10A11000CBC20108CCC201080FB404B070470000E4
:10A120000FB437B51B4C256855B9032229460120C9
:10A1300002F080FB2B462A462946206002F09EFB57
:10A14000154D2B68013B03331ED86421206802F0B3
:10A1500083FD8022002111480DF0BCFF07AB802158
:10A16000069A0E4801930FF047FB7F2803DD0C4948
:10A170000C480FF001F82B68084898470023206826
:10A180001A46194602F07AFB03B0BDE8304004B02D
:10A19000704700BF981F0020101F0020181F0020CC
:10A1A000E4AF0108931F00200FB410B50D4CA2B00E
:10A1B0002368013B033310D825AB8021249A02A8E1
:10A1C00001930FF019FB7F2804DD07490DF183008F
:10A1D0000EF0D2FF236802A8984722B0BDE81040D5
:10A1E00004B07047141F0020E4AF010870B50446A6
:10A1F000054E4518AC4200D170BD304614F8011B25
:10A20000FFF78EFFF6E700BFECC2010838B50C4639
:10A210001546FFF785FF20462946FFF7E7FFBDE813
:10A2200038400148FFF77CBF7CDF010810B50446C9
:10A2300070B102F02FFA204602F01AFA02F0DAF8B2
:10A24000BDE81040034A93880133938002F0F0B8D0
:10A2500010BD00BF9C1F002070B5234D04462B6825
:10A260008AB001332B6000283BD0632B1F4E0BDDDF
:10A2700003F0B2FD0523002201A903F0DFFC03F087
:10A28000DBF9002330602B6003F0D6F9336803F567
:10A290007A73984204D903F0CFF9002330602B6021
:10A2A000134A144D13781BB92B606B600123137094
:10A2B00002F0F0F9204602F0D9F9064668B12246CC
:10A2C00000210DF007FF02F095F82B8801332B8059
:10A2D00002F0AEF830460AB070BD6B8801336B8077
:10A2E000F8E70646F6E700BFA81F0020AC1F0020D5
:10A2F000A41F00209C1F0020006800BA704700883F
:10A3000040BA80B2704700687047837842781B0477
:10A31000007843EA02231843704700887047FFF72C
:10A32000F2BF0370130E4370130C8370130AC370D3
:10A330000271052070470B0E03700B0C43700B0A63
:10A340008370C170042070470B0A037041700220B3
:10A3500070470B0A017043700B0C090E8370C170BB
:10A3600004207047A0F14103052B02D83738C0B252
:10A370007047A0F16103052B01D85738F7E7303853
:10A38000C0B20A2828BFFF207047002210B5441E23
:10A3900021B114F8010F08B1002A01DA104610BDEE
:10A3A000FFF7E0FF01390F28C9B202D840EA0212D4
:10A3B000EEE74FF0FF32F1E738B505460C460EF0F8
:10A3C00051FD611B013190FBF1F303FB11002844A7
:10A3D00038BD000010B504460EF016FD014B1C60A0
:10A3E00010BD00BFBC020020024B1868013018608D
:10A3F0000EF00ABDBC0200200078013070470FB497
:10A4000004B070472DE9FF470D460021DFF8A4A0F6
:10A4100003AF06469146DAF800003A4698460391A3
:10A4200002F05AFD0128039B36D14BB14FF0E023D7
:10A430004FF08052C3F8042DBFF34F8FBFF36F8FDF
:10A44000B5F5C87F88BF4FF4C87531462A461A480B
:10A450000DF018FE194C184B3946DAF80000A580AB
:10A460002360A4F8069084F8088002F019FB039B8F
:10A470004BB14FF0E0234FF08052C3F8042DBFF3EF
:10A480004F8FBFF36F8F0E480097002301220421E6
:10A49000006803F06FFE039B4BB14FF0E0234FF0D9
:10A4A0008052C3F8042DBFF34F8FBFF36F8F04B0FA
:10A4B000BDE8F087B4210020182000200C200020E7
:10A4C000C02100200348002301220221006803F07C
:10A4D000E1BD00BFC02100201FB5002303AA0B4827
:10A4E0000092102101220068039303F043FE039BB6
:10A4F0004BB14FF0E0234FF08052C3F8042DBFF36F
:10A500004F8FBFF36F8F05B05DF804FBC0210020B3
:10A510001FB5002303AA0B48009280210122006886
:10A52000039303F027FE039B4BB14FF0E0234FF062
:10A530008052C3F8042DBFF34F8FBFF36F8F05B068
:10A540005DF804FBC02100201FB50346104A1068C7
:10A55000B3B1002303AA009208210122039303F060
:10A5600009FE039B4BB14FF0E0234FF08052C3F83C
:10A57000042DBFF34F8FBFF36F8F05B05DF804FB61
:10A580000122082105B05DF804EB03F083BD00BF94
:10A59000C02100201FB503F055F80D4B03AA186029
:10A5A0000092012200230B4811460068039303F038
:10A5B000E1FD039B4BB14FF0E0234FF08052C3F815
:10A5C000042DBFF34F8FBFF36F8F05B05DF804FB11
:10A5D000BC210020C02100201FB500230C4A4021CF
:10A5E000107003AA0B48009200680122039303F045
:10A5F000C1FD039B4BB14FF0E0234FF08052C3F8F5
:10A60000042DBFF34F8FBFF36F8F05B05DF804FBD0
:10A61000FC1F0020C021002000487047F41F0020CC
:10A620001248002303224FF4807110B5006803F034
:10A6300031FD4FF0E0234FF08052C3F8042DBFF3FB
:10A640004F8FBFF36F8F0A4C206802F091FC40B12E
:10A65000BDE81040002307481A461946006802F07A
:10A660000DB9012003F040F9EEE700BFC021002042
:10A67000B8210020B0210020F8B5124B014618681F
:10A6800002F0EAFA0446D0B14FF0E0254FF08056D0
:10A690000D4F002303224FF40071386803F0FAFCD9
:10A6A000C5F8046DBFF34F8FBFF36F8F386802F0AA
:10A6B0002FFFC5F8046DBFF34F8FBFF36F8F204698
:10A6C000F8BD00BFB0210020C0210020014B186060
:10A6D000704700BFA821002070B5044678B1037808
:10A6E000032B0CD1436853B10025054E1868F2695D
:10A6F00090476068F369056098476560257070BD94
:10A70000D01F002010B50E480E4C00230522214614
:10A71000006802F0B3F8012807D1002363600A4BF8
:10A720001B6863B1BDE810401847084B2178084802
:10A730005B6998472046BDE81040FFF7CDBF10BDCC
:10A74000AC21002000200020A8210020D01F0020E4
:10A75000F2C201087FB50024094E0022306801A929
:10A7600002F0E8F9651C30B9064B07485B69E1B2B5
:10A77000984704B070BD01A8FFF7AEFF2C46ECE788
:10A78000AC210020D01F002019C30108014B18681C
:10A79000704700BFAC21002010B50446064B010AEB
:10A7A000A3F84A00202000F091FBE1B22120BDE88F
:10A7B000104000F08BBB00BFEC24002008B5FFF771
:10A7C000EBFF0122014B83F8522008BDEC2400204E
:10A7D000002238B50B4B05461D200C4683F84C2053
:10A7E00083F84E1000F0CCFB20F0060343EA44014E
:10A7F0001D20C9B200F06AFB2946BDE8384023207D
:10A8000000F064BBEC24002013B5164C0120A368B3
:10A810009847002341F6FE720093009B934218DD97
:10A82000A36802209847002341F6FE720193019B22
:10A83000934212DD0C4BB5211C6C4020A047A02197
:10A840004120A04700210120234602B0BDE810406E
:10A850001847009B01330093DFE7019B013301930D
:10A86000E5E700BFD01F00200CC60108094B07B563
:10A870001B6CC2213B209847002341F6FE720193D6
:10A88000019B934202DD03B05DF804FB019B0133A1
:10A890000193F5E70CC601082DE987488D4B8E48DA
:10A8A0008E4F03608E4B8F4C83608F4B8F4E436077
:10A8B0008F4BDFF84092C3608F4BDFF8408203611B
:10A8C0008F4BDFF840A283618F4BC3613B68984791
:10A8D00063698E489847002330681A46194601F08C
:10A8E000CDFF99F8040068B94FF0FF33194601AA6B
:10A8F00003F086FB68B9656903F05EFA0146844897
:10A90000A847EEE741F288334FF0FF31002001AA5B
:10A91000EEE7019BDA0516D500F098FA002000F06A
:10A92000E9FDFB6A9847FFF715FF63697948984787
:10A930000023D8F800001A46194601F09FFF0020B6
:10A9400003F050F8CDE79B0510D500F07FFAFFF734
:10A950008DFFFB6A9847FFF7FDFE63696E489847D5
:10A960006421D8F8000002F077F9BAE7D8F80000BF
:10A9700002F0FEFA012803D1636968489847B0E7FE
:10A98000DAF8003023B94FF4B5716548FBF716FECD
:10A99000019B1D0604D50722624B1A70FFF7B2FE19
:10A9A000019B580750D50021306802F055F9012865
:10A9B0004AD10C20A3699847054688B90C216369E0
:10A9C000594898472B462A462946306801F056FFD9
:10A9D000002886D140F27F115148FBF7EFFD80E758
:10A9E000524BA269988880B29047504B834698B9E1
:10A9F00099884F4889B2636998472846E369984720
:10AA00005B465A465946306801F038FF00287FF40B
:10AA100068AF40F28711DFE71A1D03CAC5F800B01E
:10AA20006860A96019689A88584692B20DF02AFBAE
:10AA300003223C4B1A705D60FFF764FE0023306810
:10AA40001A46194601F01AFF019BD90709D50122C0
:10AA5000344B1A7000225A60364A12689A60FFF727
:10AA600051FE019BDB0606D505222E4B1A700022F3
:10AA70005A60FFF747FE019B1D0706D50422294BAC
:10AA80001A7000225A60FFF73DFE019B980706D519
:10AA90000222244B1A7000225A60FFF733FE019BFA
:10AAA000990606D506221F4B1A70234A5A60FFF7F3
:10AAB00029FE019B5B067FF514AF204B1B78002B12
:10AAC00014BF08220922174B1A7000225A60FFF7A0
:10AAD00019FE06E795A50008B01F00200CC6010866
:10AAE00005A40008D01F0020C5A40008B421002040
:10AAF00049A50008F41F0020D9A40008B8210020AF
:10AB0000D9A50008AC21002011A500084AC30108FE
:10AB100060C301087EC30108A6C30108BDC30108C4
:10AB20007DDF010800200020D3C301080C20002095
:10AB300009C40108BC210020FD1F0020FC1F0020CB
:10AB4000044B10B55B6998470446FFF75DFE20464D
:10AB500010BD00BF0CC60108F0B5724C0546264674
:10AB60000F460FCD0FC695E80F0086E80F0097E857
:10AB7000030063696C4E013B033388BF6B4B254672
:10AB800088BF6361636886E80300013B033385B0D7
:10AB900007D96748636998474FF430716548FBF7F8
:10ABA0000DFD2368013B033307D963486369984768
:10ABB0004FF431715F48FBF701FDA368013B03339C
:10ABC00007D95E48636998474FF432715948FBF7DB
:10ABD000F5FCE368013B033307D95948636998479B
:10ABE0004FF433715348FBF7E9FC2369013B03330E
:10ABF00007D95448636998474FF434714D48FBF7BF
:10AC0000DDFCE369013B033304D94FF43571494856
:10AC1000FBF7D4FCA369013B033304D94FF436712D
:10AC20004448FBF7CBFC484B0FCB8DE80F0095E871
:10AC30000F0000F0E1F823689847FFF7E5FD434B6C
:10AC400042205B6C98472228014663693FD1404807
:10AC5000984703220021012001F0ECFD3D4B1860D4
:10AC6000012001F0B1FE3C4B186020B94FF43D715A
:10AC70003048FBF7A3FC03220021012001F0DAFD9C
:10AC8000364D286020B94FF43E712A48FBF796FCF8
:10AC9000002328681A46194601F0F0FD20B940F259
:10ACA000F9212448FBF78AFC4FF0FF31286801F0B6
:10ACB000D3FF00220C21032001F0BCFD284B1860BB
:10ACC00078B963692748984740F2FF2103E0264896
:10ACD000984740F2EA211748FBF770FC002005B0C6
:10ACE000F0BD224B224A1A6033680BB9042333604B
:10ACF000204B1D680DB10120F1E701933368FA2262
:10AD000000931D4901231D4802F05EFA0128F2D08C
:10AD100063691B489847074840F21131FBF74EFC26
:10AD20002846DCE7D01F0020F41F0020FFA3000806
:10AD300041C401087DDF010882C40108B9C40108CB
:10AD4000F1C401082AC50108E01F00200CC6010853
:10AD500066C50108B4210020B0210020B8210020E0
:10AD6000AC21002098C501087DC50108F01F002016
:10AD7000F9A30008C0210020CCC5010899A800084B
:10AD8000D4C5010870B5084E044633680D4623B992
:10AD900040F221310548FBF711FC29462046336873
:10ADA000BDE87040184700BFF01F00207DDF01089C
:10ADB00000F03CB80120704708B5FFF72DFC43793F
:10ADC000002B0CBF8020002008BD0000094B002292
:10ADD000194610B51C68844202D89C68844205D884
:10ADE0000132152A03F10803F4D1FEE701EBC20298
:10ADF000107910BDA0C6010884B030B503AC84E85A
:10AE00000F00064C03AD0FCD0FC495E80F0084E88A
:10AE10000F00BDE8304004B0704700BF502500204F
:10AE2000014B1878704700BFEC240020C82307B5F9
:10AE30000093002304481A460321006803F0C8FA6F
:10AE400003B05DF804FB00BFC821002013B5104C0F
:10AE50000120A368984700230093009BB3F5CC7FA3
:10AE60000FDDA36800209847002342F6FE7201938D
:10AE7000019B934208DD0220A36802B0BDE81040A8
:10AE80001847009B0133E7E7019B01330193EFE78C
:10AE9000502500202DE9F04107460B4E0020F368B5
:10AEA0000C4615469847336947F08000984725447B
:10AEB000AC4204D1F3680120BDE8F0411847336982
:10AEC00014F8010B9847F3E75025002007B501223D
:10AED0008DF807100DF10701FFF7DCFF03B05DF8F7
:10AEE00004FB000000000000134A10B55060134A34
:10AEF000904219D00BF032FE0DA3D3E900230BF0E2
:10AF0000D1FF0CF03FF90446C4F307410620FFF7D8
:10AF1000DDFFC4F307210720FFF7D8FFE1B20820C7
:10AF2000BDE81040FFF7D2BF054CEDE7AFF300805E
:10AF30000000000080844E40EC240020F01FCB3342
:10AF4000CD3CD9002DE9F04107460C4E0020F368B6
:10AF50000C4615469847336907F07F00984725440B
:10AF6000AC4204D1F3680120BDE8F041184700204D
:10AF70003369984704F8010BF2E700BF5025002021
:10AF800007B501220DF10701FFF7DCFF9DF807006F
:10AF900003B05DF804FB000001282DE9F047884666
:10AFA00004D0022854D00020BDE8F087704D27203F
:10AFB000AC8BFFF7E5FFA4B220F0F8000134204489
:10AFC0000BF0CCFDAB7F0022002B3CD1694B0BF08A
:10AFD00089FC064630200F46FFF7D2FF30F0F90318
:10AFE0000CBF0023634B0022304639460BF07AFC3D
:10AFF000064640460F460BF0C1FD02460B46304662
:10B0000039460BF06FFC95F820300022EBB9002395
:10B010000BF068FC0022584B0BF01AFEAE69044698
:10B0200030460D460BF09AFD02460B462046294657
:10B030000BF038FF0022514B0BF00AFE0BF000FC26
:10B040000CF0A0F8B0E70023C1E74FF08043DFE742
:10B05000DFF81CA1DAF84020022A00F28280484B77
:10B0600003EBC203D3E900450120DAF844309840ED
:10B070000BF084FD02460B46204629460BF012FFDA
:10B0800002460B4600203B490BF00CFF04460D46E0
:10B09000BAF84A0080B20BF071FD0022394B0BF078
:10B0A00021FC22462B460BF0D3FDDAF844300F4644
:10B0B0009AF84E109AF84C200646002A14BF142025
:10B0C00000209B00C3F11C0303EB011303EBC80337
:10B0D000181A0BF043FD8046DAF844009AF848301D
:10B0E0008946002B14BF02230023C3EB80000BF022
:10B0F00035FD02460B46404649460BF0D3FE0BF0A9
:10B10000A7FA804689469AF8490004300BF036FDCC
:10B1100042464B460BF09CFD0022002380468946A8
:10B120000CF026F818B94FF000084FF00009002283
:10B1300040464946104B0BF0D5FB22462B460BF000
:10B1400087FD32463B460BF0CDFB00220B4B0BF04C
:10B150007FFD05A3D3E900230BF0C4FB0BF0F4FA49
:10B160006EE7002400257FE72B8716D9CEF7EF3F47
:10B17000EC2400200000F03F0000204000408F4001
:10B1800088C6010800001140012808B504D0022833
:10B190000AD04FF0FF3008BD1120FFF7F1FEC0F3D9
:10B1A0004700404200B2F6E71B20FFF7E9FE8B386C
:10B1B000F8E700000B4B10B55B68044660B902204D
:10B1C00098470120FFF7DCFE00F0F8012143012041
:10B1D000BDE81040FFF77ABE03280CBF0120002015
:10B1E000EEE700BF5025002013B5C82400230B480C
:10B1F00000941A460321006803F0EAF80023084887
:10B2000000941A460321006803F0E2F80020FFF7DB
:10B21000D1FF0022034B1A7002B010BDC8210020DC
:10B220004C250020EC24002013B5C82400230B4833
:10B2300000941A460321006803F0CAF80023084866
:10B2400000941A460321006803F0C2F80120FFF7BA
:10B25000B1FF0022034B1A7002B010BDC8210020BC
:10B260004C250020EC24002073B5594C0646637829
:10B27000012BDAB22FD0022A5DD000254FF4C8721C
:10B28000002154480CF026FF01232370524B18680C
:10B290004FF0FF33002E00F08D804FF47A7101FBE8
:10B2A00006F20093B2FBF1F20023042103F090F8C0
:10B2B0006378012B40F083800520FFF77BFF0D2092
:10B2C000FFF75EFE40F020010D20C9B202B0BDE8DC
:10B2D0007040FFF7FBBD402094F82250FFF750FE6E
:10B2E0000C214020FFF7F2FD4120FFF749FE60F0FE
:10B2F0000E01C9B24120FFF7E9FD3520FFF740FEFE
:10B3000000F03F00112184F83A003F20FFF7DEFDF6
:10B3100000230D2084F82C3084F82D302387E38619
:10B32000FFF72EFE00F04001EDB241F02E010D209E
:10B33000FFF7CCFDA2E794F8513033201BB3FFF7A1
:10B340001FFE40F04101C9B23320FFF7BFFD1921B4
:10B350003B20FFF7BBFD94F8525094F84F30EDB20C
:10B36000E3B11D211120FFF7B1FD4020FFF708FEDA
:10B3700000F033014020FFF7A9FD00210F20FFF767
:10B38000A5FD0021D3E7FFF7FBFD00F0BE0141F072
:10B3900001013320FFF79AFD1D21D9E70F2111206C
:10B3A000FFF794FD4020FFF7EBFD00F03C0141F07A
:10B3B0000101DFE7009332463346032176E72DB1E2
:10B3C000052002B0BDE87040FFF7F4BE0620F8E7A4
:10B3D000EC240020CC210020C821002037B54FF4F8
:10B3E0007A72642350432B4DB0FBF2F20093042198
:10B3F0000023286802F0ECFF0022274B274C1A702C
:10B400006378012BDAB214D0022A26D002232370EB
:10B410002C6802F011F90523024600930121002354
:10B42000204602F0D5FF032003B0BDE83040FFF70F
:10B43000C1BE14214020FFF749FDB0214120FFF794
:10B4400045FD94213520FFF741FD3520FFF798FD9C
:10B4500000F03F0084F83A00D8E794F84F3073B119
:10B46000F5211120FFF732FD4020FFF789FD00F0A4
:10B470003301402041F04001FFF728FDC6E7F721E6
:10B480001120FFF723FD4020FFF77AFD00F03F0178
:10B49000EFE700BF4C25002070250020EC240020A1
:10B4A00010B5124C6378012BDAB204D0022A09D00D
:10B4B00040F21E4101E040F20741BDE810400C4857
:10B4C000FBF77CB8FA211120FFF700FD4020FFF7C1
:10B4D00057FD00F0FC014020FFF7F8FC0323072094
:10B4E0002370BDE81040FFF765BE00BFEC240020CC
:10B4F0007DDF010808B51A4B5A7882422ED0587069
:10B500005B780020022B13D0FFF754FE0120FFF7D9
:10B5100037FD00F07F010120FFF7D8FC002140201B
:10B52000FFF7D4FC30214120BDE80840FFF7CEBC36
:10B53000FFF740FE0120FFF723FD60F07F01C9B255
:10B540000120FFF7C3FC00214020FFF7BFFC0021D2
:10B550004120FFF7BBFC43213120E5E708BD00BFD8
:10B56000EC2400201D4B13B5186000231C4C1A4618
:10B570004FF47A711B48009402F008FF1A4B1860D0
:10B5800020B94FF486711948FBF718F800234FF4DF
:10B590007A711A461648009402F0F8FE154B1860AE
:10B5A00020B94FF487711148FBF708F8FFF74EFCFC
:10B5B0000020FFF79FFF0020FFF7FCFD4FF4C8724B
:10B5C00000210D480CF086FD002201210B4B83F871
:10B5D000282083F829101A7002B010BDC421002061
:10B5E00085BB000860C601084C2500207DDF0108EE
:10B5F00063C60108C8210020CC210020EC240020D3
:10B6000073B50E4614460546FFF774FF3046FFF744
:10B610006BFC0520FFF7CEFD00230193019BB3F5E2
:10B62000CC7F0BDD2846FFF7AFFD0546FFF7DCFDBD
:10B63000A542CCBF0020012002B070BD019B0133A8
:10B64000EBE773B500240220FFF754FFFF21112020
:10B65000FFF73CFC0520FFF7ADFD25462646019689
:10B66000019BB3F5CC7F0DDD2C20FFF789FC00F0AA
:10B670000100A0400134202C45EA0005EFD1284606
:10B6800002B070BD019B01330193E9E700000000A7
:10B690002DE9F04F834687B00093109B0E4601932F
:10B6A0009DF85C309DF86010029315469DF864305B
:10B6B0009DF8582004910393BDF84470BDF84840AC
:10B6C0009DF84C809DF850909DF854A00592FFF78E
:10B6D00011FFDDE90331BBF1010F06D0BBF1020F11
:10B6E000059A66D007B0BDE8F08F7D4C019A2661BF
:10B6F0002846A561626184F81E8084F81F9084F852
:10B7000020A084F8211084F82230A7830BF026FAB9
:10B710000B46024670A1D1E900010BF0C3FB0BF010
:10B7200031FDC0F3072185B20220FFF7CFFBE9B25C
:10B730000320FFF7CBFB3046FFF748FB0146122002
:10B74000FFF7C4FB0198FFF741FB01461320FFF709
:10B75000BDFB2520390AFFF7B9FB2620F9B2FFF718
:10B76000B5FBE37FE3B9A37FD3B184F829B04946A1
:10B770003220FFF7ABFB3020FFF702FCB8F1000FDF
:10B7800014BF0021802100F06F0040EA0A1A302027
:10B7900041EA0A01C9B207B0BDE8F04FFFF796BB16
:10B7A00000234FF4D2714F4884F82930FAF706FF8E
:10B7B000DDE7DFF82CB10098CBF84060CBF84450BF
:10B7C0008BF84900ABF84A708BF84C808BF84D90A1
:10B7D0008BF84EA08BF84F20029A062D8BF8502044
:10B7E0002A4638BF06220C2A8BF8511028BF0C229B
:10B7F0008BF85230002E5CD1A2F10B03012B5CD8E8
:10B8000001238BF848301D200192FFF7B9FB9BF80C
:10B810004810009B41EA4A0141EA880141EAC3011C
:10B8200041EA8611C9B21D20FFF750FB1E20FFF729
:10B83000A7FB019AC4F3012141EA021200F00C00B7
:10B840000243D1B21E20FFF741FB1F20E1B2FFF7F8
:10B850003DFB2020390AFFF739FB2120F9B2FFF721
:10B8600035FBB8F1000F03D049462220FFF72EFB2D
:10B870009BF84F306BB14B20FFF782FB60F07F01EC
:10B88000C9B24B20FFF722FB24209BF85010FFF792
:10B890001DFB062D4FF0310011D8FFF771FB00F0B2
:10B8A000F80141F005013120FFF710FB0C21372092
:10B8B00071E7012E01D10B2DA2D80023A1E7FFF7DC
:10B8C0005FFB00F0F80141F003013120FFF7FEFAC1
:10B8D0000A21ECE7AFF300800000000080847E4185
:10B8E000EC2400207DDF01082DE9F04F89B01D46D2
:10B8F0009DF84C30079101939DF85C30924604937B
:10B900009DF86030009005939DF86430129E02937C
:10B910001A9BBDF8507003939DF854809DF8589081
:10B92000FFF7E8FD0920FFF72BFB04465A20FFF73D
:10B9300027FB04F07F03924C834660680693FFF771
:10B940003BFA069B0799034313F0800F03F0F00CBA
:10B9500029D011291DDD14290B46A8BF14234BF053
:10B9600007025FFA82FB591F4CEA01010920C9B2A4
:10B970000693FFF7ABFA59465A20FFF7A7FA009B48
:10B98000012B069B17D0009A022A6AD009B0BDE8A5
:10B99000F08F02290B46B8BF02230BF0F80242F0E9
:10B9A000040B991EE0E70E290B46A8BF0E2343EABD
:10B9B000E373591CD8E72372029BC4F80CA02561DD
:10B9C000A661A78384F81E8084F8209084F8213033
:10B9D000039B504663620BF0C1F865A3D3E90023D3
:10B9E0000BF060FA0BF0CEFB84B2C0F30721042009
:10B9F000FFF76CFAE1B20520FFF768FA30460BF06A
:10BA0000ADF802460B465CA1D1E900010BF04AFA01
:10BA10000BF0B8FBC0F3072184B20220FFF756FAFF
:10BA20000320E1B2FFF752FA2520390AFFF74EFA58
:10BA3000F9B22620FFF74AFA3020FFF7A1FAB8F151
:10BA4000000F14BF0021802100F06F0040EA0919A7
:10BA5000302041EA0901C9B209B0BDE8F04FFFF753
:10BA600035BA062EB24638BF4FF0060A84F83C308D
:10BA7000019B2564666484F84930049BA4F84A70ED
:10BA800084F84C8084F84F30059BBAF10C0F84F891
:10BA90005030029B84F84E9084F85130039B28BFAD
:10BAA0004FF00C0ADFF8D8B06365002D4CD1AAF135
:10BAB0000B03012B4CD801238BF848309BF84F30F7
:10BAC0006BB14B20FFF75CFA60F07F01C9B24B20ED
:10BAD000FFF7FCF924209BF85010FFF7F7F91D2021
:10BAE000FFF74EFA94F84810019B41EA490141EAF8
:10BAF000880141EAC30141EA8511C9B21D20FFF75F
:10BB0000E5F91E20FFF73CFA00F00F0141EA0A11A7
:10BB10001E20C9B2FFF7DAF92020390AFFF7D6F95B
:10BB20002120F9B2FFF7D2F9062E4FF0310011D8DB
:10BB3000FFF726FA00F0F80141F005013120FFF788
:10BB4000C5F90C21372087E7012D01D10B2EB2D882
:10BB50000023B1E7FFF714FA00F0F80141F0030108
:10BB60003120FFF7B3F90A21ECE700BFAFF3008003
:10BB70000000000080844E400000000080847E4170
:10BB8000EC24002010B5254C2378012BDAB202D02A
:10BB9000022A34D010BD6378012B29D100230B2158
:10BBA0003E2084F82C3084F82D302387E386FFF77D
:10BBB0008DF910213F20FFF789F994F8223003F026
:10BBC000FF029BB10D20FFF7DBF940F02001C9B265
:10BBD0000D20FFF77BF9124B1B68002BDAD0DB68D6
:10BBE000002BD7D0BDE81040002018472270F2E7A4
:10BBF00094F85230002BEED0FFF716FBEBE7002352
:10BC000001222370074B1A70054B1B68002BC1D013
:10BC10005B68002BBED0BDE810401847EC24002024
:10BC2000C42100207025002007B50022154B8DF897
:10BC3000072083F82C2083F82D201A87DA8683F8D2
:10BC40002E2093F8223023B903B05DF804EBFFF700
:10BC5000CBBA3F20FFF794F98DF807009DF8073025
:10BC6000DB0603D510213F20FFF730F90D20FFF749
:10BC700087F940F040010D20C9B203B05DF804EB34
:10BC8000FFF724B9EC2400202DE9F04107460C4EC3
:10BC90000020F3680C4615469847336907F07F008B
:10BCA00098472544AC4204D1F3680120BDE8F04137
:10BCB0001847002033699847C04304F8010BF1E7A7
:10BCC000502500200A4601460020FFF7E3B8000097
:10BCD000F7B55F4C064663780D46012BDAB212D0F9
:10BCE000022A42D000252846FFF778FB6378012B13
:10BCF00040F0AB80002D00F0A880564E564D3378B2
:10BD0000002B76D0A1E000232387E186A37F73B1C7
:10BD1000C9B23220FFF7DAF83120FFF731F9C5F365
:10BD2000022100F0F80001433120FFF7CFF86B1E2D
:10BD30003F2B10D8EDB284F83B500025304694F8E4
:10BD40003B10FFF7BFFF94F83B30228F13449BB2A8
:10BD50002387606AC8E72A4631463F480CF092F9CB
:10BD60002B23012584F83B30E8E794F85130332049
:10BD700033B3FFF705F900F0BE013320FFF7A6F853
:10BD800019213B20EDB2FFF7A1F82946222084F8C3
:10BD90005C50FFF79BF800210E20FFF797F8002179
:10BDA0000D20FFF793F80120FFF7EAF830F0F807CD
:10BDB00011D029463046FFF785FF0025606D93E7D7
:10BDC000FFF7DEF800F0BE0141F001013320FFF77C
:10BDD0007DF81D21D5E7FFF727FA0197019BB3F501
:10BDE000CC7FE6DC019B01330193F7E7012001F0F2
:10BDF0007BFD3F20FFF7C4F88306F7D4E38E228F44
:10BE00009BB294F83B1092B2208F9B1A8B4280B267
:10BE10000BDD94F83B102844FFF754FF94F83B30B7
:10BE2000228F13449BB2238769E7E18E238F284436
:10BE3000C91AC9B2FFF746FFE38E218F228F9BB24A
:10BE400092B213445B1A9BB2238703B0F0BD00BFCC
:10BE5000EC24002070250020CC2100200A46014659
:10BE60000020FFF76FB80A4601460020FFF70CBF1D
:10BE700038B505460C46FFF73DFB012D02D0022DDB
:10BE80000AD038BD064B9B7F002BFAD121463220C9
:10BE9000BDE83840FFF71AB821462320F8E700BF75
:10BEA000EC2400207FB50022694C8DF80B2023780C
:10BEB0000392012BD9B204D0022900F0A68004B06D
:10BEC00070BD6378012BDAB236D0022AF7D1402157
:10BED0001220FEF7FBFF1220FFF752F88DF80B003F
:10BEE0009DF80B305B4E13F0200F2BD02021122039
:10BEF000FEF7ECFF94F8523003F0FF0203B9227012
:10BF000000225548009203AB0821006802F060FA55
:10BF1000039B4BB14FF0E0234FF08052C3F8042D48
:10BF2000BFF34F8FBFF36F8F3368002BC7D01B69F0
:10BF3000002BC4D09847C2E740F229514748FAF78E
:10BF40003DFBBCE71920FFF71BF840B284F858000E
:10BF500094F8583094F858501B0642BF6DB26D42A9
:10BF6000C5F385054FF01A004CBF6D42AD08FFF7D1
:10BF700007F8002DB8BF2D1840F30B13B4BF8B3D4D
:10BF80008B389BB2ACBF1B185B191BB21320A4F8F3
:10BF90005A30FEF7F5FF84F85C001020FEF7F0FF42
:10BFA00001460D20FEF792FF94F85C102C48FFF735
:10BFB00055FF94F8523003F0FF029BB926480092D7
:10BFC00003AB08210068227002F002FA039B4BB118
:10BFD0004FF0E0234FF08052C3F8042DBFF34F8F92
:10BFE000BFF36F8F3368002B3FF469AF9D68002D5E
:10BFF0003FF465AF94F85C10B4F85A2094F85830C8
:10C0000017485BB212B2A84759E71348009203AB36
:10C010000821006802F0DCF9039B4BB14FF0E023EC
:10C020004FF08052C3F8042DBFF34F8FBFF36F8FD3
:10C030006378022B03D108211220FEF747FF00236B
:10C040002370044B1B68002B3FF439AF1B686FE76C
:10C05000EC240020C4210020C82100207DDF01083D
:10C06000CC2100202DE9FF4100256C4C8DF80B50B0
:10C0700023780395012BDAB205D0022A00F0CC8098
:10C0800004B0BDE8F0816378012BDAB225D0022A32
:10C09000F6D16348009503AB2A460821006802F0F8
:10C0A00097F9039B4BB14FF0E0234FF08052C3F858
:10C0B000042DBFF34F8FBFF36F8F80211220FEF747
:10C0C00005FF00232370574B1B68002BD8D0DB687B
:10C0D000002BD5D001209847D2E73F20FEF750FF34
:10C0E0008DF80B009DF80B309A06C9D59DF80B30E2
:10C0F000DB0619D5E18E228F4B4892B289B2FEF74A
:10C1000053F84A4E4A4F94F83A30AB4205DC49485E
:10C11000FEF74AF8FFF788FDB2E7384616F8011B2C
:10C12000FEF742F80135EEE794F8293023B940F2E2
:10C13000DD514148FAF742FA94F82830022B3CD1FD
:10C14000238F3A489BB294F83A101844FFF78BFEBD
:10C15000238F9BB2002B4BD094F83A30228F13449C
:10C160009BB22387228FE38E92B29BB29A4287D3EF
:10C170002E4DE28E294692B230480BF083FFFF230A
:10C180002B7011236B70DD23AB70EE23EB7094F8F2
:10C190002E50E48EFFF748FD224B6DB21B68A4B20F
:10C1A000002B3FF46DAF9E68002E3FF469AF002373
:10C1B0002A4621462148B04762E7214F0020FB680C
:10C1C000984700203B6998470026DFF8608094F884
:10C1D0003A30B34203DC0120FB689847B8E70020FF
:10C1E0003B69258F9847ADB24544A8550136EEE727
:10C1F00094F82D30002B8DD094F83A100B48FEF7B0
:10C20000C1FDE086E38E9BB2B3F5C87F82D2E38E98
:10C210009BB2002BA0D17DE7637831E7EC240020AE
:10C22000C8210020C421002066C60108CC210020BE
:10C230007BC601087CDF01087DDF01085C2300204C
:10C240005025002010B51B4C2378012BDAB202D008
:10C25000022A2AD010BD6378012BD9B218D0022946
:10C26000F8D194F84F30002BF4D01220FEF72EFEB8
:10C27000114B1B68002BEDD05C69002CEAD01C2010
:10C28000FEF77EFE2346BDE8104000F03F00184751
:10C2900000231120238784F82D10FEF771FE40083B
:10C2A000404240B284F82E00D4E76378D9B2022B22
:10C2B000D6E700BFEC240020C421002070B51F4B3E
:10C2C0005A78022A05D11B78012BDAB202D0032A50
:10C2D00013D070BD1220FEF753FEC306F9D510210E
:10C2E0001220FEF7F3FD164B1B68002BF1D0DB6923
:10C2F000002BEED0BDE8704018471220FEF740FE3C
:10C3000010F001040E4D0DD005211220FEF7DEFDC8
:10C310002B68002BDDD09B69002BDAD00120BDE813
:10C320007040184704211220FEF7D0FD2B68002B27
:10C33000CFD09B69002BCCD02046F0E7EC24002026
:10C34000C421002006480068006880F3088862B6AF
:10C3500061B6BFF34F8FBFF36F8F00DF00BF0000E8
:10C3600008ED00E0002307B501930B4B1B68013378
:10C3700003D0CA210948FAF721F94FF0500383F39B
:10C380001188BFF36F8FBFF34F8F019B002BFCD041
:10C3900003B05DF804FB00BFC00200207DDF010890
:10C3A0004FF0807340F8043C054B21F0010140F848
:10C3B000081C40F80C3C40F8202C4038704700BF67
:10C3C00065C300080000000000000000000000003D
:10C3D000074B19680868B0E8F00F80F30988BFF3CD
:10C3E0006F8F4FF0000080F311884EF00D0E7047F4
:10C3F000A42500204FF0500383F31188BFF36F8F03
:10C40000BFF34F8F084A13680133012B13600AD121
:10C410004FF0E023D3F8043DDBB223B140F27511B5
:10C420000248FAF7CBB87047C00200207DDF010850
:10C4300010B5074C236823B94FF4BE710548FAF7CD
:10C44000BDF82368013B23600BB983F3118810BD4D
:10C45000C00200207DDF0108000000000000000095
:10C46000EFF30980BFF36F8F0D4B1A6820E9F00FCF
:10C4700010602DE908404FF0500080F3118801F062
:10C4800059FA4FF0000080F31188BDE808401968A0
:10C490000868B0E8F00F80F30988BFF36F8F70472A
:10C4A000A425002008B54FF0500383F31188BFF393
:10C4B0006F8FBFF34F8F01F0D3F828B14FF0E02317
:10C4C0004FF08052C3F8042D002383F3118808BD78
:10C4D0004FF0E02300221A619A6141F267025A612B
:10C4E00007221A617047000013B5284B284C1A78B0
:10C4F000D2B20192FF221A701B78264ADBB28DF865
:10C5000003309DF8033003F050031370072300221B
:10C5100023609DF80310581E09062DD412B1032B79
:10C52000236004D04FF49B711B48FAF747F8236847
:10C53000164A1B0203F4E0632360019B0024DBB274
:10C5400013704FF0E023D3F8202D42F47002C3F8AB
:10C55000202DD3F8202D42F07042C3F8202DFFF794
:10C56000B7FF0E4B1C60FFF7EDFE01F0E3F9FFF79C
:10C57000F9FE204602B010BD9DF8033001225B0099
:10C58000DBB28DF803300346C3E700BF00E400E0F0
:10C5900074250020712500207DDF0108C0020020E5
:10C5A00008B5EFF305830F2B0AD90E4A9B5C0E4AA0
:10C5B00012789A4204D940F2A5210C48F9F7FEFFFF
:10C5C0004FF0E0230A4AD3F80C3D126803F4E0630D
:10C5D000934206D9BDE8084040F2B5210348F9F777
:10C5E000EDBF08BDF0E300E0712500207DDF01080C
:10C5F0007425002070B50C46064601F015F80D4B69
:10C600000D491D682A198A4207D90C23336001F0AD
:10C61000B7F84FF0FF35284670BD1A60074A136817
:10C620001B1B1360064B19682144196001F0A8F820
:10C63000F1E700BFC40200206C6B0020C80200209C
:10C640007825002008B5EFF305831BB1C22103480C
:10C65000F9F7B4FFBDE8084000F0E6BF7DDF010850
:10C6600001F08EB800F0E0BF01F08AB80BF0DCBC3E
:10C670000BF0E2BC00B58BB068460BF0A5FF034B96
:10C6800008981B6818440BB05DF804FBC802002032
:10C690000020704770470000004870476C2B002056
:10C6A00010B50446FFF7A6FEA46BFFF7C1FEB4FA6F
:10C6B00084F0400910BDF8B51546026C0446866B3F
:10C6C00052B9076847BB806801F0EEFB0546A760DA
:10C6D00001362846A663F8BD65B940680BF0D2FC68
:10C6E0006368226C1344A26863609342F0D32368AA
:10C6F0006360EDE7C0680BF0C5FC226CE368514253
:10C700009B1A2268E36093423EBFA3685B18E36014
:10C71000022D01D116B1013E0025D9E73546D7E7F4
:10C7200003461A6C084610B462B1DC689968144478
:10C730008C4228BF1968DC6028BFD960D96810BC5A
:10C740000BF0A0BC10BC704770B50446FFF752FE5A
:10C7500094F8455004F124066DB2002D14DCFF233B
:10C7600084F84530FFF764FEFFF744FE94F8445028
:10C7700004F110066DB2002D12DCFF2384F8443062
:10C78000BDE87040FFF754BE636A002BE7D0304627
:10C7900001F0CCF908B101F04BFA013D6DB2DCE7D4
:10C7A0002369002BE9D0304601F0C0F908B101F04F
:10C7B0003FFA013D6DB2DEE738B50D46044620B9BB
:10C7C00040F203111A48F9F7F9FEFFF713FED4E916
:10C7D0000F314B432268D0185B1A1344A060E3600A
:10C7E0000020FF23A063626084F8443084F8453061
:10C7F000A5B9236973B104F1100001F097F948B1AC
:10C800004FF0E0234FF08052C3F8042DBFF34F8F59
:10C81000BFF36F8FFFF70CFE012038BD04F110004D
:10C8200001F028FF04F1240001F024FFF2E700BF2B
:10C830007DDF0108F8B50D461746064620B94FF4CE
:10C84000BB710D48F9F7BAFE05FB06F05030FFF753
:10C850000DFF044658B165B100F150030121204697
:10C86000C4E90F652360FFF7A7FF84F84C702046EA
:10C87000F8BD0346F2E700BF7DDF01082DE9F04374
:10C8800085B00F461E460446019220B940F2F121C0
:10C890004C48F9F793FE37B9236C23B140F2F221EB
:10C8A0004848F9F78BFE022E07D1E36B012B04D029
:10C8B00040F2F3214348F9F781FE01F093FA30B9D1
:10C8C000019B23B140F2F6213E48F9F777FE4FF085
:10C8D0000008C146FFF78EFDA26BE36B9A4201D3BD
:10C8E000022E1BD1324639462046FFF7E4FE636A2A
:10C8F0001BB104F1240001F019F948B14FF0E02315
:10C900004FF08052C3F8042DBFF34F8FBFF36F8FEA
:10C91000FFF78EFD012005B0BDE8F083019D1DB934
:10C92000FFF786FD0020F6E7B8F1000F02D102A85C
:10C9300001F03CF9FFF77CFD00F076FEFFF75AFDB1
:10C9400094F84430FF2B08BF84F8449094F84530A5
:10C95000FF2B08BF84F84590FFF76AFD01A902A8E4
:10C9600001F030F940BBFFF745FDA26BE36B9A4243
:10C970000FD1FFF75DFD019904F1100001F09CF863
:10C980002046FFF7E1FE00F0FBFE50B14FF001083A
:10C99000A0E7FFF74DFD2046FFF7D6FE00F0F0FEC2
:10C9A000F4E74FF0E0234FF08052C3F8042DBFF3BB
:10C9B0004F8FBFF36F8FE9E72046FFF7C5FE00F00A
:10C9C000DFFEAFE77DDF0108024610B50021012040
:10C9D000FFF730FF044638B100231A46194683603A
:10C9E0000360C360FFF74AFF204610BD2DE9F843FE
:10C9F000894690461F46044620B940F2C331274875
:10CA0000F9F7DCFDB9F1000F06D1236C23B14FF427
:10CA100071712248F9F7D2FD022F07D1E36B012B88
:10CA200004D040F2C5311D48F9F7C8FDFFF7B8FD45
:10CA3000EFF311864FF0500383F31188BFF36F8F2C
:10CA4000BFF34F8FA26BE36B9A4201D3022F22D127
:10CA500094F845503A46494620466DB2FFF72BFE02
:10CA60006B1C13D1636A0BB901200BE004F12400A5
:10CA700001F05CF80028F7D0B8F1000FF4D00120E5
:10CA8000C8F8000086F31188BDE8F88301356DB25F
:10CA900084F84550E8E70020F4E700BF7DDF010897
:10CAA00070B50D46044620B94FF48C612048F9F763
:10CAB00085FD236C23B140F264411D48F9F77EFDEA
:10CAC000236833B9A36823B140F269411848F9F7E4
:10CAD00075FDFFF765FDEFF311864FF0500383F30B
:10CAE0001188BFF36F8FBFF34F8FA26BE36B93423D
:10CAF0001CD994F845100132FF294BB2A26310D122
:10CB0000636A0BB9012009E004F1240001F00EF87A
:10CB10000028F7D0002DF5D00120286086F3118879
:10CB200070BD01335BB284F84530EBE70020F5E7D8
:10CB30007DDF01082DE9FF410E460446019220B930
:10CB40004FF4A0614348F9F739FD36B9236C23B19E
:10CB500040F204513F48F9F731FD01F043F930B993
:10CB6000019B23B140F209513A48F9F727FD00270C
:10CB7000B846FFF73FFCA56BE5B131462046013DC5
:10CB8000FFF7CEFDA563236973B104F1100000F037
:10CB9000CDFF48B14FF0E0234FF08052C3F8042D91
:10CBA000BFF34F8FBFF36F8FFFF742FC012004B03C
:10CBB000BDE8F081019D1DB9FFF73AFC0020F6E7C2
:10CBC00017B902A800F0F2FFFFF732FC00F02CFDCD
:10CBD000FFF710FC94F84430FF2B08BF84F8448022
:10CBE00094F84530FF2B08BF84F84580FFF720FC00
:10CBF00001A902A800F0E6FF00BB2046FFF750FDA8
:10CC0000B0B1019904F1240000F056FF2046FFF76F
:10CC10009BFD00F0B5FD48B94FF0E0234FF0805286
:10CC2000C3F8042DBFF34F8FBFF36F8F0127A0E729
:10CC30002046FFF789FD00F0A3FDF7E72046FFF748
:10CC400083FD00F09DFD2046FFF72AFD0028EDD072
:10CC5000B4E700BF7DDF0108F0B585B0044601915F
:10CC600020B940F291515248F9F7A8FC236C23B146
:10CC700040F295514E48F9F7A1FC01F0B3F830B9F4
:10CC8000019B23B140F29A514948F9F797FC0025DE
:10CC90002F462E46FFF7AEFBA36BEBB1013BA36320
:10CCA000236813B901F0A0F9A060236973B104F1FE
:10CCB000100000F03BFF48B14FF0E0234FF08052EE
:10CCC000C3F8042DBFF34F8FBFF36F8FFFF7B0FB97
:10CCD0000125284605B0F0BD019B4BB925B140F2B6
:10CCE000E1513348F9F76AFCFFF7A2FB0025F0E7B2
:10CCF00017B902A800F05AFFFFF79AFB00F094FC66
:10CD0000FFF778FB94F84430FF2B08BF84F84460A9
:10CD100094F84530FF2B08BF84F84560FFF788FB87
:10CD200001A902A800F04EFF50BB2046FFF7B8FC57
:10CD300000B323683BB9FFF75DFBA06801F062F820
:10CD40000546FFF775FB019904F1240000F0B4FEDD
:10CD50002046FFF7F9FC00F013FD48B94FF0E0233F
:10CD60004FF08052C3F8042DBFF34F8FBFF36F8F86
:10CD700001278FE72046FFF7E7FC00F001FDF7E70A
:10CD80002046FFF7E1FC00F0FBFC2046FFF788FCA3
:10CD90000028EDD0002D9CD0FFF72CFB616A19B163
:10CDA000236B1968C1F10501A06801F0C9F89BE780
:10CDB0007DDF01082DE9FF410E460446019220B9AE
:10CDC0004FF4CD614348F9F7F9FB36B9236C23B131
:10CDD00040F26C613F48F9F7F1FB01F003F830B91C
:10CDE000019B23B140F271613A48F9F7E7FB002754
:10CDF000B846FFF7FFFAA36BE3B131462046E5687A
:10CE0000FFF78EFC636AE56073B104F1240000F063
:10CE10008DFE48B14FF0E0234FF08052C3F8042D4F
:10CE2000BFF34F8FBFF36F8FFFF702FB012004B0FA
:10CE3000BDE8F081019D1DB9FFF7FAFA0020F6E781
:10CE400017B902A800F0B2FEFFF7F2FA00F0ECFB0F
:10CE5000FFF7D0FA94F84430FF2B08BF84F84480E1
:10CE600094F84530FF2B08BF84F84580FFF7E0FABF
:10CE700001A902A800F0A6FE00BB2046FFF710FCA7
:10CE8000B0B1019904F1240000F016FE2046FFF72E
:10CE90005BFC00F075FC48B94FF0E0234FF0805286
:10CEA000C3F8042DBFF34F8FBFF36F8F0127A0E7A7
:10CEB0002046FFF749FC00F063FCF7E72046FFF748
:10CEC00043FC00F05DFC2046FFF7EAFB0028EDD0B4
:10CED000B4E700BF7DDF01082DE9F843894690469D
:10CEE000054620B940F2FB612048F9F767FBB9F12C
:10CEF000000F06D12B6C23B140F2FC611B48F9F7FF
:10CF00005DFBFFF74DFBEFF311874FF0500383F309
:10CF10001188BFF36F8FBFF34F8FAC6B1CB395F8C5
:10CF200044604946284676B2FFF7FAFB013C731C81
:10CF3000AC6313D12B690BB901200BE005F1100094
:10CF400000F0F4FD0028F7D0B8F1000FF4D0012074
:10CF5000C8F8000087F31188BDE8F883013676B27F
:10CF600085F84460E8E72046F4E700BF7DDF01086C
:10CF700010B5044620B940F28A710548F9F71EFB46
:10CF8000FFF738FAA46BFFF753FA204610BD00BF35
:10CF90007DDF010810B5044620B940F2A4710648AF
:10CFA000F9F70CFBFFF726FAA06BE46B241AFFF7E6
:10CFB0003FFA204610BD00BF7DDF0108002310B5F9
:10CFC000064A52F833402CB942F8331002EBC3033F
:10CFD000586010BD0133052BF3D1FAE77C25002002
:10CFE000002310B5074A02EBC3014C68844204D108
:10CFF000002042F83300486010BD0133052BF2D108
:10D00000FAE700BF7C25002010B5044620B94FF494
:10D01000F8610548F9F7D2FA2046FFF7E1FF20460C
:10D02000BDE81040FFF724BB7DDF010870B5044662
:10D030000D461646FFF7DEF994F84430FF2B04BF87
:10D04000002384F8443094F84530FF2B04BF0023BC
:10D0500084F84530FFF7ECF9A36B2BB9324629462B
:10D0600004F1240000F042FD2046BDE87040FFF7C7
:10D070006BBB000080B5174D174F184E2B6873B966
:10D08000174B1B68012BF8D94FF0E0234FF080526B
:10D09000C3F8042DBFF34F8FBFF36F8FEDE7FFF79A
:10D0A000A9F9FB68DC68201D01F015FB3368013B22
:10D0B00033602B68013B2B60FFF7BAF904F1540091
:10D0C0000BF024FF206BFFF7D3FA2046FFF7D0FACE
:10D0D000D4E700BF182600208C260020142600204C
:10D0E000B0250020F8B51A4B1A4D06461C68286872
:10D0F0000F46043001F0EFFA40B92A681649D06AA9
:10D1000001220B68824023EA02030B60731C07D1E3
:10D1100037B1296811480431BDE8F84001F0B8BAC8
:10D120002B68A4195C6007D30D4B18682968BDE80B
:10D13000F840043101F0B8BA0A4B18682968043184
:10D1400001F0B2FA084B1A68A24288BF1C60F8BD11
:10D15000A0260020A42500202826002078260020D4
:10D16000AC250020A825002058260020064A136878
:10D170001968064B19B94FF0FF321A6070471268F0
:10D18000D268D2685268F8E7A82500205826002007
:10D1900010B5044620B940F2F2610848F9F70EFADA
:10D1A0006269074B9A4207D1A06A064B984203D0A6
:10D1B000B0FA80F0400910BD0020FCE77DDF0108D7
:10D1C00078260020602600202DE9F84F4FEA820AD9
:10D1D000064650460D461F46DDF82C90FFF746FAEE
:10D1E0008046002800F0B580BC20FFF73FFA0446D7
:10D1F000002800F0AB80C0F8308025B94FF458719A
:10D200005B48F9F7DBF95246A521206B0AF062FF73
:10D21000236BAAF1040A9A442AF0070A6B1E04F150
:10D2200034020F3513F8011F02F8011B09B19D42AA
:10D23000F8D10A9D4FF0000B042D28BF042504F1FE
:10D2400004084046C4E9135BE56284F843B001F08A
:10D250001CFAC5F1050504F1180001F016FA602268
:10D260005946C4F8B4B02461A561646284F8B8B0CA
:10D2700004F154000AF02EFF3E4B3A46A3653E4BA4
:10D280003146E3653D4B50462366FFF789F8206041
:10D29000B9F1000F01D0C9F80040FFF7ABF8384BE7
:10D2A000384E1A68384F01321A603568002D53D154
:10D2B00034601B68012B1FD1B9464846013501F087
:10D2C000D9F9052D09F11409F7D1DFF8C090304DD7
:10D2D000484601F0CFF9284601F0CCF92D4801F07D
:10D2E000C9F92D4801F0C6F92C4801F0C3F92C4BBF
:10D2F000C3F800902B4B1D6001252B4A2B49136866
:10D30000086801331360E26A636405FA02F30343B9
:10D3100014200B6000FB0270414601F0B9F9FFF7E1
:10D3200087F8234B1B6873B13368DA6AE36A9A4261
:10D3300009D24FF0E0234FF08052C3F8042DBFF321
:10D340004F8FBFF36F8F2846BDE8F88F4046FFF739
:10D350008FF94FF0FF35F6E7154B1B68002BCBD14B
:10D360003368DA6AE36A9A4298BF3460C4E700BF60
:10D370007DDF010844E7010864E7010824E70108AC
:10D3800014260020A4250020B02500202C260020F3
:10D3900040260020602600208C26002078260020D1
:10D3A000A8250020AC2500202426002028260020C7
:10D3B00074260020F8B504462B4DFFF71BF804B97E
:10D3C0002C68261D304601F086F960B91420E76A02
:10D3D000264B78431B5833B901222549BA400B68C4
:10D3E00023EA02030B60A36A1BB104F1180001F0E9
:10D3F00072F9204A1368013313602B68A34222D1CB
:10D4000031461D4801F044F91C4A1368013313608A
:10D41000FFF70EF81A4B1B68A3B12B68A34211D17A
:10D42000184B1B6823B140F2B6411748F9F7C6F80C
:10D430004FF0E0234FF08052C3F8042DBFF34F8F1D
:10D44000BFF36F8FF8BD114A04F154001368013B1C
:10D4500013600BF05BFD206BFFF70AF92046FFF726
:10D4600007F9FFF783FED3E7A4250020B0250020AD
:10D4700028260020242600208C26002018260020A4
:10D4800074260020202600207DDF010814260020BD
:10D49000F8B5044620B940F24C511748F9F78EF818
:10D4A000164B1B68A34220D0FEF7A4FF144B6569FE
:10D4B0001F68144B1E68FEF7BBFFBD4217D0B54274
:10D4C00015D0114B9D4208D1A36A83B994F8B830A6
:10D4D000012B0CBF02200320F8BD0C4B9D4208D04D
:10D4E000002D0CBF04200120F6E70020F4E7022005
:10D4F000F2E70420F0E700BF7DDF0108A42500204B
:10D50000A8250020AC250020782600208C260020AD
:10D5100070B5044620B940F21C711A48F9F74EF86C
:10D52000194D2B68A3422BD054B3FEF763FF20465E
:10D53000FFF72EFE00B3261D304601F0CCF8012384
:10D540001249E26A08689340034314200B60104BB1
:10D55000314600FB023001F09BF82B68E26ADB6A7F
:10D560009A4209D34FF0E0234FF08052C3F8042DC4
:10D57000BFF34F8FBFF36F8FBDE87040FEF758BF0A
:10D5800070BD00BF7DDF0108A425002028260020F3
:10D59000B025002013B500241A4B502201931A49DC
:10D5A00023461A480094FFF70FFE01281DD100F012
:10D5B000C7FE012819D14FF0500383F31188BFF340
:10D5C0006F8FBFF34F8F124B124A1B685433136097
:10D5D0004FF0FF32104B1A60104B1860104B1C605C
:10D5E00002B0BDE81040FEF77FBF013007D140F622
:10D5F00004010C4802B0BDE81040F8F7DFBF02B0EC
:10D6000010BD00BF5426002050C7010875D0000887
:10D61000A425002030050020582600207426002074
:10D62000A02600207DDF0108024A13680133136041
:10D63000704700BF20260020014B1868704700BFCC
:10D64000A026002008B5FEF7ABFF014B186808BD07
:10D65000A0260020014B1868704700BF1426002048
:10D660002DE9F84F3A4B1B68002B6AD1394B1D68E6
:10D6700001351D609DB9384C23681B6823B140F605
:10D6800062213648F8F79AFF354B22681968216005
:10D690001A60344A136801331360FFF767FD324E96
:10D6A00000243368314FAB4210D91422304B1B6831
:10D6B000DB6A5343FB58022B28BF01242D4B1B6808
:10D6C000002B0CBF20460120BDE8F88FDFF888A0B2
:10D6D000DFF8A490DAF800301B681BB94FF0FF3375
:10D6E0003360E2E7DAF80030DB68D3F80CB0DBF83F
:10D6F0000420954201D23260D7E70BF1040840467E
:10D7000000F0E9FFDBF828201AB10BF1180000F057
:10D71000E2FF0122DBF82C00D9F8003082401A43E6
:10D72000C9F800201422414602FB007000F0B0FF4F
:10D730000F4BDBF82C201968CB6A9A4228BF0124D2
:10D74000C8E70E4A0024136801331360B6E700BF30
:10D7500020260020A0260020A82500207DDF01082B
:10D76000AC2500205C26002058260020B025002093
:10D77000A4250020A4260020282600201C26002006
:10D780002DE9F8432F4C236823B940F668012E4851
:10D79000F8F714FFFEF72EFE2368013B2360246890
:10D7A0002CB10024FEF744FE2046BDE8F883274B49
:10D7B0001B68002BF5D0264D264EDFF89C801FE01D
:10D7C000EB680127DC6804F1040904F1180000F09B
:10D7D00082FF484600F07FFF1420E26A316807FAB2
:10D7E00002F30B4300FB02804946336000F050FF18
:10D7F0001A4BE26A1B68DB6A9A4201D3184B1F601E
:10D800002B68002BDCD10CB1FFF7B0FC154D2C6858
:10D8100044B10127124EFFF723FF00B13760013CEE
:10D82000F9D12C600E4B1B68002BBAD04FF0E023CF
:10D830004FF08052C3F8042DBFF34F8FBFF36F8FAB
:10D840000124AFE7202600207DDF010814260020F8
:10D850006026002028260020B0250020A4250020D6
:10D86000A42600201C26002038B50C46054620B909
:10D8700040F2CA411948F8F7A1FE24B940F2CB4161
:10D880001648F8F79BFE164B1B6823B140F2CC41BB
:10D890001248F8F793FEFFF7C7FE124B2A68186884
:10D8A00014192CBF0121002182422C600ED971B9BC
:10D8B000FFF766FF48B94FF0E0234FF08052C3F8FE
:10D8C000042DBFF34F8FBFF36F8F38BD09B9A0424E
:10D8D000EED20021201AFFF705FCE9E77DDF010801
:10D8E00020260020A026002010B5044650B94FF095
:10D8F000E0234FF08052C3F8042DBFF34F8FBFF3E6
:10D900006F8F10BD094B1B6823B14FF4A461084809
:10D91000F8F754FE00212046FFF786FEFFF7E2FBF2
:10D92000FFF72EFF0028E2D0EBE700BF2026002003
:10D930007DDF0108244B70B51A68244B12B1012217
:10D940001A6070BD224E1A6033681B6B1A68B2F100
:10D95000A53F0BD15A68B2F1A53F07D19A68B2F141
:10D96000A53F03D1DB68B3F1A53F04D0306831682F
:10D970003431F8F7EFFD174B1C68B4FA84F4142324
:10D98000E4B2C4F11F046343134DEB5823B940F6CE
:10D9900088311248F8F712FE142000FB04F3EA184D
:10D9A0005168083349682B44994200FB045408BF6E
:10D9B0004B68516008BF53606368094ADB68336095
:10D9C000336854331360BCE720260020A4260020CF
:10D9D000A425002028260020B02500207DDF010896
:10D9E00030050020F8B504462B4DFEF703FD04B9C1
:10D9F0002C68261D304600F06EFE60B91420E76AE0
:10DA0000264B78431B5833B901222549BA400B688D
:10DA100023EA02030B60A36A1BB104F1180000F0B3
:10DA20005AFE31461F4800F033FE94F8B8301E4EBF
:10DA3000012B04BF002384F8B830FEF7F9FC3368EB
:10DA40002BB1FEF7D7FCFFF791FBFEF7F1FC2B683B
:10DA5000A34213D1336893B1144B1B6823B14FF425
:10DA6000D9611348F8F7AAFD4FF0E0234FF0805238
:10DA7000C3F8042DBFF34F8FBFF36F8FF8BD094A72
:10DA800011680C4A1268914201D12B60F6E7BDE89B
:10DA9000F840FFF74FBF00BFA4250020B0250020AD
:10DAA000282600207826002074260020202600202A
:10DAB0007DDF01081426002038B50D46044620B944
:10DAC00040F69F310748F8F779FD074B2046196863
:10DAD000183100F0E9FD2846BDE838400121FFF784
:10DAE00001BB00BF7DDF0108A425002070B50E46F4
:10DAF0001446054620B940F6CA310A48F8F75EFDDB
:10DB0000094B28461968183100F0C2FD002C214647
:10DB100008BF3046BDE8704018BF4FF0FF30FFF738
:10DB2000E1BA00BF7DDF0108A425002038B5C36835
:10DB3000DC6824B940F6FA311548F8F73FFD04F1E6
:10DB40001805284600F0C7FD124B1B68E3B9251DD8
:10DB5000284600F0C0FD01230F49E26A086893409F
:10DB6000034314200B6029460C4B00FB023000F0ED
:10DB70008FFD0B4BE26A1B68DB6A9A4285BF01206E
:10DB8000084B0020186038BD29460748EFE700BF62
:10DB90007DDF01082026002028260020B025002057
:10DBA000A4250020A426002060260020034B1B682B
:10DBB0000360034B1B684360704700BF5C26002076
:10DBC000A026002070B50C46054620B940F66541F8
:10DBD0001448F8F7F3FC24B940F666411148F8F709
:10DBE000EDFCFEF707FC104B196823685A1C10D097
:10DBF0000E482E6800686A68864201D08A420FD9B2
:10DC0000881A83420AD95B1A134428462360FFF717
:10DC1000CDFF0024FEF70CFC204670BD00232360DE
:10DC20000124F7E77DDF0108A02600205C26002004
:10DC30000122014B1A607047A426002070B50C46E3
:10DC40001646054608B91B4A156805F1340262609C
:10DC5000EA6A052B22612A6B2560E2616A6CA26088
:10DC6000EA6C62614FF00002A26119D011490968A3
:10DC7000A94209D12273D6B10023296BCA5CA52A17
:10DC800013D09B08238470BD032B2373F3D1FFF7BC
:10DC9000CBFCAB6A0BB102232373FFF771FDEAE7FC
:10DCA0002846FFF7F5FB2073E5E70133E6E7268416
:10DCB000E9E700BFA42500202DE9F84F0D680646CE
:10DCC0000C4617462DB300254FF0240B4B6801F18D
:10DCD00008085B6843454B6004BFCB684B604B68EA
:10DCE000D3F80CA063680BFB05615B6801229845C3
:10DCF000636008BFD8F8043005F1010508BF636010
:10DD00006368D3F80C903B464846FFF797FFCA4537
:10DD1000E8D12846BDE8F88F2DE9F0471746FFF710
:10DD200083FC1F4B05461B688B4237D80526002411
:10DD30004FF0140A4FF02408DFF86890013E08FB0A
:10DD4000045001220AFB0691FFF7B6FF0444002E9F
:10DD5000F4D1154B0222196808FB0450FFF7ACFF01
:10DD6000124B04441968022208FB0450FFF7A4FF79
:10DD70000444042208FB04500D49FFF79DFF0444AE
:10DD800008FB045003220B49FFF796FF044407B138
:10DD90003E60FFF7F5FC2046BDE8F0870024F8E779
:10DDA00014260020B0250020A8250020AC25002046
:10DDB0008C2600207826002008B9064B1868026BD4
:10DDC0000020135CA52B02D0C0F38F0070470130F8
:10DDD000F7E700BFA4250020014B1868704700BF7B
:10DDE000A4250020054B1B6833B1054B1B68002B95
:10DDF0000CBF0220002070470120704774260020CD
:10DE0000202600202DE9F0410446002835D0234D7E
:10DE1000C36A2A68D26A934237D214268269204F95
:10DE2000002AA8BF2A6806FB0373A2BFD26AC2F108
:10DE30000502826142699A4221D100F104084046FC
:10DE400000F049FC174B48B9E06A4643BA592AB971
:10DE500001211A68814022EA01021A602A681968C1
:10DE6000D26AE262012404FA02F008431860142026
:10DE7000414600FB027000F00BFC204603E02B68DB
:10DE8000DB6AC3620120BDE8F0812B68C06CDC6AEC
:10DE9000A0422CBF00200120F5E700BFA4250020F0
:10DEA000B025002028260020F8B5044608B9002037
:10DEB000F8BD1F4B1B68834204D040F67A711D48A1
:10DEC000F8F77CFB236D23B940F67B711948F8F70E
:10DED00075FB236DE16AE26C013B91422365E6D05C
:10DEE000002BE4D1261D304600F0F5FB124F134AFB
:10DEF00050B91421E06A41437B582BB901251368BE
:10DF0000854023EA05031360E36C1420C3F1050187
:10DF1000A161E3620124116804FA03F500FB0370B8
:10DF20000D433146156000F0B3FB2046C0E700BF4B
:10DF3000A42500207DDF0108B02500202826002030
:10DF4000F8B50D460446002845D0036D23B940F6C8
:10DF5000C9712148F8F732FBE16CE36A8D4238BFA2
:10DF60000D46AB4237D0236D012B34D11B4B1B68C0
:10DF7000A34204D140F6E4711748F8F71FFBA269E9
:10DF8000E36A002AE562A4BFC5F10505A561142571
:10DF9000134E626905FB03639A421CD1271D384664
:10DFA00000F099FBE26A0F4C40B9554373592BB905
:10DFB00001212368914023EA0103236001231420F7
:10DFC000216893400B4300FB026039462360BDE8A3
:10DFD000F84000F05DBBF8BD7DDF0108A4250020FE
:10DFE000B025002028260020044B1A681AB11968B1
:10DFF0000A6D01320A651868704700BFA425002029
:10E000002DE9F041224C1E4680460F461546FEF78C
:10E01000F1F9236893F8B830022B18D00121226857
:10E02000D2F8B43023EA0803C2F8B430236883F886
:10E03000B81066B13046FFF755F84FF0E0234FF0C7
:10E040008052C3F8042DBFF34F8FBFF36F8FFEF7DD
:10E05000EFF9FEF7CFF91DB12368D3F8B4302B6088
:10E06000236893F8B830022B03BF22680125D2F849
:10E07000B430002504BFBB43C2F8B430002223688B
:10E0800083F8B820FEF7D4F92846BDE8F08100BF38
:10E09000A4250020F8B50E4617461D46044620B9B3
:10E0A00041F219212F48F8F789FAFEF7A3F915B1C3
:10E0B000D4F8B4302B60022394F8B85084F8B83008
:10E0C000EDB2042F1AD8DFE807F00E030906150099
:10E0D000D4F8B4100E43C4F8B46004E0D4F8B430FB
:10E0E0000133C4F8B430012D12D00124FEF7A0F999
:10E0F0002046F8BD022DEED10024F7E7D4F8B43065
:10E100000133F0D041F24A211648F8F757FAEAE70E
:10E11000261D304600F0DFFA1420134AE36A116826
:10E120009D400D431560114A314600FB032000F06D
:10E13000AFFAA36A23B141F259210A48F8F73EFA2F
:10E140000B4BE26A1B68DB6A9A42CED94FF0E023A0
:10E150004FF08052C3F8042DBFF34F8FBFF36F8F82
:10E16000C3E700BF7DDF010828260020B02500207E
:10E17000A42500202DE9F843089F0D4691461E4630
:10E18000044620B941F28C213648F8F717FAFEF719
:10E1900007FAEFF311884FF0500383F31188BFF3B0
:10E1A0006F8FBFF34F8F16B1D4F8B43033600223B2
:10E1B00094F8B86084F8B830F6B2B9F1040F1AD800
:10E1C000DFE809F00E0309061500D4F8B4100D437A
:10E1D000C4F8B45004E0D4F8B4300133C4F8B43017
:10E1E000012E12D0012088F31188BDE8F883022E99
:10E1F000EED10020F7E7D4F8B4300133F0D041F28B
:10E20000CF211848F8F7DAF9EAE7A36A23B141F217
:10E21000DA211448F8F7D2F9134B1B68EBB9251D26
:10E22000284600F058FA01231049E26A0868934032
:10E23000034314200B6029460D4B00FB023000F015
:10E2400027FA0C4BE26A1B68DB6A9A42CAD901239F
:10E2500007B13B60084A1360C4E7084804F118019D
:10E26000EDE700BF7DDF01082026002028260020E2
:10E27000B0250020A4250020A42600206026002030
:10E2800010B5044608B9084B1C68FEF7B3F8002027
:10E2900094F8B830022B0ABF84F8B8000446012471
:10E2A000FEF7C6F8204610BDA4250020F8B50F4C97
:10E2B000FEF7A0F82568ADB90D4F0E4E384600F0B8
:10E2C000D9F9304600F0D6F90B4B2A461F600B4BAC
:10E2D0000C210A201E60FEF7ADFA206010B108493B
:10E2E000FEF76CFEBDE8F840FEF7A2B8DC26002081
:10E2F000B0260020C4260020A8260020AC2600203E
:10E3000055C70108914208B5416000610AD8D21A88
:10E3100083699A420DD2084B011D186800F0C4F9B8
:10E32000002008BD9A4201D2994202D2034B011D3E
:10E33000F3E70120F5E700BFAC260020A826002067
:10E3400007B5FFF7B3FF0C4B1B6843B90B484FF4FD
:10E350008971F8F733F9002003B05DF804FB084B2E
:10E36000C822019301230749009307480023FEF7C1
:10E370002BFF0028EAD0EFE7DC2600207DDF010834
:10E38000E02600205AC70108D5E400082DE9F04135
:10E3900080462C200D4617461E46FEF767F90446B8
:10E3A00088B125B94FF4B6710848F8F707F9FFF7B7
:10E3B0007DFF069BC4E90657C4F8008026626362AD
:10E3C000201D00F062F92046BDE8F0817DDF0108E4
:10E3D0002DE9FF410C4690461E46054620B94FF4F4
:10E3E000C3710F48F8F7EAF80E4F386878B1052C7A
:10E3F000CDE9014803950DDCFFF7F4FC002302286A
:10E4000014BF1A460A9A386801A9FEF737FA04B011
:10E41000BDE8F0810023324601A9FEF7E7FAF6E7EE
:10E420007DDF0108DC2600202DE9F04F85B006468F
:10E43000FFF702F9DFF88C800546D8F800308342F8
:10E440003DD94FF00009204FDFF880A03B681A68E3
:10E450005AB91F4A11681360012339602846336096
:10E46000C8F8005005B0BDE8F08FDB68DC68D3F871
:10E4700000B0211D0846039100F02DF9636A204683
:10E480009847E3690399012BE0D1A3695B449B455D
:10E4900005D238686360246100F006F9D6E70023EE
:10E4A0005A4619462046CDF80090FFF791FF002804
:10E4B000CCD140F272315046F8F780F8C6E700231D
:10E4C000CCE700BFD8260020A82600207DDF010869
:10E4D000AC2600202DE9F047624F634E86B03B68C2
:10E4E0001D68002D68D00024DB681D68FFF79CF8CC
:10E4F00003A8FFF799FF039B8246DFF87081002B8A
:10E5000078D1002C5AD1A8425ED3FFF739F93B6885
:10E51000DB68D3F80C9009F1040000F0DCF8D9F8BE
:10E520001C30012B15D1D9F818102B4652464846FD
:10E530002944FFF7E7FE60B123462A4621464846B4
:10E540000094FFF745FF20B94FF4F4713046F8F717
:10E5500035F84846D9F8243098470022D8F800000A
:10E5600003A9FEF7E7FA0028B9D0039B002BF4DBE0
:10E57000059C636913B1201D00F0ADF802A8FFF7F8
:10E5800053FF039B0546092BE7D801A252F823F05D
:10E59000FBE50008FBE50008FBE500085BE500087B
:10E5A0003BE600085BE60008FBE50008FBE5000829
:10E5B0005BE500083BE60008012497E72C4B1B684D
:10E5C0001C68B4FA84F464092246D8F80000A5EB6C
:10E5D0000A01FEF72BFDFFF7D3F80028BDD14FF05D
:10E5E000E0234FF08052C3F8042DBFF34F8FBFF3E9
:10E5F0006F8FB2E7FFF7C4F8AFE7A169049B02464B
:10E6000019442046FFF77EFE0028A6D0636A204604
:10E610009847E369012BA0D10023A2690499204601
:10E620000A4400931946FFF7D3FE002895D140F223
:10E6300001313046F7F7C2FF8FE7049BA36123B98E
:10E640004FF446713046F7F7B9FFA1692B462A46C9
:10E6500020462944FFF756FE7FE72046FEF708F8DC
:10E660007BE700BFA82600207DDF0108DC26002014
:10E67000AC2600204FF0FF3200F10803C0E902236E
:10E680004360036100230360704700230361704708
:10E6900043689A684B608A609A6851609960036821
:10E6A000086101330360704730B50C68631C0AD100
:10E6B00003695A684A6091608B6059600368086119
:10E6C0000133036030BD00F108021346526815683B
:10E6D000A542FAD9EDE70369D0E901128A605160D9
:10E6E0005968814208BF5A60002202611A68013AE3
:10E6F0001A60186870470000021E18BF012200212E
:10E700000148F8F771BD00BF00040240F9F7CCB929
:10E7100038B505460C460020FFF7EEFF45F08000B7
:10E72000FFF7F4FF2046FFF7F1FFBDE83840012076
:10E73000FFF7E2BF08B50120F8F746FB0A20F8F71B
:10E7400043FB0B20F8F740FB0720F8F73DFB0520C3
:10E75000F8F73AFBBDE808400420F8F735BB0000A5
:10E7600070B5204B04469D78EDB958B902211E487A
:10E77000F8F735FD23461A460221BDE870401A48D5
:10E78000F8F762BC012805D102211748F8F722FDED
:10E790002B46F0E7022823D102460146BDE870402F
:10E7A0001148F8F791BC012D14D138B904210E4855
:10E7B000F8F715FD002304211A46DEE7012804D1ED
:10E7C00004210948F8F706FDF4E7022808D10246BB
:10E7D0000421E3E76A21BDE870400448F7F7EEBE84
:10E7E00070BD00BFE4260020000002407DDF01086C
:10E7F00008B50020FFF7B4FFF8F71EFA0120FFF775
:10E80000AFFFF8F719FA0220FFF7AAFFBDE80840AA
:10E81000F8F712BA08B500210120F9F7C5F8012070
:10E82000FFF76AFF0023094819461A46F8F70CFC5F
:10E83000B5214020FFF76CFFA0214120FFF768FFC2
:10E84000BDE8084000210120FFF762BF000402403C
:10E8500010B5FFF76FFF0120FFF74EFF0023374889
:10E8600019461A46364CF8F7EFFB00210120F9F75C
:10E870009BF823787BB1002306211A462F48F8F72E
:10E88000E3FB06212D48F8F7A5FCF8F7D5F9192187
:10E890005820FFF73DFFFFF7ABFFFFF7BBFF6378A3
:10E8A0005BB1002304211A462648F8F7CDFB00236C
:10E8B0000D211A462448F8F7C7FB002201211F4802
:10E8C000F8F702FC00220A211C48F8F7FDFB0022A1
:10E8D0000B211A48F8F7F8FB002207211748F8F730
:10E8E000F3FB002205211548F8F7EEFB0022042176
:10E8F0001248F8F7E9FB0523022201210F48F8F737
:10E9000081FA052302220A210C48F8F77BFA052335
:10E9100002220B210948F8F775FA05230222072184
:10E920000648F8F76FFA094B1B782BB9BDE8104081
:10E93000BE210748F7F742BE10BD00BF00040240E9
:10E94000E42600200000024000080240E7260020E4
:10E950007DDF010882B00190064B9DF80620BDF8CE
:10E9600004109A7001221980034B1A7002B0FFF74D
:10E970006FBF00BFE4260020E72600201A4B10B529
:10E980005B78D3B10128194C18D104211848F8F745
:10E9900021FC0D211748F8F722FC23786BB10023E6
:10E9A00004211A461248F8F74FFB00230D211A469E
:10E9B0001048F8F749FB0023237010BD40B904212B
:10E9C0000B48F8F70CFC0D210A48F8F703FCE4E7C4
:10E9D000022204210648F8F777FB02220D210548A0
:10E9E000F8F772FB0123E7E7E4260020CC020020C1
:10E9F000000002400008024008B5FFF79BFEFFF749
:10EA0000F7FEFFF707FFF9F72BF8012200211F4857
:10EA1000F8F75AFB0220FFF7B1FF0220FFF7A0FE34
:10EA2000022201211948F8F74FFB02220A21174858
:10EA3000F8F74AFB02220B211448F8F745FB0222A3
:10EA400007211248F8F740FB022205210F48F8F78A
:10EA50003BFB022204210D48F8F736FB0C4B1B78D8
:10EA60001BB9E2210B48F7F7A9FD0B4B1B785BB1F3
:10EA7000002306211A460548F8F7E6FABDE80840E3
:10EA800006210248F8F7ABBB08BD00BF00040240F6
:10EA9000E72600207DDF0108E426002010B5064CA3
:10EAA000022220460021F8F70FFB2046BDE8104067
:10EAB00002220121F8F708BB00140240F8B5104CFF
:10EAC000D4F8803298472346002210F5617541F151
:10EAD0000006D3E90874B84271EB0404B8BFC3E977
:10EAE0000801D3E90674BD4276EB040402F1010289
:10EAF000B8BFC3E90656102A03F12803E9D1F8BDCF
:10EB0000F026002010B5044618B9BB210748F7F7D6
:10EB100055FD074BD3F880329847D4E90632984226
:10EB200071EB0202ACBF0020181A10BD7DDF010896
:10EB3000F02600202DE9F84F054628B9BDE8F84F2A
:10EB4000DC213148F7F73ABD0026304C33462246E7
:10EB5000117A0133A94208BF0136102B02F12802B5
:10EB6000F6D1002E4ED0062D03D940212648F7F7C6
:10EB700025FD274B53F83570002F41D1E72122485E
:10EB8000F7F71CFD7E431027DFF87C80237AAB4229
:10EB900031D163687BB32369012B03D1D021404677
:10EBA000F7F70CFDD4E9060150EA010322D0D4E9BD
:10EBB00008A9B0EB0A0061EB090108F023FC8346C9
:10EBC0002069013808F004FC0146584608F00CFDA5
:10EBD0008346304608F0FCFB594608F051FC594684
:10EBE00008F044FB08F038FE10EB0A0049F100037E
:10EBF000C4E906032661013F04F12804C6D101E0FF
:10EC0000012FBFD1BDE8F88F7DDF0108F02600207D
:10EC100074C901084FF47A73B0FBF3F341F658322C
:10EC2000A3F55223A3F6183393422DD81B4B1C4A4D
:10EC30000344934228D91B4B1B4A0344934223D9D4
:10EC40004CF24E32194B034493421DD9184B984253
:10EC50001CD903F5371303F5D863984218D903F587
:10EC6000122303F5F863984214D903F5122303F530
:10EC7000F863984210D903F5DB2303F5BA63984291
:10EC80008CBF062005207047002070470120704788
:10EC90000220704703207047042070473F373ACC6A
:10ECA0009E8601007F0F31CC3E0D0300AF312ACC90
:10ECB00040DA8E332DE9F04385B0E0B1D0E9039816
:10ECC0004FF47A710D4B4468D3F88C62037AB4FB2D
:10ECD000F1F4062B96BF0A4A0A4D52F823500778E2
:10ECE000FFF710FF3B46CDE901902A462146064832
:10ECF000CDF80080B04705B0BDE8F083F0260020D5
:10ED0000ACC9010862C701086FC7010870B5154C8E
:10ED1000054694F894320E4623B94FF49671124882
:10ED2000F7F74CFC25B940F22D110F48F7F746FCD8
:10ED300026B94FF497710C48F7F740FC0023094AB5
:10ED40001178A94202D15168B14206D00133102B8B
:10ED500002F12802F4D1002070BD282000FB0340FE
:10ED6000FAE700BFF02600207DDF01082DE9F04F13
:10ED7000DFF8B8B099469BF8943293B0924601916F
:10ED800023B940F241112A48F7F718FC0026FFF793
:10ED900095FEB0464FF0FF373446244DEB68019A9C
:10EDA000934218DBBAF1000F10D12846FFF7AAFEF4
:10EDB00080B3B84236D30ED1D4E90823D5E908018F
:10EDC000FBF701F9002818BF2C4604E00021284673
:10EDD000D0470028E9D10136102E05F12805DDD1F4
:10EDE000B9F1000F01D0C9F800707FB9B8F1010F77
:10EDF0000CD9384608F1FF31FBF7DEFA12AB03EB12
:10EE00008000282350F8404C03FB04B4204613B084
:10EE1000BDE8F08F12AB03EB880343F8406C08F1B8
:10EE20000108C6E707462C46D5E700BFF0260020BC
:10EE30007DDF0108000000002DE9F0470F46044681
:10EE400020B94FF4C2712048F7F7B8FB236923B902
:10EE500040F285111C48F7F7B1FBDFF87080D8F855
:10EE600080329847C4E9080105462069894608F0C0
:10EE7000AFFA394608F004FB394608F0F7F907F015
:10EE80008FFE0FA3D3E9002308F00CF807F0E0FB96
:10EE900008F078F9451949F10001C4E90651064620
:10EEA000384608F0B3FCD8F88C5202463346AC46DC
:10EEB00061680748BDE8F047604700BFAFF30080D6
:10EEC0000000000080842E417DDF0108F026002034
:10EED000B6C701082DE9F0410E461746054620B990
:10EEE0004FF4C8711348F7F769FB26B940F2911146
:10EEF0001048F7F763FB0021384608F07DFC20B985
:10EF00004FF4C9710B48F7F759FB4FF010080A4C42
:10EF10002378AB4206D16368B34203D13946204619
:10EF2000FFF78AFFB8F1010804F12804F0D1BDE829
:10EF3000F08100BF7DDF0108F026002008B5FFF753
:10EF400069FE003818BF012008BD00002DE9F0411E
:10EF50003E4D074695F894320E4694B023B94FF4CF
:10EF6000D9713B48F7F72AFB3046FFF7E7FF044625
:10EF700058B94FF47A71D5F89032B6FBF1F13548B3
:10EF80009847204614B0BDE8F08131463846FFF777
:10EF9000BDFE04460028F4D180462C4B5A683AB195
:10EFA00008F10108B8F1100F03F12803F6D1E8E7E2
:10EFB00095F894321BB977212548F7F7FFFA1FB966
:10EFC00078212348F7F7FAFA282200210DEB0200F6
:10EFD00009F080F83046FFF71DFE062804468DF83C
:10EFE000300003D940211A48F7F7E8FA0B966E462D
:10EFF00019488DF8287050F8343000EBC40042688E
:10F000000AACCDE90D230FCC0FC60FCC0FC694E888
:10F010000300282404FB0854EC46274686E8030036
:10F02000BCE80F000FC7BCE80F000FC796E803004D
:10F03000D5F88C3287E803004146084898472046B7
:10F04000FFF738FE207AFFF775FD9AE7F0260020DB
:10F050007DDF0108F6C7010874C9010825C8010849
:10F060000D4B10B593F89432044623B94FF4EA716E
:10F070000A48F7F7A3FA6CB163685BB10848FBF77D
:10F080004FF82046FFF716FE0023207A63602372B4
:10F09000FFF750FD002010BDF02600207DDF0108A5
:10F0A00046C80108144B2DE9F04193F89432054607
:10F0B0000F4623B94FF4F6711048F7F77FFA25B9D8
:10F0C00040F2ED110D48F7F779FA00260A4C04F5E5
:10F0D00020782378AB4208D16368BB4205D1204633
:10F0E000FFF7BEFF002818BF064628344445F0D17C
:10F0F0003046BDE8F08100BFF02600207DDF01082A
:10F100002DE9F041114F054697F8943223B94FF499
:10F11000FE710F48F7F752FA25B940F2FD110C487D
:10F12000F7F74CFA1026094C2378AB4204D16368F8
:10F1300013B12046FFF794FF013E04F12804F3D1F8
:10F14000D7F88C320348BDE8F0411847F02600207C
:10F150007DDF010856C801082DE9F04105460E463D
:10F160001746134C04F520782378AB4207D1626828
:10F170002AB100239F420BDC2046FFF771FF2834A1
:10F180004445F1D10024A74208DC0120BDE8F0810C
:10F1900056F823108A42F2D00133EBE7284656F89E
:10F1A0002410FFF7D3FE0028F0D00134EBE700BFB6
:10F1B000F0260020014B93F894027047F0260020BF
:10F1C00010B5074C2378FA2B04D94FF40D7105487C
:10F1D000F7F7F4F920780130C0B2207010BD00BFFD
:10F1E000E82600207DDF010884B070B504AC84E817
:10F1F0000F001C4C94F8941231B1D4F890321A4894
:10F20000BDE8704004B018474FF42672204604F55C
:10F21000207504AE08F05EFF0FCE0FC533682B607B
:10F2200013B9124BC4F89032D4F88C3213B90F4B87
:10F23000C4F88C32D4F8883213B1D4F884324BB984
:10F24000D4F88C320A4898470A4BC4F888320A4BE3
:10F25000C4F88432012384F89432BDE8704004B0CD
:10F26000704700BFF026002072C8010819A10008ED
:10F27000ABC80108398001082980010830B4002595
:10F280000E4BD3E9082452EA040C04D0121844EBC4
:10F290000104C3E90824D3E9062452EA040C04D08B
:10F2A000121844EB0104C3E906240135102D03F1C3
:10F2B0002803E6D130BCFFF701BC00BFF0260020D8
:10F2C00070B50446044E451814F8011B3046FAF791
:10F2D00027FFAC42F8D170BDF4D401082DE9F84302
:10F2E0000025DDE90878C0E9011216463946424694
:10F2F000C0E90335C0E90555C0E907550570456209
:10F30000044600F11C0904F0A5FA38B93146084852
:10F31000FAF706FF2B210748F7F750F943463A461C
:10F320004946204604F044FA2046BDE8F88300BF71
:10F3300010AC01087DDF010810B504461C30F1F760
:10F34000EAF804F11000F1F7E6F8204610BD0000DD
:10F3500070B5044690B00146924A01A805F029FA1A
:10F360002146914A04A805F024FA21468F4A07A8AD
:10F3700005F01FFA8E4A21460AA805F01AFA8D49AF
:10F38000204605F00DFA05468B48FAF7C9FEDDE97F
:10F3900001239B1A082B06D08848FAF7C1FEBF212B
:10F3A0008748F7F70BF9DDE904239B1A082B06D0F1
:10F3B0008448FAF7B5FEC3218148F7F7FFF8DDE985
:10F3C0000A239B1A102B06D07F48FAF7A9FEC72103
:10F3D0007B48F7F7F3F8DDE907135B1A102B0CD124
:10F3E00001234A1E01F10F0012F8016F002E18BF11
:10F3F00000239042F8D1002B53D07448FAF790FEC6
:10F400005DB37348FAF78CFE674A21460DA805F0F4
:10F41000D0F97048FAF784FE08210198FFF750FFF1
:10F420006D48FAF77DFE08210D98FFF749FF6B48FC
:10F43000FAF776FE10210A98FFF742FF6848FAF7BC
:10F440006FFE0D980A9A019900F0E8FF0DA8F1F7F8
:10F4500062F86448FAF764FE61E06348FAF760FE18
:10F460006248FAF75DFE0A99019800F035FF60489E
:10F47000FAF756FE042101980844FFF721FF5D4882
:10F48000FAF74EFE10215C48FFF71AFF5B48FAF7C7
:10F4900047FE10215A48FFF713FF5148FAF740FE84
:10F4A000D7E710220A9808F0DDFD564A44490028A3
:10F4B00008BF11465448FAF733FE002D40D04448A7
:10F4C000FAF72EFE384A21460DA805F072F94F488A
:10F4D000FAF726FE08210198FFF7F2FE4C48FAF7EA
:10F4E0001FFE08210D98FFF7EBFE4A48FAF718FEB9
:10F4F00010210798FFF7E4FE4748FAF711FE1021A4
:10F500000A98FFF7DDFE3648FAF70AFE0D98079BCA
:10F510000A9A019900F096FF0DA8F0F7FCFF304819
:10F52000FAF7FEFD0AA8F0F7F6FF07A8F0F7F3FFD9
:10F5300004A8F0F7F0FF01A8F0F7EDFF10B070BDE0
:10F540002948FAF7EDFD3548FAF7EAFD079A0A99D6
:10F55000019800F005FF2648FAF7E2FD0421019822
:10F560000844FFF7ADFE2E48FAF7DAFD10212248D5
:10F57000FFF7A6FE2B48FAF7D3FD10212A48FFF724
:10F580009FFE2A48FAF7CCFD10212948FFF798FE84
:10F590002848FAF7C5FD1A481021FFF791FE1048D8
:10F5A00058E700BFDFC90108E6C90108EEC9010834
:10F5B000F5C901085DBD0108FCC9010813CA0108AD
:10F5C0007DDF010823CA010834CA010844CA0108C2
:10F5D0005FCA010865CA010876CA010888CA01081D
:10F5E0007CDF01082FCB0108A8CA0108ADCA0108B9
:10F5F000DECA0108F0CA01086C0400201CCB010817
:10F600009C040020C8C901084ECB01086BCB01083F
:10F610007DCB010890CB0108B0CB0108FBCB0108E2
:10F6200034CC0108A0CC01087C040020B7CC010830
:10F630008C040020CECC01082DE9F04100259DF876
:10F640001870C0E90112C0E903353946C0E9055513
:10F65000C0E90755057045620446164600F11C08CE
:10F6600004F086F838B931460748FAF759FD2021E9
:10F670000648F6F7A3FF3A464146204604F066F8EE
:10F680002046BDE8F08100BF10AC01087DDF010815
:10F690002DE9F0410025069FC0E90112C0E90335BC
:10F6A0003946C0E90555C0E907550570456204466D
:10F6B000164600F11C0804F049F938B931460748EC
:10F6C000FAF72EFD20210648F6F778FF3A46414624
:10F6D000204604F01DF92046BDE8F08110AC010879
:10F6E0007DDF0108F0B50126044608270D468DB0E0
:10F6F000564B574A3146009602A8FFF79DFF02A9D4
:10F70000204605F03FFA02A8FFF716FE514BCDE95F
:10F7100000571A460DEB07000421FFF7DFFD0DEB44
:10F720000701204605F02EFA0DEB0700FFF704FE57
:10F73000EB19494A019700930DEB0700474B042151
:10F74000FFF7CCFD0DEB0701204605F01BFA0DEB92
:10F7500007001027FFF7F0FDEB190093404B042141
:10F760001A46019702A8FFF7B9FD02A9204605F045
:10F7700009FA203502A8FFF7DFFD3A4B3A4A009517
:10F780000421019702A8FFF7A9FD02A9204605F070
:10F79000F9F902A8FFF7D0FD0C230025334A0093A6
:10F7A0000221334B02A8FFF773FF02A9204605F0A0
:10F7B000E9F902A8FFF7C0FD2E4B2F4A314600960B
:10F7C00002A8FFF739FF02A9204605F0DBF902A8DD
:10F7D000FFF7B2FD294B2A4A0221009502A8FFF744
:10F7E00057FF02A9204605F0CDF902A8FFF7A4FDB6
:10F7F000244B254A0221009502A8FFF749FF02A9E0
:10F80000204605F0BFF902A8FFF796FD1F4B204ADE
:10F810003146009602A8FFF70FFF02A9204605F027
:10F82000B1F902A8FFF788FD07231A4A00930221C5
:10F83000194B02A8FFF72CFF204602A905F0A2F9F8
:10F8400002A8FFF779FD0DB0F0BD00BFE5CC0108BF
:10F850005DBD0108DFC90108E6C9010873CD0108D3
:10F86000F5C901088CCD0108EEC9010839BD0108B0
:10F87000FFCC010858CD01083CBD0108B6CD0108F8
:10F8800040BD0108F4CD010849BD01082FCE010893
:10F8900055DE010852BD01084BCE010810B5084CD9
:10F8A000D4F834321BB95C210648F6F787FED4F849
:10F8B00034020023BDE8104003222021FEF7EABBFA
:10F8C000D00200207DDF0108F0B51F461446C7B006
:10F8D00005460E46F122002109A808F0FBFB09AA03
:10F8E0001021384602F0ECFF204609F04DFC074697
:10F8F0001022002101A808F0EDFB102F3A46214606
:10F9000028BF102201A808F0BDFB09AA05A901A87B
:10F9100003F050F83246284605A908F0B3FB47B07B
:10F92000F0BD000037B50E4C0E4D94F82F30022B71
:10F9300012D194F82130012094F8F321D4F8F41175
:10F940000093082302F06CFF6B6B002098470423A0
:10F9500084F82D3003B030BDEB6A98470123F7E7F8
:10F96000D00200200CC60108044B5A7F22B993F83C
:10F97000330080F00100704700207047D002002063
:10F98000F0B570279DB005460E463A460021684600
:10F9900008F0A0FB082133460DEB010004AC0B4A34
:10F9A000FFF792FF334620461021094A08AEFFF7C1
:10F9B0008BFF94E80F0086E80F003A466946284618
:10F9C00008F060FB28461DB0F0BD00BF7ACE0108EC
:10F9D00082CE010808B50548FAF7A2FB044A92F85E
:10F9E000F831013382F8F83108BD00BF89CE010833
:10F9F000D00200200022024B83F8F821704700BF9C
:10FA0000D002002084B070B58AB00EAC84E80F003C
:10FA1000724C4FF410722546002120460EAE08F0BD
:10FA200059FB0FCE0FC596E8030014AB85E8030021
:10FA30000FCB04F1180585E80F000E9B0BB9684B3E
:10FA400023600F9B0BB9664B2360109B23B94FF4C7
:10FA5000C7716448F6F7B2FD129B23B94FF4C97120
:10FA60006048F6F7ABFD119B23B94FF4CB715D48AD
:10FA7000F6F7A4FD139B23B94FF4CD715948F6F75F
:10FA80009DFDA3690BB90323A36101F0D3FE94F894
:10FA9000203013B9012384F8203001F0C3FE94F81C
:10FAA000213013B90E2384F82130636A0BB94E4B11
:10FAB000636201F0ABFEFAF769FEC4F83002013868
:10FAC000033008D949486368984700200AB0BDE868
:10FAD000704004B07047002204210120FCF7AAFE08
:10FAE0000322C4F83C0200210120FCF7A3FEC4F865
:10FAF000380220B940F2C3113A48F6F75FFD002200
:10FB000004210120FCF796FEC4F83C0120B940F224
:10FB1000C7113448F6F752FD002204210120FCF7FA
:10FB200089FEC4F8400120B94FF4E5712D48F6F77D
:10FB300045FD4FF48163A4F80032002384F834308B
:10FB4000012384F80432FFF735FB05AD70B9A368D3
:10FB500022690593236807920893E2686368069216
:10FB60000993009395E80F00FFF73EFBFFF728FB92
:10FB700084F8320001F09EFE23681D4E07936368EF
:10FB800031460893236904960693E368059306F1CA
:10FB9000A00318468DE803000393F03695E80F00A4
:10FBA00002F0D8F80196A3694FF4CD720093114981
:10FBB00001231148FDF708FB012804D040F2EF11A2
:10FBC0000848F6F7FBFC002303220421D4F8340292
:10FBD000FEF760FA012084F8310077E7D0020020B8
:10FBE00019A100087DDF010808E6D333BDCE010866
:10FBF00014040020F0CE0108D500010810B50F4C08
:10FC0000D4F8343223B94FF4FC710D48F6F7D6FC22
:10FC1000002303220421D4F83402FEF73BFA42F217
:10FC20001071D4F83802FDF717F80023D4F8380221
:10FC30001A46BDE810401946FCF720BED00200204D
:10FC40007DDF010838B50E4DD5F8383223B940F2C2
:10FC500009210C48F6F7B2FC0021D5F83802FCF770
:10FC6000FBFF0128044608D10023D5F838021A46C4
:10FC70001946FCF703FE204638BD0020FCE700BF14
:10FC8000D00200207DDF010810B5FFF7DBFF68B16F
:10FC9000074C0023D4F8340203220821FEF7FAF9B6
:10FCA000D4F83402BDE81040FDF732BC10BD00BFEF
:10FCB000D0020020002307B54EF65E2201934EF6D7
:10FCC0006023411E91428CBF02461A46044B01A993
:10FCD000D3F84001FCF72EFF019803B05DF804FB58
:10FCE000D002002070B5FFF7ADFF1A4B28B15B685A
:10FCF000194898470024204670BDD3F83C01FDF711
:10FD000037F904460028F5D1014602F035F90646D8
:10FD10000028EFD0047001F08FFC054618B930467A
:10FD200002F07AF9E7E70D4A13680133136073B9FB
:10FD30001368013313606B60042328462B7001F0B5
:10FD40009FFC10B9284601F089FC6C68D3E7136862
:10FD5000F1E700BFD0020020F8CE0108882900207A
:10FD60002DE9F0418AB00446884615460193FFF715
:10FD700069FF20B1002738460AB0BDE8F0814D4E3A
:10FD8000D6F83C01FDF7F4F807460028F2D1002D23
:10FD90005DD1B8F1000FEDD12046414602F0ECF8FC
:10FDA00004460028E6D09DF80530002B52D00423ED
:10FDB0000370FFF70FFE0F2206A903A80AF006FE44
:10FDC0009DF804303BB10D23012202A903A88DF850
:10FDD00008300AF009FE9DF806303BB102230122EB
:10FDE00002A903A88DF808300AF0FEFD96F82E202F
:10FDF00096F82F30934203D196F83030934217D0C3
:10FE00002023022A18BF00228DF8083094F8783099
:10FE100002A90BBF43F0040343F001038DF809204E
:10FE20008DF8092003A8022284F878300AF0DCFD5E
:10FE300096F81432059996F8F0011944C9B201F008
:10FE4000B9FE804509D9204602F0E6F893E7E02D97
:10FE500090D8A1E702230370ADE7059A32B120469E
:10FE60000399D2B200F086FF0028ECD065772046D7
:10FE700001F0E2FB05460028E5D000230E4A83602E
:10FE800013680133136083B91368013313606B6027
:10FE9000022328462B7001F0F3FB40B9284601F0FD
:10FEA000DDFB73680548984765E71368EFE76F68FF
:10FEB00061E700BFD00200208829002024CF01087C
:10FEC000034B93F8141293F8F00101F073BE00BFD6
:10FED000D00200200E2808BF0120024BD87783F8FB
:10FEE000F0017047D0020020024B83F8200083F815
:10FEF000F1017047D0020020014B83F821007047C8
:10FF0000D002002008B5FAF7F7F9024BC3F8480110
:10FF100008BD00BFD0020020034630B5054C00F1FB
:10FF20001005224618685968083303C2AB421446CC
:10FF3000F7D130BD8C040020034630B5054C00F1EC
:10FF40001005224618685968083303C2AB421446AC
:10FF5000F7D130BD7C040020034630B5054C00F1DC
:10FF60001005224618685968083303C2AB4214468C
:10FF7000F7D130BD6C040020034630B5054C00F1CC
:10FF80001005224618685968083303C2AB4214466C
:10FF9000F7D130BD9C04002010B50446FFF7BCFF2C
:10FFA0002046FFF7C9FF2046BDE81040FFF7D4BF49
:10FFB00030B51025C3B0224CF122002105A808F06D
:10FFC00089F82A46002101A808F084F894F85B31EA
:10FFD00029468DF8053094F85A3105AA8DF8063077
:10FFE00094F8593104F5B6708DF8073094F858310B
:10FFF0008DF8083094F857318DF8093094F856315F
:020000040801F1
:100000008DF80A3094F855318DF80B3094F854314E
:100010008DF80C3002F054FC052305AA04F5C671D6
:1000200001A88DF8043002F0C5FC062305AA04F5EA
:10003000BE7101A88DF8043002F0BCFC43B030BDA5
:10004000D00200200246024B0068516803C370478B
:100050001C0400200246024B0068516803C370472D
:1000600024040020034630B5054C00F1100522465B
:1000700018685968083303C2AB421446F7D130BD43
:100080002C040020034630B5054C00F11005224633
:1000900018685968083303C2AB421446F7D130BD23
:1000A0003C040020014B9877704700BFD00200202D
:1000B000014B83F82E007047D002002038B504466B
:1000C00000680D46884203D008B101F0C7FA2560E8
:1000D00038BD000080B5FAF787F90123754DDFF8C8
:1000E000D881764F85F82D300A234FF0FF3100205C
:1000F000714AFDF785FF012864D1D8F80000430755
:1001000016D53B7833B1FAF78BFA0020FAF7DEFA0E
:1001100000233B70022385F82D300023D5F83802E8
:100120001A461946FCF7AAFB0020FDF75BFCDBE74B
:1001300010F0080621D03B787BB941F28830FAF7FD
:100140009BFA18B99F215E48F6F738FA5D48FAF72E
:10015000BDFA01233B70FFF7E5FB0020FEF790F8A6
:100160004FF4FA61D5F83802FCF776FD0028BBD1D0
:10017000A6215348F6F722FAB6E710F0200041D046
:100180003B78E3B195F82D30042B18D14E4C324614
:100190002146D5F83002FCF70DFE01280DD1237859
:1001A000072B2CD032462146D5F83002FCF7C2FC92
:1001B000012802D12046FAF78FFAFFF7B3FB00209F
:1001C000FEF75EF83B78002B8ED001F06BFA044608
:1001D000002889D00378012B1AD195F82C10AA6A2F
:1001E00001B192B9B2FA82F238485209F9F798FF90
:1001F000204601F0B9FA204601F030FA74E701F028
:10020000E3F9DAE7FEF73CF86EE701F027FAAC6AAB
:10021000032385F82D302378032B06D8012B19D81A
:100220008BB16B682A48984709E0043B012BF8D84A
:1002300028480021FFF742FF204600F037FE204605
:1002400001F00CFA03E0DA211D48F6F7B7F9FFF7E1
:1002500069FB49E71F482146FFF730FFFFF784FBA2
:1002600068B101F031FA044618B9E6211448F6F7EE
:10027000A5F902232046237001F050FAE7E701F0C8
:1002800023FA064618B9ED210D48F6F797F93146DD
:10029000204600F001F9737E53B14FF47A70FDF7F8
:1002A00023FB3146204600F0F7F87368002BF2D0AC
:1002B0003046E1E7D00200209C2900208C29002054
:1002C0007DDF01089DF80008902900203ECF01083D
:1002D0007ECF0108F802002010B50430C6B00C46ED
:1002E000FFF710FE1C4B0DF1050203F10C0153F852
:1002F000040B8B4242F8040BF9D11B8810211380A8
:1003000000238DF81330022309AA20468DF804300B
:1003100002F0D6FA09AA05A901A802F04BFB05A82C
:10032000FFF72AFE012309AA102120468DF8043088
:1003300002F0C6FA09AA05A901A802F03BFB05A82C
:10034000FFF72AFE4FF48872044B9A83102283F839
:10035000442146B010BD00BFA2CF0108D00200204A
:1003600030B50430C7B00D461446FFF7CBFD294B1E
:100370000DF1050203F10C0153F8040B8B4242F816
:10038000040BF9D11B882846138000238DF8133005
:100390000223012509AA10218DF8043002F090FAF9
:1003A00009AA05A901A802F005FB05A8FFF7E4FDCD
:1003B00009AA102120468DF8045002F081FA09AAFA
:1003C00005A901A802F0F6FA05A8FFF7A5FD032389
:1003D00009AA05A901A88DF8043002F0EBFA05A8D6
:1003E000FFF7AAFD042309AA0DEB030005A98DF868
:1003F000043002F0DFFA05A8FFF7AEFD40F211125B
:10040000054B9A83112283F8FD5183F8442147B0AC
:1004100030BD00BFA2CF0108D002002038B50D4684
:100420001446FFF70FFE2846FFF714FE2046FFF79D
:1004300019FE2046FFF726FE1022014B9A8338BD95
:10044000D002002070B50E4615461C46FFF7FAFD97
:100450003046FFF7FFFD2846FFF704FE2046FFF772
:1004600011FE1122024B9A83BDE87040FFF7A0BD38
:10047000D002002010234168064A106C884202D145
:1004800092F83C0020B9013B02F11002F5D1184668
:10049000704700BFD00200202DE9F04306460C460D
:1004A00087B019B918216748F6F788F816B133787C
:1004B000022B03D01A216348F6F780F833691BB981
:1004C0001B216048F6F77AF833691B78042B05D0B6
:1004D000022B03D01D215B48F6F770F833785A4D94
:1004E00063700023D5E97C870393584A95F8F1118E
:1004F00095F8320003ABFEF739FC814620B90123A1
:10050000237007B0BDE8F083039B33B101F0D2FB49
:1005100003232370039B6360F3E7B3680133012B6C
:10052000B36011D1D5F8E42130690132C5F8E42176
:10053000B5F8FE2185F82C300132A5F8FE2100F037
:10054000D3F8306900F036FCD5F8482133695A6099
:10055000D5F8E4215A8195F8F92142B1002285F8B5
:10056000F9211A7A42F004021A72B5F8FA21A3F8B6
:100570007A20484601F0C6F9014695F8F031306915
:100580004FF47A7C80F87C3080F87D1095F8042256
:100590004FF0000902F00F02012A38BF012205AB1B
:1005A00005EB0111019304AB00933C3102FB0CC33A
:1005B0000CFB02F2CDF8109000F0DAFE00289ED07D
:1005C000FDF73AF8F060D4F8A00084F8009008B184
:1005D00001F022FD049B0598C4F8A0302246314664
:1005E000C4F80A001A4800F05BF88022316904F16F
:1005F000200007F047FD4FF0000CC4E9048784F8A1
:1006000000C095F833300598C4F888C0C4F80A00D3
:100610002376B26895F80232D4F8A0109A4200D23C
:1006200061B184F819C085F82CC0003918BF0121C8
:100630000091617E0748F9F773FD62E7012060765B
:10064000F3E700BF7DDF0108D00200207504010838
:10065000F8020020B1CF010808B5104A10B10023FC
:10066000A2F8FE31937FBBB1B2F8FE3192F80012CE
:100670008B4211D992F801225B1A93FBF2F102FB33
:1006800011334BB901F0DEF830B901F0E9F818B9CF
:10069000BDE8084001F0F4B808BD00BFD00200205A
:1006A00070B5D2F8A0400646154674B10021204628
:1006B00001F080FBFFF79EF92378052B01BF012392
:1006C00086F8D1316389A6F8D2312046FFF7C4FFFE
:1006D0002046D5F80A1000F0A3FB24B1237A5B076B
:1006E00044BF01232B7270BD134B10B49A7F02B329
:1006F000027A42F00102027293F8F011DA7F91421D
:1007000008D193F83C40A4B193F84C408CB193F8D5
:100710005C4074B1B3F8FE4193F800329C4208D9B2
:10072000914206D0037A10BC43F002030372FFF734
:1007300051B910BC704700BFD0020020431EDBB28D
:100740001F2B11D80D4A0A28D35C0ED8012202FAB9
:1007500000F010F4A46F08D0094A92F814221A4449
:100760000E2A02DD002070470023064A1078184444
:100770000E28CCBF00200120704700BF6DD00108BB
:10078000D0020020AF29002010B504782046FFF7E2
:10079000D5FF78B1084A09481378C454013313705F
:1007A00041B1074A92F81432D118013381F8054259
:1007B00082F8143210BD00BFAF290020A02900200C
:1007C000D00200202DE9F04F002593B0CDE90A12A8
:1007D0009DF87090A34E059006934D4502D313B03B
:1007E000BDE8F08F069B5C5D5F192046FFF7A6FF12
:1007F000019028B99C4813B0BDE8F04FF9F790BCC0
:10080000631E1F2B00F29C82DFE813F020009A0287
:100810002C004C0270015501BB013A024C02E2016E
:100820009A024E023201640266029A029A029A0207
:100830009A029A029A029A029A029A029A029A02D8
:100840009A029A029A029A029A028702A9EB050377
:10085000DBB2012B4FF0000400F0008186F8FD416F
:100860000224FBE04FF0000BA9EB0503DBB203937E
:1008700007235C468DF83C30039A231D934202DA2D
:100880003B5D032B11D0BBF1000F05D09DF83C3030
:100890006FF300038DF83C309DF83C30072B40F09F
:1008A000CF800024DFF8C481C3E03B19D3F8018076
:1008B000053408F00F030893C8F303130493C8F337
:1008C0000F230993C8F30313062B4FF0000AE4B279
:1008D000CDF8408003D908F0F003F02B35D14FF666
:1008E000FF71C8F3076303F07003C8F30F22602B96
:1008F00008BF0A46002307925A4A02930799D8B2C2
:100900000D920C9301F06EF8DDE90C32014698B1BE
:10091000106C88B106EB031C9CF844C004984FEAA5
:100920001C1E0CF00F0C844506D80298DDF810C090
:10093000E64528BF084602900133102B02F1100251
:10094000DCD1029B0BB14FF0020A089B072B05D9A3
:100950009DF8403003F00F030F2B01D14AF0040A39
:10096000C8F3076808F07008B8F1600F0AD14AF0C0
:10097000010AB8F1000F0ED0019BB8F1600F18BF4B
:100980009B4608E0B8F1000F40F0DC81099801F0C7
:1009900007F80028EBD19DF83C300AF0070A23F055
:1009A000070343EA0A0A8DF83CA065E73B19D3F830
:1009B00001A09DF83C30053403F00703072BCDF868
:1009C00040A0E4B235D19DF84030C3F3031186F85E
:1009D000F0110AF00F010F294FEA131205D0002978
:1009E0003ED003F00F0386F8F1319DF84310CAF3AF
:1009F0000F20C1F3021100F0FBFF20B940F2751186
:100A00004046F5F7DBFD96F84431102B09D11AF07A
:100A1000706F01BF01229DF8433062F303038DF82C
:100A200043309DF843301A0703D0C3F3030386F81D
:100A30000232039A231D9A4202DD3B5D032BB5D09F
:100A400054B10323002110A88DF84030FFF79CFE1D
:100A500000210FA8FFF798FE01F02CF92C443FE08D
:100A60000123C0E7D0020020EECF01087DDF01089E
:100A7000A9EB0503DBB2052B40F26081781CF9F786
:100A800042FC002397F905209A42ACBFAF4AB04A16
:100A9000801843F1000296F8043218180B9B42F1BB
:100AA0000002022B02D1013042F10002059BC3E992
:100AB0001C020624D2E7062300210FA88DF83C3043
:100AC000FFF762FE0A9B002103F01F03A1488DF887
:100AD0004030FFF759FE002110A8FFF755FE6C1CAF
:100AE000E4B2A5423FF47BAE254676E6A9EB0503CA
:100AF000DBB2042B4FF0000240F22081D7F8013026
:100B00008DF83820C3F30211DAB210930B46052991
:100B10009FBF9DF8383086F8F21143F004038DF83A
:100B20003830C2F3030302F00F02062A9CBF86F896
:100B3000F3319DF838300DF141009CBF43F00203C2
:100B40008DF838306427F9F7E0FB47433846FEF765
:100B5000F5F99DF8383088B1C6F8F47143F0010317
:100B60008DF8383005230FA801218DF83C30FFF7B0
:100B70000BFE01210EA8FFF707FE6FE760F30003ED
:100B8000EEE7A9EB0503DBB2052B40F2D780D7F8DF
:100B900001007B7910900DF141008DF8443000F098
:100BA000A7FE9DF8442001469DF8400000F0BEFEDF
:100BB0008DF8380001F07EF807230FA800218DF88A
:100BC0003C30FFF7E1FD00210EA8FFF7DDFD70E7E7
:100BD000A9EB0503DBB2042B4FF000047FF63EAF18
:100BE000D7F801300DF1410010938DF8384000F036
:100BF0007FFE044602469DF840105748F9F790FAE8
:100C00002046FEF79BF928B19DF8383043F00103E8
:100C10008DF838309DF840300F2B2FD80133DAB2E1
:100C200006EB031393F82C1006EB02122C3239B1A9
:100C30001B6B2BB19DF8383043F002038DF8383030
:100C40009DF83830012103F00303032B4FF00A0312
:100C500008BFD4600FA88DF83C30FFF795FD012147
:100C60000EA8FFF791FD9DF838103C48C1F34002F3
:100C700001F00101F9F754FA0524EFE60022DFE75D
:100C8000A9EB0503DBB2012B58D07B78012103F0DF
:100C90000F0386F8043208238DF8403010A8FFF7C0
:100CA00073FDDDE5AC1C1BE7A9EB0503DBB2012BF3
:100CB00044D001237A78110902F00F0203FA01F1FE
:100CC000934086F801320C2386F800128DF84030EC
:100CD0000021E3E7EC1C03E7A9EB0503DBB2012BE2
:100CE0002CD0B3687C789847012223090A3302FA92
:100CF00003F3C6F820320F23C6E9860104F00F047F
:100D0000002110A8C6F824428DF83C208DF8403010
:100D1000FFF73AFD00210FA8C1E7A9EB0503DBB2FD
:100D2000012B0BD07B780BB1022B07D196F830202A
:100D30009A423FF495AD86F8303091E500248DE677
:100D40002C46CEE6DDF804B025E600BF6E3DD51298
:100D50006F3DD512D304002025D0010844D00108EE
:100D600038B10078032803D0431F584258417047D8
:100D700001207047037A70B504460C301E0900EB61
:100D8000131002EB13130F2B154609DC07F07AF949
:100D90000120237A05EB131565F30713237270BD49
:100DA000C6F10F0207F06EF9237A002043F0F0033A
:100DB0002372F4E773B5134E04463278124DC2B174
:100DC0001249FFF7D7FF0F220021104807F082F9E0
:100DD0000023337095F8FD314BB1012302222046E8
:100DE00001A98DF804308DF80530FFF7C3FF02B07C
:100DF00070BD95F81422002AECD005F20521FFF70A
:100E0000B9FFE7E7AF290020D0020020A029002089
:100E1000024B00F00F0083F804027047D00200205C
:100E2000F0B585B00446039110B3FFF799FFF8B110
:100E30000020144B9DF90E1083F8050283F814026C
:100E4000207A93F81EC09DF80F20677F257F060942
:100E5000BCF1000F05D010F0010018BF012083F88D
:100E6000FC013EB1009604F10C032046FFF7AAFCFA
:100E700005B0F0BD002FFBD1002DF9D00095A36E79
:100E8000F3E700BFD002002003234168064A106C3C
:100E9000884202D192F83C0020B9013B02F11002D5
:100EA000F5D11846704700BFD00200202DE9F04769
:100EB000054686B018B10378043B012B03D91B21EA
:100EC000B548F5F77BFB2B690BB11B781BB11C21D7
:100ED000B148F5F773FBB14C94F8F161D4E97C8724
:100EE00000F0A0FC00F0A6FC002331460393AC4ABE
:100EF00094F8320003ABFDF739FF28B9284600F01B
:100F000033FC06B0BDE8F08700F0FCFC04EB0019F0
:100F1000039809F13C0998B100F0CCFE00F0D4FB35
:100F2000044618B938219C48F5F748FB2B78204631
:100F3000637003232370039B636000F0EFFBE0E723
:100F4000AB680133AB60227F102A3AD1012B0AD162
:100F5000D4F8E4314FF6FF710133C4F8E431F9F706
:100F60002BFAA4F8DC01B4F8DC310133A4F8DC314D
:100F700000262A69B4F8DC3104969382894B03CBAE
:100F8000D06011612A69103B03CB05AB91605060C2
:100F900094F8F3A184F8F361019304AB009341F258
:100FA000883241F270734946286900F0E1F9B0B91E
:100FB000284600F0D9FB049801F02EF884F8F3A13C
:100FC0009FE7112A06D1636904F5A6709847A4F833
:100FD000DC01CDE74B217048F5F7F0FAC8E7049B38
:100FE00084F8F3A113B11A78012A06D0284600F03C
:100FF000BBFB049801F010F883E7227F102A00F071
:101000009480112A40F08D8093F82230049AD168A0
:1010100002F15306C4F8481102F1630E002B00F0F0
:101020008680112384F844313346DFF87C91CC4626
:10103000186859680833ACE803007345E146F6D1F7
:10104000DFF868E102F1230302F13309F44618687E
:1010500059680833ACE803004B45E646F6D1DFF8A3
:1010600050E102F14309F446186859680833ACE8C6
:1010700003004B45E646F6D1DFF838E1F446186840
:1010800059680833ACE80300B342E646F6D19368EA
:10109000A363137CC3F3030384F8F331137CC3F31A
:1010A000021384F8F231507CFFF7B2FE002394F86B
:1010B0002E20049812F0FD0F00F1120018BF84F8E2
:1010C0002E30C4E97A33C4F8E43184F82F3084F840
:1010D000303000F0CDFC00F0EDFD012384F833301A
:1010E00000F0F2FA064618B9CB212B48F5F766FA5C
:1010F0008022296906F1200006F0C4FF0023049A2B
:101100000598C6F8A02094F83320C6E90487C6F8ED
:101110000A00C6F88830327633702B783046737008
:101120000BE77D211C48F5F749FA33466EE710239B
:1011300084F844313346DFF870C066461868596851
:10114000083303C67345B446F7D102F1230633468C
:10115000DFF8589002F1330ECC46306871680836DB
:10116000ACE803007645E146F6D11E46DFF8409034
:10117000CC46306871680836ACE803007645E14635
:10118000F6D1DFF830C0664618685968083303C6E0
:101190007345B446F7D17AE77DDF0108D00200201D
:1011A000890E0108240400209C0400208C040020E7
:1011B0007C0400206C0400202DE9F04385B0064635
:1011C0000C468DF80F202BB1012200200DF10F01EC
:1011D000F9F760FEFCF730FA1E4B1F4DDFF87C80FC
:1011E0009DF80F109B6A07462046984741F28832C7
:1011F0002946D8F83002FBF79DFC044600B32B7853
:10120000012B21D12846AC68F9F766FA4FF47A70C1
:10121000A4EB070909FB000006F0DAF87168024642
:1012200098F83200FDF756FE00F044FD3B46CDE94C
:101230000049D8F8005072689DF80F100848A84778
:10124000204605B0BDE8F0832846F9F745FA0024AA
:10125000F6E700BF0CC60108BC290020D002002020
:101260008DD001082DE9F84FDFF8E8B01E46DBF815
:10127000343005468946144640F6B8379847DFF8BB
:10128000D8A0DFF8D8804FF47A7307FB05F2324913
:10129000B2FBF3F2D8F83002FBF74CFC28B9DBF8CC
:1012A000303098474FF0FF302DE09AF80030072B90
:1012B00007D15046F9F710FA4FF47A65F9F778FD3F
:1012C000E1E7032BDBF830701FD1DAF804502879FE
:1012D0002968844228BF04464846224606F0D2FECA
:1012E000D8F8008095F90830B5F90620A9881C487F
:1012F000C0471EB1EB8833802B7AB3701648F9F7DC
:10130000EBF9B8472046BDE8F88F042B0CD1124802
:10131000F9F7E2F9B847D8F80040FCF78DF9014633
:101320001048A0470020EEE7052B0AD10A48F9F73C
:10133000D3F9B847D8F80040FCF77EF901460A48CF
:10134000EFE7F5210948F5F739F90348F9F7C4F94A
:10135000B847A7E70CC60108B0290020D00200203A
:10136000C0D00108EAD0010802D101087DDF0108E0
:101370002DE9F04F8E4CC9B00E4691469846FF229B
:1013800094F8443108A9539F029000F05DFE824614
:1013900018B9002049B0BDE8F08F94F8F01194F826
:1013A000F25172688D4298BF4D1B08468CBF0025D4
:1013B000EDB2D4F800B00592049100F0A9FB0390BF
:1013C00094F8F10100F0BAFBDDE90412039B0090F0
:1013D0007848D847F2682846D4F800B0039200F065
:1013E00097FB29460346039A7348D84794F8F311AC
:1013F000D4F8F4210846D4F800B00492039100F028
:1014000087FBDDE9031203466C48D8474246236850
:1014100049466B4898470121029800F0CBFC94F8AC
:1014200021300020009394F8F13194F8F021716894
:1014300001F0F6F952460023304608A9FFF7BCFE3A
:1014400082460028A5D0029B594C93F8783013F0BF
:10145000050F09D013F0040318BF022394F82F20BE
:101460009A4218BF84F82F30FF22002108A806F006
:1014700031FE94F821302A460093F16808230120B8
:1014800001F0CEF9A9F1140005F068FB44A3D3E9FB
:10149000002305F0DDFB05F075FE054609F2AB20E3
:1014A00005F05CFB40A3D3E9002305F0D1FB05F078
:1014B00069FE8146A8F1140005F050FB38A3D3E97A
:1014C000002305F0C5FB05F05DFEA0F114034B45BC
:1014D00094BFC5EB030BC5EB090B4FF47A7909FBFD
:1014E00005F10646B1FBF9F107A8CDF81CA0FCF701
:1014F000BBF9FF223B46584608A9FFF7B3FE421C42
:1015000005463FF446AF00281ADD2468FCF794F83E
:101510005346024629462B48A0470FB10123FB70D2
:101520000023529A9D42136008DD214BE9B293F8E3
:10153000442108A801F008F9529B1860012029E70E
:1015400094F821300120009394F8F3210823D4F873
:10155000F41101F065F909FB06F107A8B1FBF9F1F7
:10156000CDF81CA0FCF780F908F2AB2005F0F6FAE4
:101570000DA3D3E9002305F06BFB05F003FE3B460A
:10158000FF2208A9801BFFF76DFE431C05463FF4B0
:1015900000AF0028C4DD002FC2D00223BFE700BF88
:1015A0000AD7A3703D0AEF3FA4703D0AD7A3F03FCE
:1015B000D002002018D101084AD1010870D10108D9
:1015C00096D10108B1D1010830B5C3B06B46FF22F6
:1015D0004FF47A6002A9FFF745FE041E24DD0023C4
:1015E000144D0193D5F8482195F84431E1B202A891
:1015F00000F06CFE03460190B0B10278052A01D0DC
:10160000032A14D11846002100F0D4FB0198FFF7FB
:1016100023F8DDE90010FFF703FC00230122D5F8D1
:101620003C0201A9FBF72AF9204643B030BD00F087
:10163000F3FCF9E7D002002038B5074B0546DB681C
:1016400014209847044620B11422002106F042FDE0
:101650002561204638BD00BFD002002010B50446E9
:1016600050B1006900F0D8FC00232361034B2046F1
:10167000BDE810401B69184710BD00BFD002002014
:10168000002307B5019006481A4601A9D0F83C018D
:10169000FBF7F4F8431E5842584103B05DF804FBD1
:1016A000D0020020002307B50193064B93F83420A5
:1016B00022B9D3F83C0101A9FBF73CFA019803B029
:1016C0005DF804FBD0020020064B10B5A820DB68B3
:1016D0009847044618B1A822002106F0FBFC2046DA
:1016E00010BD00BFD002002010B5044698B1D0F85C
:1016F000883013B1203000F079FCD4F8A00020B17C
:1017000000F08AFC0023C4F8A030034B2046BDE85B
:1017100010401B69184710BDD00200201FB5104CA7
:101720000190D4F84001FBF735FC024640B9D4F8EB
:10173000400103A9FBF7FEF910B10398FFF7D4FFAE
:101740000023D4F840011A4601A9FBF797F820B905
:101750004FF4BC710348F4F731FF04B010BD00BF73
:10176000D00200207DDF010838B50546FFF7ACFF49
:10177000044620B940F27D110548F4F71FFF01230C
:1017800023702B7820466370BDE83840FFF7C6BF52
:101790007DDF010810B50D4C031D04EB0313197117
:1017A0009A600123013004EB0010026380F82C30B2
:1017B000114694F83200FDF7C9FB28B9BDE8104086
:1017C0000B210348F4F7FABE10BD00BFD002002081
:1017D0007DDF01080C4B014670B4102000221D462D
:1017E00093F83C401CB11E6C8E4208BF2246013863
:1017F00003F11003F4D122B995F8320070BCFDF763
:1018000051BC70BC704700BFD0020020044B93F85D
:10181000222083F8F3215A6AC3F8F421704700BFED
:10182000D0020020024B93F8202083F8F12170476A
:10183000D0020020024BDA7F83F8F021704700BF0E
:10184000D0020020054B93F8202093F8F11191422B
:101850003ABF012083F8F12100207047D002002018
:10186000064A92F8F031D17F99423DBF03F1FF3330
:10187000012082F8F0310020704700BFD002002024
:1018800010B5502400202146074AFFF783FF214668
:101890000120064AFFF77EFF2146BDE810400220E6
:1018A000034AFFF777BF00BFA027BE33E034C13340
:1018B0002042C43310B50D4CFFF7A8FF94F8320056
:1018C000FDF71EFCFFF7DCFF03225020002104F18E
:1018D00074030132102A187043F8041C596003F88D
:1018E000081C03F11003F4D110BD00BFD00200208A
:1018F000437882781B02007843EA02430343642062
:1019000058437047002310B54168074A146CD8B299
:101910008C4202D192F83C402CB90133102B02F1D9
:101920001002F3D1002010BDD00200202DE9F041BB
:101930000546EB1E0C2B0E4617464FF000000CD848
:1019400069B9164B013503EB0515286B85F82C108A
:10195000FFF740FF4FF003002E63BDE8F081C7F3AF
:101960000314062C08468CBF00240124FDF7E6FA78
:1019700044EA400404F00304032C2046EDD1074B55
:10198000324603EB0513D3F8408039462846FFF76B
:1019900001FF4046FFF71EFF2046DEE7D002002091
:1019A000002110B50C460C4BC20707D51C6C24B99E
:1019B0000A48F8F7B5FB204610BD01240131102973
:1019C0004FEA500003F11003EED1002CF3D104488C
:1019D000F8F7A6FBEFE700BFD0020020DCD101083A
:1019E000F8D1010841FA00F000F001007047000052
:1019F0004FF6FF73062908BF184600232DE9F04172
:101A00001A4C154627461A469E4690B0266CDEB103
:101A100040FA03F107EB031C9CF844C00CF00F08DC
:101A2000A84502D8B5EB1C1F10D984F83CE001335F
:101A3000102B04F11004E9D1694697F83200FDF744
:101A40008BFB10B0BDE8F0813146E3E701F0010106
:101A500084F83C100029EAD010A901EB820102F1C0
:101A6000010C41F8406C5FFA8CF2E0E7D0020020F4
:101A700038B50446FFF73CFF0546FDF75FFA28B18D
:101A80002A464FF050010320FFF784FEE01CFFF7C9
:101A90002FFF0546FDF752FA28B12A464FF05001B4
:101AA0000420FFF777FEA01DFFF722FF0546FDF794
:101AB00045FA28B12A464FF050010520FFF76AFE8B
:101AC00004F10900FFF714FF0546FDF737FA28B1C6
:101AD0002A464FF050010620FFF75CFE04F10C008F
:101AE000FFF706FF0446FDF729FA38B12246BDE8A4
:101AF00038404FF050010720FFF74CBE38BDC31FE0
:101B0000052B9ABFC0F10C00C0B20E207047000038
:101B100007289ABF014B185C00207047C6D2010805
:101B2000052804D90628034818BF0020704702483A
:101B3000704700BF90D0030048E80100072810B5A7
:101B4000044604D940F277110348F4F737FD034BFC
:101B500013F9240010BD00BF7DDF0108D0D20108B9
:101B6000142808B506DD12484FF4BE71F4F726FDBF
:101B7000082008BD02280EDD04280EDD06280EDD33
:101B800008280EDD0A280EDD0C280EDD0E28CCBF3D
:101B900000200120EDE70720EBE70620E9E705201C
:101BA000E7E70420E5E70320E3E70220E1E700BFE1
:101BB0007DDF01080F2938B505460C4604D940F2EF
:101BC000A7111348F4F7FAFC0F2D12D8DFE805F03F
:101BD0000808080B0E0E0E0E1111111111111D1D0A
:101BE000C4F1330038BDC4F17300FBE7C4F1F20067
:101BF000F8E740F2BF110648F4F7E0FC4FF4E0715B
